:100000000C940D120C942C120C942C120C942C1297
:100010000C942C120C941D140C94B3150C942C12EB
:100020000C942C120C948C1A0C942C120C942C12F0
:100030000C942C120C942C120C94232F0C942C1234
:100040000C942C120C944D170C94C4160C94E113C0
:100050000C942C120C9420230C942C120C942C1223
:100060000C942C120C942C120C942C120C942C1218
:100070000C942C120C946A2E0C944C160C94721541
:100080000C942C120C94137A0C942C12322E302EC9
:100090003000696E636F6D70617469626C652048D1
:1000A000570020202530325800204D430045617311
:1000B00079436F6E74726F6C005F03AF01D7006B92
:1000C00000470035001A001100010203171804054B
:1000D00006151107080916120A000B0C13100F0E53
:1000E0000D14040E1F0E0E0E0E000E0E0E0E1F0E21
:1000F0000400040E1F001F0E04000004040400107E
:10010000081300100B1300130B1300010219000158
:100110001A1900191A19080C1E1F1E0C08000206D5
:100120000F1F0F0602000E11111F1B1B1F001F0ABD
:100130000A0A0A0A1F001C101810160505050C17DC
:10014000141714170C00040A110A0A0E00001C10E0
:100150001812160202071C101816110204071C10B0
:100160001816110201061C101815150701010000D0
:1001700000171515151712121212120000000000B8
:1001800000171117141717111311170000000000A2
:100190000015151711111714171117000000070586
:1001A00005050505050707070707070707070305EF
:1001B00009121418100003070F1E1C181000000667
:1001C00009121412090600060917170906001F1163
:1001D0001F001F111F001F111F001F1F1F001F1FC7
:1001E0001F001F111F001F1F1F001F1F1F00040ED5
:1001F0001F04041F0E04010101050D1F0C0411044E
:100200000A11111F1100110E111111110E000A0017
:10021000111111110E000E11111611111610001CE2
:100220001F1F1F131010001C13111D131010001896
:10023000171119171010001F11111F101010C303F0
:10024000F333CF0FFF3F00C030F00CCC3CFC03C3B6
:1002500033F30FCF3FFFAAC08030F0B020E0A00CF6
:10026000CC8C3CFCBC2CECAC08C88838F8B828E82E
:10027000A803C38333F3B323E3A30FCF8F3FFFBFA1
:100280002FEFAF0BCB8B3BFBBB2BEBAB02C2823216
:10029000F2B222E2A20ECE8E3EFEBE2EEEAE0ACA12
:1002A0008A3AFABA2AEA0040609770486858784457
:1002B0006454744C6C5C7C426252724A6A5A7A464C
:1002C0006656764E6E5E7E41615171496959794537
:1002D000659F754D6D5D7D436353734B6B5B7B47D2
:1002E0006757774F6F5F7F1018141C121A161E1174
:1002F00019151D131B171FD0D8D4DCD2DAD6DED1C6
:10030000D9D5DDD3DBD7DF9098949C929A969E91B5
:1003100099959D939B505504060507C4C6C5C7848F
:1003200086858734363537F4F6F5F7B4B6B5B72495
:10033000262527E4E6E5E7A4A6A5A701C18131F1BA
:10034000B121E1A10DCD8D3DFDBD2DEDAD09C989D9
:1003500039F9B929E9A9206D332020200000204D6A
:100360004D4920200000204D4D0220200000204457
:100370004343202000002053544F50200000534896
:100380004F52542100002048414C542000002020AE
:100390002020202000002050524F472000005245CE
:1003A000534554200000202054504D20000055504B
:1003B00044415445000020202020002533640025BE
:1003C0002D31312E31317300252D35640025632FF9
:1003D00025632025630025630046253032643D25D2
:1003E000630020200102202020202020200025332F
:1003F000640025336400252D3564002D2D2D2D201E
:1004000020004144523A20256C64202020202020E6
:100410002020202000232D007E0E0E0E0E1B1B1C04
:100420000E1B1B7E0E0E0E0E0D5D004D5253540022
:100430004D4658005357555044415445005243527D
:100440000052430054504D00434647535953004314
:1004500046474143430043464744554D500054529C
:100460004B434C4541520054524B4144440054527A
:100470004B44554D50004C4F43434C454152004C6A
:100480004F43414444004C4F4344554D50004C535E
:10049000005054574C005054524C00505457420096
:1004A000505452420050545744005054524400504B
:1004B000545750005054525000505457520050540A
:1004C00052520050410050440043410043560053F3
:1004D0004F00420040400053450053530053520028
:1004E0004D540056005900540046580046004C43F5
:1004F000004C0048414C5400474F00210053544FDA
:1005000050002E00484600485400484C0048003F28
:10051000005A7A41004D4320696E2053544F5000D9
:100520004D4320696E2048414C5400696C6C6567EE
:10053000616C207475726E6F75742061647265737E
:1005400073006C6F6B2062757379006E6F20736C33
:100550006F7420617661696C61626C65006E6F20FA
:100560006461746100636F6D6D616E6420717565A7
:1005700075652066756C6C007475726E6F7574208D
:1005800071756575652066756C6C00706F77657246
:10059000206973204F666600626164207061726139
:1005A0006D657465722076616C756500756E6B6E35
:1005B0006F776E20636F6D6D616E64004552524FB0
:1005C000523A20005741524E494E473A2000455278
:1005D000524F52002530386C580052435220257536
:1005E000202564202575005243202564004D4D00D0
:1005F0004D4D00444343004D4D004D4D002A454EA6
:10060000442A0042415544524154452025750D006D
:100610004D41474D415854494D452025640D004DED
:1006200041474D494E54494D452025640D007338CE
:10063000384D4F44554C45532025640D0053484FC9
:10064000525454494D452025640D004445464155BA
:100650004C54444343004E45474154495645534842
:100660004F5254004C4F4E475041555345005B5339
:10067000595354454D5D0D00444343004D4D0025F5
:10068000642C20005B414343464D545D0D005B5498
:1006900052414B54494F4E535D0D005B4C4F434FFD
:1006A0005D0D0053455249414C20256C750D004DA0
:1006B00043552041544D6567613132380D00484142
:1006C00052445741524520485725640D00322E3080
:1006D0002E300056455253494F4E20005B494E463E
:1006E0004F5D0D0025732564006E6F007965730002
:1006F0002C202573004D3300444343004D4D320000
:100700004D4D31002C200025642C202564002A4505
:100710004E442A004D3300444343004D4D32004DBA
:100720004D31002A454E442A0054696D656F757439
:10073000004269742072656164206572726F720094
:100740004E6F2070616765004E6F2061636B004ED5
:100750006F206465636F6465720053686F72742103
:10076000004275737921004E6F0059657300457220
:10077000726F72004F6B002564002564203D2024B9
:1007800025303258203D2000504100505800504143
:100790000041646472202575203D202425303458A2
:1007A00020203D3E202043563137203D2025642027
:1007B000282425303258292C202043563138203D1A
:1007C0002025642028242530325829004C6F6E677C
:1007D0002041646472203D20257500256400256455
:1007E000000D5D002575003537363030005345204B
:1007F0002564004D6F64756C65202325642028698D
:100800006E70757420312E2E38202620392E2E3110
:100810003629203D20005352202564004D542025C8
:1008200064202564000D5365724E722E2025386CAD
:100830007500322E302E30004D432052657669739C
:10084000696F6E200052455345540054504D20703E
:10085000726F6772616D004443432070726F6772FC
:10086000616D00507772206F6E0048616C74656432
:100870002100507772206F66660054202564202581
:100880006320256400465820257500462025750004
:10089000444343004D6F746F726F6C61204E6577F7
:1008A000004D6F746F726F6C61204F6C64006D331C
:1008B00000756E75736564004C20257520257520C4
:1008C00025632025630000020C151D263039434C9A
:1008D000565F69727F0002070C10151A1E23282C20
:1008E00031363A3F44484D52565B6064696E7379C5
:1008F0007F0002070B1014191D22262B3035393FBB
:1009000043484C51565B5F64696D72767B7F4861EA
:100910006C746564210D5D0046207B4C6F6B232C4D
:10092000205B46315D2C205B46325D2C205B4633DC
:100930005D2C205B46345D2C205B46355D2C205BB6
:1009400046365D2C205B46375D2C205B46385D7D4E
:100950000054207B54726E74232C205B436F6C6FA9
:10096000725D2C205B5374617475735D7D004C2047
:100970007B4C6F6B232C205B53706565645D2C2072
:100980005B464C5D2C205B4469725D2C205B4631DC
:100990005D2C205B46325D2C205B46335D2C205B5A
:1009A00046345D7D0048542048656C7020666F7247
:1009B000207475726E6F757420636F6D6D616E64F7
:1009C000730048462048656C7020666F722066751B
:1009D0006E6374696F6E20636F6D6D616E64730D0D
:1009E00000484C2048656C7020666F72206C6F6BFD
:1009F00020636F6D6D616E64730D002530386C750A
:100A000000636F72746F2028312E356D73292000BA
:100A1000006C756E676F2028342E3032356D732967
:100A2000004D6F746F726F6C610000000000000079
:100A3000004443432020202020000000000000004C
:100A4000004D4D20000000000000000000000000EC
:100A500000444343000000000000000000000000CC
:100A600000706F73697469766120284D4D2900000C
:100A7000006E6567617469766120284443432900EC
:100A800000303A206F666620202020202020202081
:100A900000313A205461696C62697473202020200F
:100AA00000323A202B2049644E6F74696679202009
:100AB00000333A202B204163636573736F72792092
:100AC0000052697072697374696E61202020202061
:100AD0000053616C766120202020202020202020DF
:100AE0000052697072697374696E61202020202041
:100AF0000053616C766120202020202020202020BF
:100B00000020737461746F206C61796F757420209C
:100B10000020737461746F206C61796F757420208C
:100B200000636F72746F2028312E356D7329202079
:100B3000006C6172676F2028342E3032356D732956
:100B4000004D6F746F726F6C610000000000000058
:100B5000004443432020202020000000000000002B
:100B6000004D4D20000000000000000000000000CB
:100B700000444343000000000000000000000000AB
:100B800000706F73697469766120284D4D290000EB
:100B9000006E6567617469766120284443432900CB
:100BA00000303A20446573616374697661646F2034
:100BB00000313A205461696C6269747320202020EE
:100BC00000323A202B2049644E6F746966792020E8
:100BD00000333A202B204163636573736F72792071
:100BE000005265737461757261722020202020208C
:100BF000004775617264617220202020202020202F
:100C0000005265737461757261722020202020206B
:100C1000004775617264617220202020202020200E
:100C2000002045737461646F204D61717565746156
:100C3000002045737461646F204D61717565746146
:100C4000004B75727A2028312E356D7329202000D3
:100C5000004C616E672028342E3032356D732900C8
:100C6000004D6F746F726F6C610000000000000037
:100C7000004443432020202020000000000000000A
:100C8000004D4D20000000000000000000000000AA
:100C9000004443430000000000000000000000008A
:100CA00000706F736974697620284D4D290000002B
:100CB000006E65676174697620284443432900000B
:100CC00000303A2061757320202020202020202031
:100CD00000313A205461696C6269747320202020CD
:100CE00000323A202B2049644E6F746966792020C7
:100CF00000333A202B204163636573736F72792050
:100D000000416E6C6167656E7A757374616E642004
:100D100000416E6C6167656E7A757374616E6420F4
:100D2000005769656465726865727374656C6C6E92
:100D30000053706569636865726E20202020202052
:100D4000002077696564657268657273742E20206F
:100D5000002073706569636865726E202020202012
:100D60000073686F72742028312E356D732920004E
:100D7000006C6F6E672028342E3032356D73290079
:100D8000004D6F746F726F6C610000000000000016
:100D900000444343202020202000000000000000E9
:100DA000004D4D2000000000000000000000000089
:100DB0000044434300000000000000000000000069
:100DC00000706F73697469766520284D4D290000A5
:100DD000006E656761746976652028444343290085
:100DE00000303A206F66662020202020202020201E
:100DF00000313A205461696C6269747320202020AC
:100E000000323A202B2049644E6F746966792020A5
:100E100000333A202B204163636573736F7279202E
:100E200000526573746F72652020202020202020DE
:100E300000536176652020202020202020202020C3
:100E400000526573746F72652020202020202020BE
:100E500000536176652020202020202020202020A3
:100E600000206C61796F75742073746174757320E0
:100E700000206C61796F75742073746174757320D0
:100E8000005B756E6B6E6F776E2073746174757333
:100E90005D00466F726D61746F20696E636F6D7077
:100EA000617400466F726D61746F20696E636F6D5F
:100EB000702E2000696E6B6F6D7061742E20466F0E
:100EC000726D617400696E636F6D7061742E20467F
:100ED0006F726D6174005B756E6B6E6F776E2065FF
:100EE00072726F725D002E2E20617474656E64657F
:100EF0007265202E2E2000233D63616E63656C6C4D
:100F000061000000000000002876756F746F2900F2
:100F10000000000000000000002E2E63616E63657B
:100F20006C6C617A696F6E652E00206572726F72EB
:100F3000650000000000000000000020736F6C6F6F
:100F4000204443432120202020202000207072696B
:100F50006D61207072656D6920474F20002A3D4108
:100F60006E6E756C6C610000000000000000207067
:100F7000726F6772616D6D617A696F6E6520002DA9
:100F8000636F72746F20636972637569746F2D008B
:100F9000206E617469766F2028313A312920202033
:100FA00000206C696E656172652028323A31292013
:100FB00020002070726F677265737369766F2031DD
:100FC0002020002070726F677265737369766F20DE
:100FD00032202000204D6F646F20414320202020CC
:100FE0002020202000204D6F646F204443202020CB
:100FF000202020202000204175746F5374657020DC
:10100000202020202020002A6C65676769200000CE
:1010100000000000000000002A7363726976690016
:101020000000000000000000002E2E207363726993
:101030007474757261202E2E20002E2E2E206C6569
:101040007474757261202E2E2E20002121212065BE
:1010500072726F726520212121202000204F4B20C9
:10106000202020202020202020202020002E20733F
:10107000616C766174616767696F202E20002E2E87
:101080002072697072697374696E6F202E2000235C
:101090003D43616E63202A3D416E6E756C202000D9
:1010A000233D5369202A3D416E6E756C6C61202092
:1010B0000020636F6E6669677572617A696F6E652D
:1010C00020005350454E544F000000000000000027
:1010D0000000002A204E657373756E205472656E91
:1010E0006F202A0020636F72746F206369726375CA
:1010F00069746F20002A2A2A2074696D65206F7533
:1011000074202A2A2A004163636573732E202025E8
:1011100034642F25346400436F6E666967757261AD
:101120007A696F6E6520200020636F6E666967754F
:1011300072617A696F6E6520002E2E2E20657370A5
:10114000657265202E2E2E202000233D626F727264
:1011500061720000000000000000002873696E202A
:101160004669636861290000000000002E2E2E20D1
:10117000626F7272616E646F202E2E2E00204661A7
:101180006C6C6F0000000000000000000000207385
:101190006F6C6F20706172612044434321200020F6
:1011A00022474F22207072696D65726F20202000E7
:1011B0002A3D43616E63656C6172000000000000AF
:1011C000002050726F6772616D6163696F6E2020DD
:1011D00020002D636F72746F206369726375697488
:1011E0006F2D00206E617469766F2028313A3129A5
:1011F00020202000206C696E6561722028323A310F
:1012000029202020002070726F67726573736976E1
:101210006F20312020002070726F677265737369D0
:10122000766F2032202000204D6F646F20414320D4
:101230002020202020202000204D6F646F20444378
:10124000202020202020202000204175746F53741E
:10125000657020202020202020002A6C65657220E7
:1012600000000000000000000000002A65736372A7
:101270006900000000000000000000002E206573DF
:101280006372696269656E646F202E20002E2E2EB7
:10129000206C6579656E646F202E2E2E2000212132
:1012A000212046616C6C6F2021212120202000200C
:1012B0004F4B2020202020202020202020202000F4
:1012C0002E2E206775617264616E646F202E2E2051
:1012D000002E2072657374617572616E646F202ECA
:1012E0002000233D426F727261202A3D43616E638C
:1012F0002E2000233D5369202A3D43616E63656CB7
:101300006172200020436F6E666967757261636960
:101310006F6E202000446573616374697661646157
:101320002020202020002A2A2A2053696E2054726F
:10133000656E202A2A2A002A636F72746F206369FF
:1013400072637569746F2A005469656D706F2065EA
:101350007870697261646F200041636365732E2049
:101360002534642F253464000000436F6E6669677E
:1013700075726163696F6E2020200020436F6E6676
:10138000696775726163696F6E2020002E2E2E20B2
:1013900077617274656E202E2E2E202000233D4C26
:1013A000F6736368656E0000000000000000286BA3
:1013B00065696E2045696E747261672900000020BE
:1013C0002E2E2E206CF673636865202E2E2E2000A4
:1013D000204665686C657200000000000000000097
:1013E00000206E75722066FC722044434321202049
:1013F0002000206572737420474F206472FC636B79
:10140000656E002A3D4162627275636800000000EB
:10141000000000002050726F6772616D6D69657227
:10142000756E6700002D2D204B75727A7363686CA2
:1014300075DF202D2D00204E617469762028313A09
:1014400031292020202000204C696E6561722028FF
:10145000323A3129202020002050726F6772657364
:101460007369762031202020002050726F677265EA
:1014700073736976203220202000204143204D6F75
:101480006475732020202020202000204443204D1C
:101490006F64757320202020202020002041757467
:1014A0006F5374657020202020202020002A6C6556
:1014B00073656E00000000000000000000002A7349
:1014C0006368722E00000000000000000000002E83
:1014D0002E2073636872656962656E202E2E00008F
:1014E0002E2E2E206C6573656E202E2E2E20200051
:1014F00000212121204665686C6572202121212070
:101500000000204F4B2020202020202020202020C1
:101510002000002E2E2073706569636865726E204E
:101520002E2E000077696564657268657273746554
:101530006C6C656E00233D4CF6736368656E202A03
:101540003D4162627200233D4A61202A3D41626250
:1015500072756368000000206CF6736368656E2026
:1015600020202020202020004155530000000000B2
:101570000000000000000000002A2A206B65696E50
:1015800065204C6F6B202A2A20002A2A204B757276
:101590007A7363686C75DF202A2A002A205A6569ED
:1015A00074FC626572736368722E2A005765696302
:1015B0006865202534642F2534640000004B6F6E6D
:1015C00066696775726174696F6E20202000204B18
:1015D0006F6E66696775726174696F6E2020002E88
:1015E0002E2E2077616974696E67202E2E2E2000C2
:1015F000233D64656C657465000000000000000018
:1016000000286E6F20656E7472792900000000005A
:1016100000002E2E2E2064656C6574696E67202E86
:101620002E2E00206661756C740000000000000022
:101630000000000020444343206F6E6C792120207D
:10164000202020200020707265737320474F206691
:101650006972737400002A3D43616E63656C00001B
:10166000000000000000002070726F6772616D69F9
:101670006E670000000000002D73686F72742063B5
:101680006972637569742D2000206E6174697665D6
:101690002028313A312920202000206C696E6561B4
:1016A000722028323A3129202020002070726F6782
:1016B0007265737369766520312020002070726F27
:1016C000677265737369766520322020002041437C
:1016D000204D6F6465202020202020202000204401
:1016E00043204D6F646520202020202020200020F2
:1016F0004175746F537465702020202020202000D5
:101700002A726561642000000000000000000000F3
:10171000002A777269746500000000000000000074
:1017200000002E2E2E2077726974696E67202E2E8F
:101730002E20002E2E2E2072656164696E67202E89
:101740002E2E2000212121206661756C742021211C
:101750002120202000204F4B20202020202020204E
:101760002020202020002E2E2E20736176696E67A7
:10177000202E2E2E2020002E2E20726573746F7264
:10178000696E67202E2E2000233D44656C2E202A92
:101790003D43616E63656C2000233D596573202ACB
:1017A0003D43616E63656C20200020636F6E666947
:1017B0006775726174696F6E2020004F46460000A5
:1017C0000000000000000000000000002A2A2A207B
:1017D0006E6F20547261696E202A2A2A002A2073B3
:1017E000686F7274206369726375697420002A2AB5
:1017F0002A2074696D65206F7574202A2A2A00508A
:101800006F696E7420202534642F25346400000035
:10181000436F6E66696775726174696F6E20202010
:101820000020636F6E66696775726174696F6E2000
:1018300020005B6E6F206D6573736167655D0025C9
:10184000642A2A2A204641494C555245202A2A2AF0
:101850000025643A2030782530386C5800253264F1
:101860002030782530386C5820202000204D33203F
:10187000656E61626C65642020202020003D253566
:10188000640030782530386C5800202535640025F8
:1018900034646D73002533642C25647300202E2E70
:1018A0002E2E202020202020202020002564206DA6
:1018B00073002025326400313200003234000034DD
:1018C0003800003936000031343400313932003309
:1018D00038340035373600303020426175640025D9
:1018E000346400202D2D2D002020202020202000D9
:1018F000204F4B2020202000253364002D2D2D006B
:101900002534643A200025366400202D2D2D2D2D00
:101910000025346400202D2D2D0043563A253464D3
:10192000204269743A25643D0043563A2020202025
:10193000204269743A203D200025357500202D2D68
:101940002D2D004142434445464748494A4B4C4DA2
:101950004E4F505152535455565758595A303132B0
:10196000333435363738392E2C3A2D2B232F3D3C46
:101970007C3E20004D4D20492020313420004D4D2B
:1019800020492020323761004D4D20492020323738
:1019900062004D4D20022020313420004D4D2002A8
:1019A0002020323761004D4D200220203237620066
:1019B000444343202020313420004443432020204E
:1019C00032382000444343202031323820006D3328
:1019D00020202031323820003A2000253575005370
:1019E00065724E722E2025386C7500322E302E30E6
:1019F00000536F6674772E205600253364004E72B4
:101A00003A202532642020004D656E75204C6F63AE
:101A10006F6D6F746976650050726F6772616D6D7E
:101A2000617A2E204443430050726F6772616D6D7E
:101A3000617A2E206D330000537461746F204C6105
:101A4000796F757400000000496D706F7374617474
:101A5000696F6E65000000004167672E20536F6656
:101A600074776172650000004C43442072657472A3
:101A70006F696C6C2E0000004D6173746572436F6A
:101A80006E74726F6C0000005573636974610000BE
:101A9000000000000000000053656C657A696F6EFD
:101AA0006120000000000000466F726D61746F20BD
:101AB00044617469200000004E6F6D652020202075
:101AC000202000000000000056616C6F726520202D
:101AD0002020200000000000435620286279746511
:101AE0002900000000000000435620286269742984
:101AF0000000000000000000496E642E2050726952
:101B00006D6172696F000000496E642E2045737428
:101B100065736F0000000000526567697374726F2F
:101B20000000000000000000506167652D4D6F64EB
:101B300065000000000000004D61696E2054726174
:101B4000636B0000000000005261696C436F6D2000
:101B500043560000000000004D6F646F20313238A2
:101B600046530000000000004D6F646F204A6F670D
:101B70006469616C00000000496D706F7374617A74
:101B80002E2073383800000043616E63656C6C6111
:101B90000000000000000000426F6F737465720067
:101BA000000000000000000056656C6F63697461FE
:101BB00020696E74657266004465632E41636365D7
:101BC00073736F7269000000466F726D61746F20ED
:101BD0004C6F636F00000000506175736120736586
:101BE000676E2E4D4D200000537570706F72742E0D
:101BF0005261696C436F6D006D6F64756C69207321
:101C0000383800000000000074657374206D6F6444
:101C1000756C692073383800506F6C2E20636F72BA
:101C2000746F636972632E0053656E732E20636F49
:101C300072746F6369722E005475747469206163E5
:101C4000636573736F726900466F726D2E206163F6
:101C5000636573736F7269006D696E2E746D702E9B
:101C6000696D70756C736F006D61782E746D702E78
:101C7000696D70756C736F00696E646972697A7AE8
:101C80006F206D33000000004D656E75204C6F6352
:101C90006F6D6F746F72610050726F6772616D6DFE
:101CA000617220444343000050726F6772616D6D32
:101CB0006172206D3300000045737461646F204DC4
:101CC0006171756574610000416A757374657300B4
:101CD000000000000000000055706461746520532E
:101CE0006F66747761726500496C756D696E6163CA
:101CF000696F6E204C4344004D6173746572436F8D
:101D00006E74726F6C00000053616C6972000000A9
:101D1000000000000000000053656C656363696F9C
:101D20006E61722000000000466F726D61746F205A
:101D30004461746F730000004E6F6D627265202005
:101D40002020000000000000466963686120202018
:101D500020200000000000004356202862797465AE
:101D60002900000000000000435620286269742901
:101D70000000000000000000446972656363696F41
:101D80006E20636F72746100446972656363696F8A
:101D90006E206C6172676100526567697374726F5F
:101DA0000000000000000000506167652D4D6F6469
:101DB0006500000000000000456E2056696120703B
:101DC00072696E6369702E005261696C436F6D2099
:101DD00043560000000000004D6F646F2031323820
:101DE000207061736F7300004D6F646F2064652015
:101DF0006D616E646F000000416A757374657320D5
:101E00007338380000000000426F72726172000087
:101E10000000000000000000426F6F737465723AAA
:101E2000000000000000000056656C6F63692E2002
:101E3000496E746572662E0041636365736F7269E3
:101E40006F733A0000000000466F726D61746F207E
:101E50006465205472656E0050617573612053652E
:101E6000F1616C204D4D00005375706F72746520E8
:101E70005261696C436F6D004D6F64756C6F7320B8
:101E80007338380000000000507275656261204DA3
:101E90006F642E2073383800506F6C2E20436F72A1
:101EA000746F636972632E0053656E732E20436FE7
:101EB00072746F6369726300546F646F732041635F
:101EC0006365736F722E0000466F726D61746F20D0
:101ED00061636365736F720044757261632E496D4F
:101EE00070756C2E6D696E0044757261632E496D5C
:101EF00070756C2E6D617800446972656363696FFB
:101F00006E206D33000000004C6F6B204D656EFC41
:101F100000000000000000004443432D50726F6732
:101F200072616D6D672E00006D332050726F6772A5
:101F3000616D6D672E000000416E6C6167656E7AA1
:101F4000757374616E64000045696E7374656C6CC2
:101F5000756E67656E000000536F66747761726519
:101F600020557064617465004C43442042656C6583
:101F700075636874756E67004D6173746572436F45
:101F80006E74726F6C000000457869740000000088
:101F9000000000000000000041757377E4686C6584
:101FA0006E20000000000000446174656E666F7270
:101FB0006D617400000000004E616D6520202020DE
:101FC000202000000000000045696E7472616720E7
:101FD000202000000000000043562028627974652C
:101FE000290000000000000043562028626974297F
:101FF000000000000000000042617369732D41641D
:1020000072657373650000006C616E6765204164E2
:102010007265737365000000526567697374657259
:102020000000000000000000506167652D4D6F64E6
:1020300065000000000000004861757074676C6501
:1020400069730000000000005261696C436F6D20ED
:1020500043560000000000003132384653204D6FD7
:1020600064650000000000005265676C65726D6F6A
:1020700064757300000000007338382D45696E7375
:1020800074656C6C756E67004B6F6E666967757210
:102090006174696F6E000000426F6F737465720047
:1020A0000000000000000000496E74657266616304
:1020B00065204261756400005765696368656E005C
:1020C00000000000000000004C6F6B666F726D61D5
:1020D00074000000000000004D4D2D5369676E61D3
:1020E0006C205061757365005261696C436F6D209F
:1020F000537570706F7274007338382D4D6F64753E
:102100006C650000000000007338382D4D6F647559
:102110006C746573740000004B75727A7363686C3D
:102120002E2D506F6C2E00004B75727A7363686CA5
:102130002E2D456D70662E00616C6C6520576569AB
:102140006368656E000000005765696368656E66C8
:102150006F726D61740000006D696E2E20536368AC
:10216000616C747A656974006D61782E20536368C0
:10217000616C747A656974006D33204164726573B3
:1021800073650000000000004C6F636F6D6F746931
:102190007665206D656E75004443432070726F67ED
:1021A00072616D6D696E67006D332070726F67725A
:1021B000616D6D696E6700004C61796F7574207395
:1021C000746174757300000053657474696E67738D
:1021D0000000000000000000536F667477617265B4
:1021E00020557064617465004C4344206261636BE8
:1021F0006C696768740000004D6173746572436FA9
:102200006E74726F6C000000457869740000000005
:10221000000000000000000053656C65637420003E
:1022200000000000000000004461746120666F72CD
:102230006D617400000000004E616D65202020205B
:102240002020000000000000456E747279202020DC
:1022500020200000000000004356202862797465A9
:1022600029000000000000004356202862697429FC
:1022700000000000000000005072696D617279205A
:102280006164647265737300457874656E642E20B2
:102290006164647265737300526567697374657213
:1022A0000000000000000000506167652D4D6F6464
:1022B00065000000000000004D61696E20747261CD
:1022C000636B0000000000005261696C436F6D2079
:1022D00043560000000000003132384653204D6F55
:1022E00064650000000000004A6F676469616C204B
:1022F0004D6F646500000000733838207365747496
:10230000696E67730000000044656C6574650000C9
:102310000000000000000000426F6F7374657200DF
:102320000000000000000000496E74657266616381
:102330006520426175640000506F696E747300001F
:1023400000000000000000004C6F632E20666F72DA
:102350006D617400000000004D4D207369676E616F
:102360006C207061757365005261696C436F6D20FC
:10237000537570706F727400733838206D6F6475A8
:102380006C65730000000000733838206D6F647551
:102390006C6520746573740053686F727420632ECB
:1023A00020706F6C2E00000053686F727420632ED3
:1023B0002073656E732E0000616C6C20506F696E27
:1023C0007473000000000000506F696E7473206623
:1023D0006F726D61740000006D696E2E73776974A1
:1023E00063682E74696D65006D61782E737769740A
:1023F00063682E74696D65006D3320616464726575
:102400007373000000000000446F776E6C6F6164AE
:10241000202E2E2E20202020000011241FBECFEFC2
:10242000D0E1DEBFCDBF12E0A0E0B1E0E0EFF8E424
:1024300001E00BBF02C007900D92A637B107D9F794
:102440001DE0A6E7B2E001C01D92AB3DB107E1F788
:102450000E9489120C9476A40C940000809176025C
:10246000089581E080937702089580E00E942263BE
:1024700081E00E9422630E94C26B0E947C850E94C0
:10248000613E80917702882311F40E943F1EA89537
:102490000895982F809176028917C9F18630B9F195
:1024A000853011F4963099F590937602892F8250F9
:1024B000823010F0973059F40E941D361092350783
:1024C00080917602823029F40E940D3802C00E9469
:1024D0008E3180917602863011F40E944C67809193
:1024E0007602813011F482E003C0882321F481E078
:1024F00064E00E94258884E064E00E942588809141
:1025000076020E94697381E080937702089580E0EB
:102510000895CF93DF930E941B6A0E9468130E9464
:10252000A7390E94CA830E940C300E94086768E0A5
:102530004EE421E00E94961387E068E04EE421E03B
:102540000E9425150E94401778940E940A1C0E9440
:102550000567DC0114968C910E943A1E82E06DEAB8
:1025600070E00E9497200E9427678130D9F482E0B2
:1025700069EA70E00E94972081E060E00E94C31E3B
:1025800082E066E50E94BD1F82E06CE870E00E9478
:1025900097200E940567EC0181E00E94E01C8823DF
:1025A00049F125C00E94276700D000D00F92EDB7F7
:1025B000FEB7319692E0ADB7BEB711969C9322EA72
:1025C00030E032832183838314820E943D200F9068
:1025D0000F900F900F900F9081E060E00E94C31E5B
:1025E00082E062E970E00E949720A895FECF80E02B
:1025F0000E94C76982E00E94E01C882319F084E0F1
:102600000E94C76983E00E94E01C882319F085E0DE
:102610000E94C76984E00E94E01C882319F081E0D1
:102620000E94C76980E00E94491281E00E94BA7945
:1026300080E00E94E01C882319F088E10E94149D2C
:102640000E94437D8FEF60E240E050E00E94166BF5
:1026500080E00E94616681E00E9461660E94AA8714
:1026600002C00E9435128091370790913807A091DF
:102670003907B0913A07805D9740A040B04088F399
:1026800089859A85009749F060E070E040E050E06D
:102690000E94DE7DBC01009711F46A817B818FEF7F
:1026A0000E94536981E011C00E94BD440E94041D34
:1026B000FFEF8F3F9F07C1F70E943512809177028D
:1026C0008823A1F31092770280E00E948C3FEECF26
:1026D0008FE78ABB1BBA80E187BB18BA80EF84BB47
:1026E0008FEF85BB8BEB81BB8CEC82BB82E082B928
:1026F00087EF83B987E78093610081EE8093620062
:1027000087E18093640089E1809365000E940A7AE2
:1027100010926A001ABE8AB78A608ABF0E9407199F
:10272000A89588E181BD8EE081BD08951092F106E3
:102730009091F1069093F0069091F0069093130714
:10274000909113079093120791E0909334078C9A1D
:10275000119A92B19E7E92B9199A93B19E7E93B9C5
:1027600092E09BB99498883008F087E0E82FF0E079
:10277000EE0FFF1FE754FF4FA591B491653010F4A1
:1027800065E003C0693008F068E04F7D6550660F72
:10279000453411F4606203C04F3409F460632230A1
:1027A00008F068608B2F992787FD9A958F7080932A
:1027B0009000A9B96093950088EB8AB980E090E019
:1027C00008951F920F920FB60F920BB60F9211241D
:1027D0008F939F93EF93FF9390911207809113072C
:1027E000981761F088B7806188BF0C9B09C0809101
:1027F000340780FF05C089B7806189BF559812C032
:10280000E0911307F0E0E051F94F84A18CB9809179
:1028100013078F5F8093130780911307803210F0A6
:1028200010921307FF91EF919F918F910F900BBE24
:102830000F900FBE0F901F9018951F920F920FB61A
:102840000F9211248F9389B78F7E89BF559A8F91EC
:102850000F900FBE0F901F90189527E0813D9207B3
:10286000C0F12FE0813A920710F481E01EC023E20C
:102870008932920710F482E018C026E3813B920768
:1028800010F483E012C026E48135920710F484E04E
:102890000CC028E8893B920710F485E006C0895DEA
:1028A000964D10F087E001C086E0789420E030E09B
:1028B0005E9902C020E030E02F5F3F4FA89597E27D
:1028C00020313907A8F368E04EE421E00E94961316
:1028D000089580E0EACF8330C9F0843028F4813055
:1028E00061F0823080F40CC08530B1F0853088F022
:1028F0008630A9F08730C9F415C020E639E017C04A
:1029000020EB34E014C020EC32E111C020E835E2C5
:102910000EC020E438E30BC020E03BE408C020E018
:1029200036E905C020E031EE02C020E030E0C90108
:10293000089539B120919000922F80E0232F30E04C
:10294000282B392B49EB50E060E0FA0185919491F6
:102950008217930729F06F5F4E5F5F4F6830A9F7CA
:10296000862F0E946B140895482FA89503C0559A8E
:102970007894A895209112078091130730E090E099
:1029800001972817390799F3809112078F3121F4A5
:1029900080911307882359F3E0911207F0E0E0518A
:1029A000F94F44A39FB7F894809112078F5F8093EB
:1029B000120780911207803210F0109212079FBF09
:1029C000559A80E090E00895F8948091F0069091F7
:1029D000F106282F30E0291B3109789437FF02C017
:1029E000205E3F4F2031310534F49498232B19F4A5
:1029F0002FEF3FEF15C0E091F106F0E0E051F94F05
:102A00009281F8948091F1068F5F8093F106809116
:102A1000F106803210F01092F106292F30E0789400
:102A2000C901089590913407882331F080913407CB
:102A300081608093340706C0809134078E7F809335
:102A40003407559A892F817008951092AC069091A1
:102A5000AC069093AB069091AB069093CE06909106
:102A6000CE069093CD0691E09093EF0691B39862D5
:102A700091BB8A981598939A92981D9892E090939A
:102A80009B009598883008F087E0E82FF0E0EE0F83
:102A9000FF1FE754FF4FA591B491653010F465E036
:102AA00003C0693008F068E04F7D6550660F8B2FDA
:102AB000992787FD9A958F7080939800A09399002D
:102AC000453411F4606203C04F3409F4606322306E
:102AD00008F0686060939D0088EB80939A0080E026
:102AE00090E008951F920F920FB60F920BB60F92BF
:102AF00011248F939F93EF93FF939091CD06809134
:102B0000CE06981761F088B7806288BF0D9B0DC014
:102B10008091EF0680FF09C089B7806289BF8091EC
:102B20009A008F7D80939A0013C0E091CE06F0E06A
:102B3000E555F94F84A180939C008091CE068F5F6C
:102B40008093CE068091CE06803210F01092CE0691
:102B5000FF91EF919F918F910F900BBE0F900FBE41
:102B60000F901F9018951F920F920FB60F920BB6F1
:102B70000F9211248F93EF93FF9389B78F7D89BFB5
:102B8000EAE9F0E0808180628083FF91EF918F918C
:102B90000F900BBE0F900FBE0F901F901895482FEF
:102BA000A89507C080919A00806280939A007894DB
:102BB000A8952091CD068091CE0630E090E0019757
:102BC0002817390779F38091CD068F3121F4809150
:102BD000CE06882339F3E091CD06F0E0E555F94FB4
:102BE00044A39FB7F8948091CD068F5F8093CD0664
:102BF0008091CD06803210F01092CD069FBF80915B
:102C00009A00806280939A0080E090E00895F894A2
:102C10008091AB069091AC06282F30E0291B31093A
:102C2000789437FF02C0205E3F4F2031310534F4E5
:102C30009598232B19F42FEF3FEF15C0E091AC06C8
:102C4000F0E0E555F94F9281F8948091AC068F5FE2
:102C50008093AC068091AC06803210F01092AC06E6
:102C6000292F30E07894C901089590913407882382
:102C700031F08091EF0681608093EF060AC0809169
:102C8000EF068E7F8093EF0680919A00806280939A
:102C90009A00892F817008951F920F920FB60F929C
:102CA0000BB60F9211242F933F934F935F936F9323
:102CB0007F938F939F93AF93BF93EF93FF93209155
:102CC000AB068091AC0630E090E0019728173907F9
:102CD00041F08091AB068F3179F48091AC06882366
:102CE00059F48091AC068F5F8093AC068091AC065E
:102CF000803210F01092AC0680919B00E091AB0600
:102D0000F0E090919C00E555F94F9283928184FD0B
:102D10000CC08091AB068F5F8093AB068091AB06B1
:102D2000803278F01092AB060CC0992351F41092C7
:102D3000AC068091AC068093AB06959881E00E942A
:102D400061668091AB069091AC06282F30E0291B7C
:102D5000310937FF02C0205E3F4F213131050CF0B1
:102D6000959AFF91EF91BF91AF919F918F917F9134
:102D70006F915F914F913F912F910F900BBE0F90EC
:102D80000FBE0F901F9018951F920F920FB60F92C3
:102D90000BB60F9211242F933F934F935F936F9332
:102DA0007F938F939F93AF93BF93EF93FF93209164
:102DB000F0068091F10630E090E00197281739077E
:102DC00041F08091F0068F3179F48091F1068823EB
:102DD00059F48091F1068F5F8093F1068091F1069E
:102DE000803210F01092F1068BB1E091F006F0E025
:102DF0009CB1E051F94F9283928184FD0CC0809187
:102E0000F0068F5F8093F0068091F0068032A8F084
:102E10001092F00612C0992381F41092F10680916D
:102E2000F1068093F006949880E00E94616681E04C
:102E300068E04EE421E00E9496138091F0069091A4
:102E4000F106282F30E0291B310937FF02C0205E30
:102E50003F4F213131050CF0949AFF91EF91BF91D2
:102E6000AF919F918F917F916F915F914F913F9122
:102E70002F910F900BBE0F900FBE0F901F901895C3
:102E800087B3876087BBBB9888B3896088BB1DB850
:102E90008EB18FB187E78DB9089578941F920F9204
:102EA0000FB60F920BB60F9211242F938F939F930F
:102EB000EF93FF938FB1E0917802F0E0E858FD4F77
:102EC0008283809178028F5F80937802809178026C
:102ED000883110F0109278029091790280917802F6
:102EE000981759F4809179028F5F809379028091CD
:102EF0007902883110F010927902E0919302F0E0AB
:102F0000E858FD4F248D27FF19C0C09A000000002B
:102F100000000000000000000000000000000000B1
:102F200000000000000000000000000000000000A1
:102F300000000000000000000000000090919302DB
:102F400080919202981771F0C098809193028F5FE0
:102F50008093930280919302883110F01092930233
:102F60002FB902C0C09A6F98FF91EF919F918F91F6
:102F70002F910F900BBE0F900FBE0F901F901895C2
:102F80008091930290919202282F30E0295E3F4F6A
:102F9000291B31092831310514F028513040C9016D
:102FA0000895482F6F9933C0C0988FB16F9A909150
:102FB000920280919302981711F44FB94BC0E0919F
:102FC0009302F0E0E858FD4F848D8FB98091930211
:102FD0008F5F80939302809193028831C0F01092AA
:102FE000930215C06F9913C0E0919302F0E0E85886
:102FF000FD4F848D8FB9809193028F5F80939302F0
:1030000080919302883110F0109293026F9A809110
:1030100092022091930290E0019630E0821793078C
:1030200009F380919202873121F4809193028823E1
:10303000C9F2E0919202F0E0E858FD4F448F809190
:1030400092028F5F8093920280919202883110F0F9
:103050001092920280E090E008954FB7F89490911A
:10306000780280917902981719F42FEF3FEF13C07F
:10307000E0917902F0E0E858FD4F8281282F30E09E
:10308000809179028F5F80937902809179028831F3
:1030900010F0109279024FBFC9010895882311F0F2
:1030A000DD9A0895DD980895882351F08091650098
:1030B0008460809365000000000000000000089517
:1030C000809165008B7F8093650008950F931F9317
:1030D000DF93CF930F92CDB7DEB7182F8AB3807FDF
:1030E0008ABB80E00E9454188091650082608093C2
:1030F0006500112321F080916500816003C08091FB
:1031000065008E7F809365000000000081E00E94D2
:10311000541809B380E00E94541810E084E0000FB6
:10312000111F8A95E1F7000000000000000081E017
:103130000E94541899B39F70902B80E099830E944D
:1031400054188AB38F608ABB9981892F0F90CF91D1
:10315000DF911F910F91089580E00E946618982FCB
:1031600087FF11C08091AF029091B00228E08130BA
:10317000920714F080E0089501969093B002809336
:10318000AF0281E008958091B602882319F49F77F9
:103190009093B7021092B0021092AF0280E00895AF
:1031A0009B01AC018091370790913807A0913907B6
:1031B000B0913A0782179307A407B50798F080915A
:1031C000370790913807A0913907B0913A0760E02E
:1031D000821B930BA40BB50B80509041A040B040D4
:1031E000A0F412C08091370790913807A091390759
:1031F000B0913A0760E0281B390B4A0B5B0B20505B
:10320000304F4F4F5F4F08F061E0862F08951092C6
:103210007D0080B7877F80BF17BE11BE89E683BF60
:103220008BE085BD8FE183BD87B7806887BF82EF64
:103230008FBD3AE13EBD4FEC50E057BD46BD85EB3A
:1032400090E09BBD8ABD99BD88BD22EC20938B0088
:1032500030938A00509381004093800090938700C0
:10326000809386000895EF92FF920F931F93209111
:103270003707309138074091390750913A077C0160
:1032800000E010E0E20EF31E041F151F01C0A89518
:10329000C801B7010E94D0188823C9F31F910F916C
:1032A000FF90EF900895FF920F931F93082F162F12
:1032B000F42E809165008D7F8093650080E00E94F0
:1032C00054188AB38F608ABB8BB3902F92959F70EE
:1032D000807F982B9BBB112321F08091650081603A
:1032E00003C0809165008E7F8093650081E00E941D
:1032F000541880E00E945418FF2029F088E090E0E4
:103300000E9433190FC08BB30F70807F802B8BBB53
:10331000000000000000000081E00E94541880E0DE
:103320000E9454181F910F91FF900895EF92FF9201
:103330000F931F9320913707309138074091390739
:1033400050913A077C0100E010E0E20EF31E041FEA
:10335000151F02C00E943512C801B7010E94D01883
:103360008823C1F31F910F91FF90EF9008950F9361
:103370001F93282F8091B502893018F48F5F8093B6
:10338000B5028091B5028430B1F0853048F48230C6
:1033900009F4BFC0833008F0B9C08130E9F409C036
:1033A0008630B1F0863090F08730A1F08830A1F4FB
:1033B000B0C0DC9AAEC01092B4021092B30280E0AA
:1033C00090E89093B2028093B10206C0DD9AA1C04A
:1033D000DD989FC0DC989DC0222309F097C06091C2
:1033E000B3027091B4024091B1025091B202CF9BEE
:1033F0003BC09B01220F331FF901EF58F34F80812F
:10340000918184239523892BF1F4F901E450F44F41
:1034100080819181842B952B91838083F901EC56D7
:10342000F44F80819181842B952B9183808385E655
:103430009CE00E940C896091B3027091B4028BE60B
:103440009CE00E940C89E091B302F091B402EE0F6F
:10345000FF1FEF58F34F808191812091B10230918D
:10346000B202822B932B29C0FB01EE0FFF1FEF58F6
:10347000F34F8081918184239523892B61F085E628
:103480009CE00E940C896091B3027091B4028BE6BB
:103490009CE00E940C89E091B302F091B402EE0F1F
:1034A000FF1FEF58F34F8091B1029091B2028095C7
:1034B0009095208131818223932391838083809111
:1034C000B1029091B202969587959093B202809343
:1034D000B102892BE9F40091B3021091B4020F5F9D
:1034E0001F4F1093B4020093B3020E940567FC01C2
:1034F000808590E00817190710F01092B50280E05F
:1035000090E89093B2028093B10202C0DE9A01C0AB
:10351000DE981F910F9108951F920F920FB60F9290
:103520000BB60F9211241F932F933F934F935F93EA
:103530006F937F938F939F93AF93BF93EF93FF937B
:103540008091AC02882309F051C181E08093AC02E4
:10355000789480E00E94B7198091AE028F5F8093CB
:10356000AE028091AE0290E0837090708130910540
:1035700019F1823091051CF4892B41F0E5C08230AD
:10358000910561F1039709F0DFC065C080913707AD
:1035900090913807A0913907B0913A070196A11D83
:1035A000B11D8093370790933807A0933907B093E4
:1035B0003A070E94EC1CC8C08091370790913807E9
:1035C000A0913907B0913A0781709070892B19F05A
:1035D0000E941E1DB9C00E94A41CB6C00E942E12DB
:1035E000833049F00E942E12823029F00E942E1260
:1035F000873009F0A9C00E94ED2F20913507309146
:1036000036078823E9F02E5F3F4F3093360720932B
:1036100035070E940567FC019681992309F494C03F
:103620008AE0989FC0011124209135073091360718
:103630002817390708F488C081E00E94491284C025
:103640002115310509F480C02150304030933607F0
:103650002093350779C00E942E12833059F18430AF
:1036600028F4813061F0823008F513C08730D9F139
:10367000883009F448C0843009F061C024C08091CA
:10368000370790913807A0913907B0913A0786FF24
:1036900004C080916200816003C0809162008E7FCF
:1036A00080936200809162008F7E4CC080916200A6
:1036B000816148C080916200806180936200809146
:1036C00062008E7F3FC0809162008E7F8093620097
:1036D0008091370790913807A0913907B0913A0748
:1036E00090FFE0CF1FC0809162008E7F80936200C8
:1036F0008091370790913807A0913907B0913A0728
:1037000091FFD0CF0FC08091370790913807A091DB
:103710003907B0913A0787FF09C0809162008E7F18
:10372000809362008091620080610CC08091620091
:103730008F7E8093620080916200816003C08091DF
:1037400062008E7E809362008091AD02882321F01A
:103750000E94AC188093AD028091AD02882309F0DD
:1037600040C090913B0780913C079817B9F1809138
:103770003C07E82FF0E0E55CF84F9281182F1F5FBF
:10378000103108F010E0903801F580913B07811767
:1037900029F1E12FF0E0E55CF84F92819F3F19F4A9
:1037A0009091B702906897FF02C01092B602892FDD
:1037B000807C803419F481E08093B6021F5F103161
:1037C00008F010E0892F60E002C0892F61E040E03E
:1037D0000E94531910933C0781E001C080E0809360
:1037E000AD0281E00E94B7191092AC02FF91EF91F7
:1037F000BF91AF919F918F917F916F915F914F9109
:103800003F912F911F910F900BBE0F900FBE0F9005
:103810001F901895CF93DF9388E290E00E943319B0
:1038200080E360E041E00E94531980E360E041E002
:103830000E94531980E360E041E00E94531980E246
:1038400060E041E00E94531988E20E94AD1E80E4CE
:103850000E94AD1E8AE00E947A1E89E20E94AD1E7F
:103860008CE10E94AD1E82E50E94AD1E89E60E9499
:10387000AD1E84E70E94AD1E80E40E94AD1E85E16E
:103880000E947A1E88E20E94AD1E80E40E94AD1E56
:103890000E94ED3CEC0101C0A89590913B078091FE
:1038A0003C079817C9F70E94AC188823A9F781E054
:1038B0000E9466188A3019F481E089AB01C019AA08
:1038C00088E00E94AD1E81E00E94AD1E86E00E944D
:1038D000AD1E8CE00E94AD1E80E060E00E94C31E21
:1038E00080E062EE70E00E94A41F81E066E271E079
:1038F0000E94A41F82E06EE271E00E94A41F83E098
:103900006EE371E00E94A41FDF91CF910895909122
:10391000BA02E92FF0E0E654FD4F82839F5F909357
:10392000BA02983010F01092BA029091BB028091C6
:10393000BA02981741F4892F8F5F8093BB028830B9
:1039400010F01092BB02089531B12091B902220FFC
:1039500036FD2160822F83708150823028F424FF4D
:1039600002C02E6001C0217F2093B9029091B8025D
:10397000990F37FD9160892F83708150823028F430
:1039800094FF02C09E6001C0917F9093B802207C9A
:10399000892F807C203831F4882341F0803C79F4F1
:1039A0008AE105C0203459F4803C21F489E10E9469
:1039B000871C0895882319F48AE10E94871C0895C2
:1039C000893110F080E00895E82FF0E0EC53FD4FCE
:1039D0008081811181E008953091F602343029F41C
:1039E00085B3806F85BB97980895979A25B380E13A
:1039F00090E002C0880F991F3A95E2F78095807F8A
:103A00002F70822B85BB08959091BB028091BA02E2
:103A1000891719F42FEF3FEF0FC0E92FF0E0E654BC
:103A2000FD4F8281282F30E0892F8F5F8093BB026A
:103A3000883010F01092BB02C90108958F929F92B6
:103A4000AF92BF92CF92DF92EF92FF920F931F93AC
:103A5000CF93DF930E942E12982F8091F702981730
:103A600029F09093F70282E20E94871C83B3E1B0B1
:103A7000EE0CEE0C90E1E9228F70E82ACC24DD24D4
:103A800095E0A92E81E0882E912CBB24B394E0917F
:103A9000F602EA9DF0011124EC0DFD1DE753FF4FE6
:103AA000F49088E18F1508F48EC00E2D0825017062
:103AB000CF2DD0E0FE01E352FD4F1081110F0E9487
:103AC0002767803819F4002371F009C001111160D3
:103AD000812F90E0817190708131910511F41F6107
:103AE00003C0892B09F4107E812F90E080769070BE
:103AF0008034910519F41F7182E00CC08032910569
:103B000019F4106E81E006C08036910511F080E056
:103B100001C083E0FE01E352FD4F1083823091F03B
:103B2000833051F1813009F04EC096E1F91621F44D
:103B30008091D902882319F48F2D0E94871CCC53C1
:103B4000DD4F34C0CC53DD4F18828F2D80680E942A
:103B5000871C0E942E128530B1F585E1F81619F404
:103B60008091DA0205C096E1F91669F58091D902D3
:103B7000882349F586E025C0FE01EC53FD4F808186
:103B80008F5F8083882309F4B08285E1F816D8F02E
:103B900096E19F1568F487E1F816A9F4CC53DD4F40
:103BA0008881853680F081E20E94871CB8820BC034
:103BB0008091D902893738F08091DA02893718F07C
:103BC00085E00E9449120894C11CD11C95E0C916D9
:103BD000D10411F0E6945BCF8091F6028F5F809361
:103BE000F602853010F01092F602DF91CF911F910E
:103BF0000F91FF90EF90DF90CF90BF90AF909F908C
:103C00008F9008959093680780936707892B89F1B7
:103C10007093660760936507809137079091380726
:103C2000A0913907B0913A079B0140E050E0280F7E
:103C3000391F4A1F5B1F209361073093620740932F
:103C4000630750936407809160078E7F80936007BD
:103C5000211531054105510561F481E090E0A0E0B6
:103C6000B0E08093610790936207A0936307B093DD
:103C700064070895813308F080E381BF089580913F
:103C8000670790916807892BA1F160916107709196
:103C9000620780916307909164070E94D01888237F
:103CA00041F180916007E0916707F09168078170AA
:103CB00009958091600791E08927809360072091A2
:103CC0003707309138074091390750913A07809172
:103CD000650790916607A0E0B0E0820F931FA41FD4
:103CE000B51F8093610790936207A0936307B09319
:103CF000640708951F93182F09C080E00E94226373
:103D000081E00E9422630E94C26BA89520913B072C
:103D100080913C0730E090E001972817390769F35C
:103D200080913B078F3021F480913C07882329F351
:103D3000F894E0913B07F0E0E55CF84F1283809146
:103D40003B078F5F80933B0780913B07803110F0EA
:103D500010923B0778941F9108951F93182F80E8C5
:103D60000E947A1E812F0E947A1E1F910895109240
:103D700068071092670781E00E94AD1E08958CE0ED
:103D80000E94AD1E08958295880F880F807C860F53
:103D900080680E94AD1E0895BF92CF92DF92EF928D
:103DA000FF920F931F93CF93DF93C82EB62E8A01F5
:103DB000109268071092670721E02817A0F13FE0F2
:103DC000361788F14115510571F1FA010190002073
:103DD000E9F73197DE2ED41A80E18D1510F490E1C9
:103DE000D92E8C2D6B2D0E94C31EE8018DE4E82E88
:103DF00087E0F82E08C08881F70181937F016991DF
:103E000082E00E94BD1F9E01201B2D15A0F3C092D1
:103E10005D07B0925E07D0925F0786E49FE164EF92
:103E200071E00E94021EDF91CF911F910F91FF90D0
:103E3000EF90DF90CF90BF900895DF93CF93CDB7F1
:103E4000DEB7A0970FB6F894DEBF0FBECDBFDE0180
:103E500011969E01205E3F4F04C09D93A217B307A9
:103E600031F0FA014F5F5F4F94919923B1F71C92A3
:103E7000AE014F5F5F4F0E94CC1EA0960FB6F89424
:103E8000DEBF0FBECDBFCF91DF9108950F931F937B
:103E9000CF93DF93082F80915D0760915E070E94AA
:103EA000C31E10E0CDE4D7E009C0002311F460E2A6
:103EB00001C0699182E00E94BD1F1F5F80915F0772
:103EC000181798F3DF91CF911F910F9108950E94D9
:103ED000C31E8EE00E94AD1E0895EF92FF920F93D5
:103EE0001F93CF93DF93382F7B01122F883028F553
:103EF000483018F5842F90E0820F911D099714F037
:103F000018E0141B330F330F330F340F832F8064EB
:103F10000E94AD1EC0E0D0E0012F10E008C0F70104
:103F2000EC0FFD1FE4918E2F0E947A1E2196C01780
:103F3000D107ACF38FEF0E94AD1EDF91CF911F919F
:103F40000F91FF90EF90089540E028E00E946D1FD0
:103F50000895813069F0813040F0833019F02FEFFF
:103F60003FEF09C00E94041D05C00E94E41402C076
:103F70000E9407169C01C90108951F93162F8130D6
:103F800009F465C0813008F45EC0823009F062C077
:103F900067FF55C00E94ED3CFC0181A98823E1F038
:103FA000143E11F414E84BC0163F11F414E947C055
:103FB0001C3F11F411E843C0143C11F41EE83FC04B
:103FC000163D11F419E93BC01C3D11F41AE937C044
:103FD000113F69F51BE933C0143E11F411EE2FC0F7
:103FE000163F11F41FEE2BC01C3F11F415EF27C034
:103FF000113F11F41EEE23C0143C39F484E06EEF3F
:1040000071E00E94A41F14E01AC0163D39F485E047
:1040100066E072E00E94A41F15E011C01C3D39F457
:1040200086E06EE072E00E94A41F16E008C01F3D0B
:1040300031F487E066E172E00E94A41F17E0812F4F
:104040000E947A1E07C0862F0E94B41403C0862FD8
:104050000E94CF151F9108951F93CF93DF93182FC0
:10406000EB0104C02196812F0E94BD1F6881662349
:10407000C9F7DF91CF911F9108950F931F93DF939D
:10408000CF93CDB7DEB7C055D0400FB6F894DEBFA2
:104090000FBECDBF9E01265A3F4F8E010F5F1F4FAF
:1040A000C8016A966EAD7FAD6A97A9010E9453A1BF
:1040B00068968FAD6897B8010E942C20C05BDF4FD7
:1040C0000FB6F894DEBF0FBECDBFCF91DF911F9129
:1040D0000F9108950F931F93DF93CF93CDB7DEB762
:1040E000C055D0400FB6F894DEBF0FBECDBF9E01C5
:1040F000265A3F4F8E010F5F1F4FC8016A966EAD63
:104100007FAD6A97A9010E942AA168968FAD689732
:10411000B8010E942C20C05BDF4F0FB6F894DEBFC1
:104120000FBECDBFCF91DF911F910F9108951F93C7
:10413000CF93DF93182FEB0104C0812F0E94BD1F86
:104140002196FE0164916623C1F7DF91CF911F9103
:104150000895582F5F705F3011F45EE001C0511177
:104160005F5F442311F490E001C098E0623061F099
:10417000633018F4613069F405C0633039F064309D
:1041800041F406C0936005C0946003C0966001C00E
:104190009760951739F4442319F4592F95E002C01C
:1041A000592F9AE080E020E030E0880F880F50FD22
:1041B000826090FD81602F5F3F4F2430310519F000
:1041C00056959695F2CF90E00895962F9F709F3068
:1041D00011F491E002C091119F5F8370813071F4FE
:1041E00020E030E080E0880F880F90FD83602F5F33
:1041F0003F4F2430310501F19695F5CF67FD06C09C
:10420000983010F44DE007C045E005C0983010F03C
:1042100042E001C04AE020E030E080E0880F880FF3
:1042200090FD826040FD81602F5F3F4F243031055B
:1042300019F096954695F2CF90E008959C01FB0108
:104240008038910520F48F77808388E00895832F4C
:10425000806C8183208380E10895F90108969C0198
:1042600053E0369527955A95E1F72F7320682183FF
:104270009C012095309595E0369527959A95E1F724
:1042800020778770282B2083662319F021602083F4
:104290000BC0822F80688083442311F0286820831C
:1042A000808191E08927808380E108950F93CF93E7
:1042B000DF93EC01A62FA695A695A695862F87706D
:1042C00078E0781B04C0220F331F441F551F8A95C6
:1042D000D2F712C0FE01EA0FF11D8081822B80838C
:1042E000802F701708F4872F680F081B232F342F97
:1042F000452F5527AF5F78E0002361F7862FDF91C8
:10430000CF910F9108950F93E42F8038910530F4E9
:1043100091609C0140E050E009E01AC022E080304A
:10432000920730F49C609C0140E050E00CE010C02B
:1043300028E08030920730F490679C0140E050E024
:104340000FE006C09C0140E050E0306C436002E1A9
:10435000CB016E2F0E9456210F9108956FB7F894EC
:104360004091690780916A07242F30E090E001971F
:104370002817390749F04F3011F050E006C08091FE
:104380006A0750E0882309F451E06FBF6FB7F894D3
:104390004091170880911808242F30E090E0019791
:1043A0002817390749F04F3011F090E006C080918E
:1043B000180890E0882309F491E06FBF892F852BBE
:1043C0000895AF92BF92CF92DF92EF92FF920F9338
:1043D0001F93CF93DF93EC015A01122F8091370383
:1043E000882309F057C0013009F054C08981282F73
:1043F00030E08881482F50E03BC080819181861752
:10440000970761F5828193818A159B0539F584812F
:10441000813021F586819781A085B1850097A1051E
:10442000B105E1F0F90183E0EE0FFF1F8A95E1F796
:10443000220F331FE20FF31FEC0FFD1F84899589B4
:10444000A689B7898C159D05AE05BF0509F48FC0F7
:10445000C48AD58AE68AF78A138B89C0C901019676
:104460003A9620E030E08031910514F49C010EC0B2
:10447000F901EE0FFF1FC901A3E0880F991FAA954C
:10448000E1F7E80FF91F3E96EC0FFD1F24173507E3
:1044900009F0B3CFEFB7F8943881A32FB0E089814A
:1044A00090E00197A817B90741F03F3011F090E074
:1044B00005C0898190E0882309F491E0EFBF99233A
:1044C00011F080E055C0FD0193E0EE0FFF1F9A95BB
:1044D000E1F7AA0FBB1FEA0FFB1FEC0FFD1F778749
:1044E0006687888190E0FC0163E0EE0FFF1F6A950C
:1044F000E1F7880F991FE80FF91FEC0FFD1FB18A34
:10450000A08A888190E0FC0143E0EE0FFF1F4A95EE
:10451000E1F7880F991FE80FF91FEC0FFD1F138BB0
:10452000888190E0FC0123E0EE0FFF1F2A95E1F760
:10453000880F991FE80FF91FEC0FFD1F028B888170
:1045400090E0FC01B3E0EE0FFF1FBA95E1F7880F92
:10455000991FE80FF91FEC0FFD1FC48AD58AE68A60
:10456000F78A88818F5F8883803108F0188281E024
:10457000DF91CF911F910F91FF90EF90DF90CF903F
:10458000BF90AF9008958091C90890E0833009F4FE
:1045900091E0892F0895FC01009729F1818590E031
:1045A000837090708330910534F48130910534F438
:1045B000892B61F018C00397B1F404C080913603D1
:1045C000816007C080913603826003C0809136030A
:1045D0008460809336038091360390E08770873043
:1045E00019F091E001C090E0892F0895809338037D
:1045F00008958091360380720895809136038F7DEF
:104600008093360310924F0310924E0308959093B7
:104610004D0380934C0310924F0310924E03089564
:104620008FB7F8948FBF80914A0390914B03089500
:104630008FB7F8948FBF80914E0390914F030895E8
:1046400078941F920F920FB60F920BB60F9211240F
:104650002F933F938F939F93EF93FF938091490301
:10466000883010F01092490324B135B1809136039F
:1046700084FF34C080914903E82FF0E0EE0FFF1F64
:10468000E75CFC4F318320838F5F80934903E9E32C
:10469000F3E020E030E081919191280F391F83E011
:1046A000E934F807C1F730934B0320934A03809114
:1046B0004E0390914F038217930724F430934F03D6
:1046C00020934E0380914C0390914D0382179307E2
:1046D0002CF480913603806280933603FF91EF9132
:1046E0009F918F913F912F910F900BBE0F900FBE16
:1046F0000F901F901895982F03C0892F862311F4CF
:10470000990FD9F7892F0895DC0152962C91529771
:10471000243009F04CC053969C915397292F215077
:1047200053962C93539758968C915897813009F44F
:1047300097C0843009F494C0803209F491C0803865
:1047400009F48EC08230E9F457968C9157978830DF
:1047500030F057961C92579753969C9325C0822F02
:10476000869586958695FD01E80FF11D808190E084
:10477000277002C0959587952A95E2F780FD09C0BC
:1047800011C0803179F0803469F0883011F4223022
:1047900048F457968C9157978F5F57968C9323E3E5
:1047A00030E063C057961C922FEF3FEF5EC05496E7
:1047B0008C9154978823C1F555968C9155978823F1
:1047C00099F553963C915397932F915053969C9300
:1047D0005397233089F45C968C915C97882361F41D
:1047E0009770973049F481E05C968C935C97539670
:1047F0003C93539790E019C05C961C925C9753963B
:104800002C915397822F869586958695FD01E80F0A
:10481000F11D808190E0277002C0959587952A95BB
:10482000E2F7982F917001C091E052968C918230FE
:1048300029F0833099F08130B1F408C0992319F43C
:1048400020E130E012C02CE530E00FC0992319F4CC
:104850002CE130E00AC02EEB30E007C0992319F4B8
:1048600027E630E002C02BE330E0C9010895CF9382
:10487000DF93DC0152969C915297943009F0F2C07C
:1048800058968C915897813039F0843029F08032D5
:1048900019F0803809F051C082E0A83FB80761F4F0
:1048A0005C968C915C97882319F08FB58F7A02C043
:1048B0008FB580658FBD0EC05C968C915C97882308
:1048C00021F080918B008F7A03C080918B008065EE
:1048D00080938B0053968C91539780FD03C0C7E65D
:1048E000D0E00CC090E05C968C915C97882309F432
:1048F00091E05C969C935C97CAE9D0E053968C91CA
:1049000053978823A1F458968C915897803879F45E
:1049100082E0A83FB80721F48FB580658FBD05C040
:1049200080918B00806580938B00CD5ED94F809104
:1049300036038F7E8093360351C082E0A83FB807CC
:10494000C1F488B599B58736910540F090E0809123
:104950001403882309F491E09093140380911403C5
:10496000882319F08FB58F7A02C08FB580658FBD0F
:104970001FC080918600909187008736910550F086
:1049800090E05C968C915C97882309F491E05C96AA
:104990009C935C975C968C915C97882321F0809126
:1049A0008B008F7A03C080918B00806580938B0091
:1049B00058968C915897803111F0803441F4809151
:1049C0003603806180933603CDE4D8E107C080913F
:1049D00036038F7E80933603C7E6D0E053968C91E2
:1049E0005397882309F0D3C058969C9158979230DA
:1049F00041F457968C915797883018F0C7E6D0E06D
:104A0000C6C059962C91599703C0892F822311F45F
:104A1000990FD9F758969C93589757961C92579789
:104A20009031D1F0913140F4943091F0983091F080
:104A3000923009F0ACC008C0903471F0903871F039
:104A4000903209F0A4C006C050968C91509707C0D0
:104A50008CE205C084E003C081E001C088E0539689
:104A60008C9395C082E0A83FB80721F48FB580658C
:104A70008FBD05C080918B00806580938B0054961C
:104A80008C915497882331F455968C9155978823AF
:104A900031F40BC0815054968C93549704C08150CC
:104AA00055968C93559781E01CC0933039F45C96F1
:104AB0008C915C97882311F080E013C053962C9161
:104AC0005397822F869586958695FD01E80FF11DF7
:104AD000808190E0277002C0959587952A95E2F72E
:104AE000817052969C915297923019F0933019F53B
:104AF00003C0CBE6D0E021C0882319F4CEECD0E08F
:104B000002C0C7E7D0E053968C9153978823A9F44D
:104B10005B968C915B97882381F48091380380FDAC
:104B200002C082E001C086E055968C93559781E0E3
:104B30005B968C932CC0C7EDD0E053968C91539725
:104B4000882329F555968C915597882301F5519620
:104B50008C91882399F48091360380FF18C080914E
:104B600037038823A1F481E00E941267882319F09B
:104B7000C35BDF4E0CC0CD5ED94F09C0913029F028
:104B8000923029F4C857DD4F02C0C05FDA4FCE0122
:104B9000DF91CF910895FC018089838B81898230D8
:104BA00010F482E0818B82898330D1F0843018F454
:104BB0008130C0F00AC08430A9F482E0868B91E095
:104BC000908F8189882309F4918B81E00E9412677C
:104BD000882319F423E136E007C02DE430E104C056
:104BE00080E1848B22E330E0C901089580E1E9E3AC
:104BF000F3E0DF011D928A95E9F7109249031092C4
:104C00004B0310924A038FEF9FE790934D038093DD
:104C10004C0308952F923F924F925F926F927F9232
:104C20008F929F92AF92BF92CF92DF92EF92FF92BC
:104C30000F931F93CF93DF935C014B01442428E033
:104C40006731720711F444244394D40111969C9166
:104C500011978C91891709F036C1442029F480916D
:104C6000360388608093360380913703813041F4A6
:104C7000C40160E070E040E050E022E000E882C063
:104C800080913703823071F4C0903403D0903503A3
:104C9000EE24FF24C40160E070E040E050E021E039
:104CA00000EC0FC18091380382FF27C0F40182819C
:104CB0009381A481B5810097A105B105F1F4C401E8
:104CC00060E070E040E050E022E00EE8CC24DD241B
:104CD00076010E94E1218091370790913807A091D9
:104CE0003907B0913A0788519C4FAF4FBF4FF4013D
:104CF00082839383A483B583E6C08091380381FFC8
:104D000030C0F40186819781A085B1850097A10507
:104D1000B10539F5C40160E070E040E050E021E009
:104D20000FE8CC24DD2476010E94E121C40160E07B
:104D300070E040E050E021E000E90E94E121809134
:104D4000370790913807A0913907B0913A078854F6
:104D5000944FAF4FBF4FF40186839783A087B187ED
:104D6000B2C0442019F00E941B3702C00E943C3997
:104D7000EC01009759F4C40160E070E040E050E0BD
:104D800021E001E0CC24DD2476019BC0898590E000
:104D9000837090708230910541F0833091050CF45E
:104DA00069C0039709F08FC051C0C8840E941837AA
:104DB00065E00E94009F923029F1933030F49923EE
:104DC00051F0913009F07FC011C0933039F1943027
:104DD00009F079C02FC068817981DD24EE24FF2499
:104DE000C40140E050E021E001E06BC068817981BE
:104DF000CC80DD80EE80FF80C40140E050E021E007
:104E000001E45FC068817981CC80DD80EE80FF8025
:104E1000C40140E050E021E002E453C068817981A0
:104E2000CC80DD80EE80FF80C40140E050E021E0D6
:104E300003E447C068817981CC80DD80EE80FF800B
:104E4000C40140E050E021E004E43BC00E94183778
:104E500090E0837090708130910581F082309105EF
:104E60001CF4892B39F02FC08230910599F00397FB
:104E700051F51CC068817981C884AFCF6881798180
:104E8000CC80DD80EE80FF80C40140E050E021E076
:104E900004E017C068817981CC80DD80EE80FF80DE
:104EA000C40140E050E021E005E00BC06881798159
:104EB000CC80DD80EE80FF80C40140E050E021E046
:104EC00006E00E94E121D40111962C911197822FC6
:104ED00090E0FC0153E0EE0FFF1F5A95E1F7880FB9
:104EE000991FE80FF91FE80DF91DC685D7851196A2
:104EF0002C911197822F90E0FC0133E0EE0FFF1F01
:104F00003A95E1F7880F991FE80FF91FE80DF91D91
:104F10002088318811962C911197822F90E0FC0106
:104F200003E0EE0FFF1F0A95E1F7880F991FE80FC6
:104F3000F91FE80DF91D028911962C91822F90E03E
:104F4000FC01B3E0EE0FFF1FBA95E1F7880F991F40
:104F5000E80FF91FE80DF91DC488D588E688F788A1
:104F6000802F8C50823008F05BC0442049F1809142
:104F7000370790913807A0913907B0913A0780938D
:104F8000CE089093CF08A093D008B093D108809119
:104F9000CE089091CF08A091D008B091D108009789
:104FA000A105B105A9F581E090E0A0E0B0E0809313
:104FB000CE089093CF08A093D008B093D10828C012
:104FC0008091370790913807A0913907B0913A073F
:104FD0008093CA089093CB08A093CC08B093CD08D7
:104FE0008091CA089091CB08A091CC08B091CD08CF
:104FF0000097A105B10561F481E090E0A0E0B0E088
:105000008093CA089093CB08A093CC08B093CD08A6
:10501000CE010E940484582E6624772410E040C0FC
:1050200080913703813009F443C080913703823087
:1050300041F4209709F437C6CE010E9469373C013C
:1050400034C6CE010E9469373C01009731F01C2D17
:10505000FC015184F3E05F2221C0802F90E0807C2E
:1050600090708038910539F0803C910561F0803472
:10507000910561F404C010E073E0572E0FC010E0FA
:10508000552453940BC010E0552408C0D5011C9240
:1050900001E010E055245394C0E0D0E041101078B6
:1050A000552001F582E00E9412678823C9F006C0EE
:1050B00063E0562E6624772410E014C0F401828544
:1050C0009385A485B5850097A105B10511F05524F8
:1050D00009C080913403909135036C0100EC69C1E3
:1050E00055245394D40111963C91832F90E0FC01F8
:1050F00053E0EE0FFF1F5A95E1F7880F991FE80F55
:10510000F91FE80DF91D23892150832F90E0FC0140
:1051100033E0EE0FFF1F3A95E1F7880F991FE80F74
:10512000F91FE80DF91D238B222309F035C1809169
:10513000CA089091CB08A091CC08B091CD080097F7
:10514000A105B105C1F06091CA087091CB088091AA
:10515000CC089091CD08685D7F4F8F4F9F4F0E9484
:10516000D018882341F01092CA081092CB081092F0
:10517000CC081092CD088091CE089091CF08A091D4
:10518000D008B091D1080097A105B105C1F0609198
:10519000CE087091CF088091D0089091D108685DB9
:1051A0007F4F8F4F9F4F0E94D018882341F010925D
:1051B000CE081092CF081092D0081092D108F401B6
:1051C00062817381848195816115710581059105E5
:1051D00059F00E94D018882339F0D40112961D92FC
:1051E0001D921D921C921597F4016681778180852E
:1051F0009185611571058105910559F00E94D018BE
:10520000882339F0D40116961D921D921D921C928E
:105210001997F401628573858485958561157105FB
:105220008105910559F00E94D018882339F0D401E6
:105230001A961D921D921D921C921D97442039F5BD
:105240008091C90880FD88C08091CA089091CB08E0
:10525000A091CC08B091CD080097A105B10509F047
:105260007BC08091C90881608093C908809137070D
:1052700090913807A0913907B0913A078093CA08F6
:105280009093CB08A093CC08B093CD0826C0809112
:10529000C90881FD61C08091CE089091CF08A0918E
:1052A000D008B091D1080097A105B10509F054C00C
:1052B0008091C90882608093C908809137079091D6
:1052C0003807A0913907B0913A078093CE089093A0
:1052D000CF08A093D008B093D108F4012181409168
:1052E000C5085091C608822F90E0FC01A3E0EE0FA4
:1052F000FF1FAA95E1F7880F991FE80FF91FE80D26
:10530000F91D57874687D40111962C91119730913A
:10531000C708822F90E0FC0163E0EE0FFF1F6A9543
:10532000E1F7880F991FE80FF91FE80DF91D328B7F
:1053300011962C913091C808822F90E0FC0143E037
:10534000EE0FFF1F4A95E1F7880F991FE80FF91F2D
:10535000E80DF91D338B20C0F4012181822F90E0EC
:10536000FC01B3E0EE0FFF1FBA95E1F7880F991F1C
:10537000E80FF91FE80DF91D128AD40111968C91DE
:1053800011978F5F11968C93119711968C911197AD
:10539000803110F011961C92B2E0B51528F0E1E0D2
:1053A0005E1608F03FC105C0F3E05F1609F07FC448
:1053B0005BC28091360384608093360384E0D5011C
:1053C00052968C935A2C4B2C80E1D5011D928A95D4
:1053D000E9F791E0F501918B83E8818F908F003C94
:1053E00009F45DC0013C48F4033089F0043009F44D
:1053F00042C0013009F0EEC00EC0023C09F49FC06B
:10540000023C08F475C0033C09F0E4C0BFC0D301FE
:1054100018961C911F67812F90E08F7790700097EE
:1054200031F08F37910511F4117801C01F5FF3013E
:105430002481358140E050E04760852D942D68E05F
:1054400004E10E945621682FD50150968C93105884
:10545000212F30E03160442737FD4095542F852DB2
:10546000942D0BE00E945621482FF501808BCE0130
:10547000652D742D0EC0960140E050E04760C501D7
:1054800068E004E10E945621482FF501808BCE018F
:10549000B5010E948321D50150968C939BC08091C9
:1054A000370790913807A0913907B0913A0780519A
:1054B000954FAF4FBF4FF40182879387A487B5877D
:1054C000960140E050E0C50168E000E10E945621ED
:1054D000682FC50124E332E140E050E000E20E9481
:1054E0005621682FC5012DE330E040E050E047C071
:1054F0009E0140E050E0A90133272227C101A0E02E
:10550000B0E0282B392B4A2B5B2BC50168E000E269
:105510000E945621682F2C2D30E040E050E0C5015C
:1055200006E00E945621682FC5012AE330E040E0E2
:1055300050E00E945621482F80E090E044C09E0138
:1055400040E050E0A90133272227C101A0E0B0E0EC
:10555000282B392B4A2B5B2BC50168E000E20E9407
:105560005621682F960140E050E0C5010EE00E94F0
:105570005621682FC5012BE330E040E050E006E003
:105580000E945621482F80E090E082CF9E0140E0AB
:1055900050E0A90133272227C101A0E0B0E0282B69
:1055A000392B4A2B5B2BC50168E000E20E94562193
:1055B000682FC5012CE330E040E050E006E00E9497
:1055C0005621482FC601B5010E948321F501808B29
:1055D0008FEF818FD50150962C91222309F467C358
:1055E000422F41503FE767E051E017C0832F330F50
:1055F00087FD3627842F869586958695F501E80FD9
:10560000F11D808190E0242F277002C09595879529
:105610002A95E2F780FD352741504F3F39F7F501D4
:10562000308345C380913603816080933603D40173
:105630001A961D921D921D921C921D97802F8C50C0
:105640008230B0F482E0F501828BFE0133E0F69502
:10565000E7953A95E1F7F070319621E0E030F207F6
:1056600011F4E0E0F0E0EA5AFD4F949184E00FC0BD
:1056700081E0F501828BCF3FD10521F018F0E0E009
:10568000F0E001C0FE01EA5AFD4F949182E0D5019D
:1056900051968C93892F8295869586958370F50116
:1056A0008283990F990F918382E1808B6114710439
:1056B00009F44AC0043041F0013431F0023421F0E1
:1056C000033411F0043491F4C60181709070892B79
:1056D00039F0D50111968C911197836011968C93B6
:1056E000F3011085442051F0107808C0D3011496BE
:1056F0008C9180FF03C09360F5019183812F90E02E
:105700008F779070892B01F1D30119968C910E94AB
:10571000D63C0F97CCF01F5FF30181850E94EC36D9
:10572000892B51F410FF08C0D50111968C91119767
:1057300091E0892711968C93812F90E08F71907062
:10574000959587951078182B0E3070F40C30F8F47E
:10575000043030F4023070F5013009F0A8C225C0E1
:10576000043009F0A4C221C00234D1F1033430F472
:105770000034D9F0013409F09AC229C0043409F484
:105780004BC00434C8F1053409F091C255C0C7704C
:10579000D070C25CDD4FFE012491D5012C930C30FA
:1057A00009F085C22C7F2C9382C2852D612F0E9427
:1057B000E5203FC0D30118966C9160786F60852D0D
:1057C0000E94E520F501808384E0818B70C2F6940D
:1057D000E794D794C7944C2D4170812F61E017C096
:1057E000B2E0F694E794D794C794BA95D1F74C2DCC
:1057F0004170812F62E01BC0A3E0F694E794D79438
:10580000C794AA95D1F74C2D4170812F63E00E9477
:10581000A920D5018C934BC2F4E0F694E794D79479
:10582000C794FA95D1F74C2D4170812F64E00E9406
:10583000A920F50180833BC2D50111968C91119767
:10584000836011968C93119782E052968C935297B5
:10585000F694E794D794C794F601EF70F070EA5B82
:10586000FD4FE491EC9323C28091360382608093D4
:105870003603F4011286138614861586D5015296D6
:105880005C92529781E051968C93519788E15096A3
:105890008C93063818F5033808F049C1063009F42E
:1058A000D0C0073078F40330F1F1043020F4013037
:1058B00009F0E1C139C0043009F495C0053009F0A0
:1058C000DAC1ADC0023808F02AC1003808F013C1AF
:1058D000802F8C50823008F0CEC119C0013950F4AD
:1058E0000F3808F09DC10E3808F094C1083808F050
:1058F0005AC141C1023909F4AFC0023908F4ABC141
:10590000033909F4B6C0043909F0B5C1C8C040E094
:105910000D3009F441E095012F5F3F4FCE0160E06B
:105920000E942D21A8C11F67F30181858C708830EA
:1059300099F48FE3D50112968C93812F90E08F77A5
:105940009070009731F08F37910511F4117801C0F4
:105950001F5FF5011183B8C017FF04C080E6F50191
:10596000818304C080E4D50111968C93F301818575
:105970000E94D63C212F30E00F97E4F0C9018F77C9
:105980009070009731F08F37910511F412E001C04B
:105990001D5F912F96959F70D50111968C9111974F
:1059A000982B11969C93119710FF46C09061119609
:1059B0009C9342C0C9018F779070009731F08F3768
:1059C000910511F411E001C01F5F212F2F70F50127
:1059D0008181282B2183D30114968C9180FF2CC0C8
:1059E0002061218329C0D701C601B695A795979557
:1059F00087958F708068D50111968C93C601817050
:105A00009070892BC9F0F30181850E94D63C0F97D5
:105A10009CF0D50111968C91119780610BC065E0C7
:105A2000F694E794D794C7946A95D1F78C2D8F702C
:105A3000806BD50111968C93B5016E5F7F4FCE01BF
:105A40006BC059E0F694E794D794C7945A95D1F770
:105A50008C2D8F70806AEDCF4DE0F694E794D7944B
:105A6000C7944A95D1F7D5011196CC9211978EED36
:105A70000CC035E1F694E794D794C7943A95D1F7E2
:105A8000D5011196CC9211978FED12968C93B5019A
:105A90006D5F7F4FCE010E941E21885EEAC0822D7D
:105AA0008F77D50111968C931197C114D104E1041D
:105AB000F10419F0806811968C93B0E82B1631042C
:105AC00070F48DEDF5018283B5016D5F7F4FCE01DE
:105AD0000E941E21885ED50150968C93CCC0F501A2
:105AE00081818283220C232C221C33083194218251
:105AF00080EC838387C0F501118295012E5F3F4FB3
:105B0000013841F4CE01816060E040E00E942D2127
:105B1000805FE1CFCE01B9010E941E21A9C08FEFA5
:105B2000D50112968C93129711961C92A4C0053839
:105B300011F488E708C0043829F484E7D5011396E6
:105B40008C9303C08CE7F50183834E01992D9370EC
:105B5000D50113968C911397892B13968C931397D9
:105B60001296CC9312971196CC92119780E2509690
:105B70008C93509714C080E7F5018283063811F4A6
:105B800088E782839E012770D50112969C91129717
:105B9000922B12969C9312971196CC9211978AE0B1
:105BA00051968C9368C0802F8B58833030F4832DAE
:105BB0008370846EF501838306C0832D83708C6EA1
:105BC000D50113968C93F5012282C182093811F018
:105BD0000C3851F495012C5F3F4FCE01816060E09D
:105BE00040E00E942D2114C00A3811F00D3851F404
:105BF00095012C5F3F4FCE0161E040E00E942D21D6
:105C0000805E37C0B5016C5F7F4FCE010E941E21C0
:105C1000805E61CF8FEBF50182838FE081832BC0A3
:105C20000E9419678FEFD50115968C9315971496DE
:105C30008C9314978EE313968C93139712967C9300
:105C4000129711966C931197003919F48FE71496F7
:105C50008C9380E30EC08C2D8F71D50111968C939F
:105C600095012E5F3F4FCE0161E040E00E942D2163
:105C7000805FF501808BD50150969C919695969505
:105C800096959150E92FFF27E7FDF095EA0DFB1D52
:105C900020E004C080812827915031971916D4F351
:105CA000F501208304C06624772410E0FBC9DF914E
:105CB000CF911F910F91FF90EF90DF90CF90BF9009
:105CC000AF909F908F907F906F905F904F903F909C
:105CD0002F9008951F920F920FB60F920BB60F924E
:105CE00011240F931F932F933F934F935F936F93C1
:105CF0007F938F939F93AF93BF93EF93FF93809185
:105D000033038823B1F08091360380FD07C08BE315
:105D100090E0909387008093860004C010928700E3
:105D20001092860087E790E0909381008093800036
:105D300075C086E193E00E943724AC012091880071
:105D40003091890005972817390728F4509381006E
:105D50004093800017C08091880090918900C2967E
:105D600090938100809380000091880010918900B9
:105D700086E193E00E94CB25080F191F1093810044
:105D80000093800080912903882309F03FC080910F
:105D90002B038823D9F580912E038823B9F58091B0
:105DA0002703882399F481E08093330380917C005A
:105DB000846080937C001FB7789486E193E067E16C
:105DC00078E00E940A261FBF1092330380912703B8
:105DD000815080932703809126038093290390911B
:105DE0002803933021F480E180932A0309C0943082
:105DF00029F481E080932E039093290310922A03C3
:105E000010922B03109232031092310386E193E03B
:105E10000E9484239093870080938600FF91EF91E6
:105E2000BF91AF919F918F917F916F915F914F91B2
:105E30003F912F911F910F910F900BBE0F900FBEAE
:105E40000F901F9018951F920F920FB60F920BB6DE
:105E50000F9211240F931F932F933F934F935F93B0
:105E60006F937F938F939F93AF93BF93EF93FF9322
:105E700080913703882331F08091360385FF02C07B
:105E800010920903809115038823A1F080913603B5
:105E900080FD05C08BE390E099BD88BD02C019BCB0
:105EA00018BC8BE390E09BBD8ABD87E790E097BD6F
:105EB00086BD70C088EF92E00E943724AC012CB5FB
:105EC0003DB505972817390718F457BD46BD0FC0D3
:105ED0008CB59DB5C29697BD86BD0CB51DB588EF36
:105EE00092E00E94CB25080F191F17BD06BD8091B7
:105EF0000B03882309F044C080910D03882309F027
:105F00003FC0809110038823D9F58091090388232D
:105F100089F481E08093150386B7846086BF1FB73C
:105F2000789488EF92E069E677E00E940A261FBF26
:105F30001092150380910903815080930903809189
:105F4000080380930B0390910A03933051F48091DE
:105F50003703882311F084E101C080E180930C03B2
:105F600009C0943029F481E08093100390930B03CF
:105F700010920C0310920D0310921403109213034D
:105F800088EF92E00E9484239BBD8ABD8AB59BB5B1
:105F900099BD88BDFF91EF91BF91AF919F918F9176
:105FA0007F916F915F914F913F912F911F910F9131
:105FB0000F900BBE0F900FBE0F901F9018950E9470
:105FC0002E12833020F0853020F0873011F081E0F0
:105FD000089580913603887008950E940567FC013A
:105FE000808182FF0DC096B3809163009095991FC8
:105FF0009927991F8695869586958095817009C009
:1060000086B390916300969596959695909591702C
:106010008078982B892F08950E940567FC01808164
:1060200082FF02C0C79A0895C79808959C01809185
:10603000C908833011F080E008953093C60820939A
:10604000C508662311F08DE001C08CE08093C7087D
:1060500083E08093C8081092C9080E940567FC017C
:10606000808186FF05C08091C90881608093C9083E
:10607000808187FD02C081E008958091C908826017
:106080008093C90881E008952F923F924F925F92CA
:106090006F927F928F929F92AF92BF92CF92DF9238
:1060A000EF92FF920F931F93CF93DF93EC012B019D
:1060B0003A01222E302E46015701009731F487E134
:1060C00098E00E944430C9E6D7E0809137038823E6
:1060D00021F088E0C731D80701F10E942E128230EA
:1060E000E0F0853010F08730C1F41FB7F894CE018E
:1060F000B201A301222D032D750164010E94E1214B
:106100001FBF882329F485E090E00E943319E5CF72
:1061100080913603877F80933603DF91CF911F9163
:106120000F91FF90EF90DF90CF90BF90AF909F9036
:106130008F907F906F905F904F903F902F90089539
:10614000CF92DF92EF92FF920F93982F80913703B7
:106150008823E9F59923D9F110926A0780916A079B
:10616000809369078EE1E8EFF2E0DF011D928A95E6
:10617000E9F70E942E12873031F480913603816056
:106180008093360311C08BEC92E20E94F63689E6CA
:1061900097E060E070E040E050E02AE002E8CC24C4
:1061A000DD2476010E9444308BE390E099BD88BDE8
:1061B00088B599B59BBD8ABD87E790E097BD86BD40
:1061C0001DBC1CBC87B7846087BFBE9A05C0BE9843
:1061D000C69887B78B7F87BF0F91FF90EF90DF90B6
:1061E000CF900895CF92DF92EF92FF920F93982F66
:1061F00080913703882399F5992389F11092180823
:1062000080911808809317088EE1E6E1F3E0DF0142
:106210001D928A95E9F787E198E060E070E040E040
:1062200050E022E002E8CC24DD2476010E944430D4
:106230008BE390E0909387008093860087E790E05F
:1062400090938100809380001092890010928800C2
:1062500080917D00846080937D00139A07C013981D
:106260001B9880917D008B7F80937D000F91FF9024
:10627000EF90DF90CF9008951F93182F8823E1F1BE
:1062800080E00E94A03080E00E94F23081E064E073
:106290000E942588809162008B7F809362008EE14E
:1062A000E8EFF2E0DF011D928A95E9F782E0809342
:1062B000360383E080930A038FEF8093F8028BE329
:1062C00090E099BD88BD88B599B59BBD8ABD87E72B
:1062D00090E097BD86BD10926A0780916A0780930F
:1062E000690710933703BD9A87B7846087BF82E040
:1062F00090E00E94961907C087B78B7F87BF1092E6
:106300003703BD98C5981F91089581E00E943C31E4
:1063100080913603806180933603089580E00E9467
:106320003C31E2E6F0E080818B7F808380E00E9458
:10633000A03080E00E94F23081E064E00E94258875
:106340000895CF92DF92EF92FF920F93009711F48E
:1063500085EA90E090933503809334036C01EE243A
:10636000FF2489E697E060E070E040E050E024E040
:1063700000EC0E9444300F91FF90EF90DF90CF909F
:10638000089582E00E943C31809136038F7E809395
:1063900036038091370790913807A0913907B09163
:1063A0003A0790E00E94A1310895CF92DF92EF92D8
:1063B000FF920F931F938B019C016A01A90166272D
:1063C0007727EE24FF2489E697E0BA01A80122E0AE
:1063D00003EC0E94443081E01F910F91FF90EF90F9
:1063E000DF90CF900895CF92DF92EF92FF920F93BC
:1063F0001F938B019C016A01A90166277727EE2470
:10640000FF2489E697E0BA01A80122E002EC0E948D
:10641000443081E01F910F91FF90EF90DF90CF907B
:106420000895CF92DF92EF92FF920F931F938B010B
:106430009C01C42EAC0166277727DD24EE24FF24BF
:1064400089E697E0BA01A80122E001EC0E944430FD
:1064500081E01F910F91FF90EF90DF90CF90089512
:10646000CF92DF92EF92FF920F93FC01613091F097
:10647000613018F0623049F51AC0002309F400E4D5
:10648000C22EDD24EE24FF2480E090E0BF01202F07
:106490000BE819C0002309F400E1C22EDD24EE242C
:1064A000FF2480E090E0BF01202F0CE80CC0002307
:1064B00009F400E1C22EDD24EE24FF2480E090E008
:1064C000BF01202F0DE80E94443081E00F91FF9022
:1064D000EF90DF90CF900895CF92DF92EF92FF92EE
:1064E0000F93FC01613091F0613018F0623049F592
:1064F0001AC0002309F400E4C22EDD24EE24FF2498
:1065000080E090E0BF01202F08E819C0002309F4C3
:1065100000E1C22EDD24EE24FF2480E090E0BF01E4
:10652000202F09E80CC0002309F400E1C22EDD246D
:10653000EE24FF2480E090E0BF01202F0AE80E94B3
:10654000443081E00F91FF90EF90DF90CF9008955D
:10655000CF92DF92EF92FF920F939C0180913703CD
:10656000813011F080E00EC0C62EDD24EE24FF2421
:1065700089E697E0B90140E050E021E004E80E949C
:10658000443081E00F91FF90EF90DF90CF9008951D
:10659000CF92DF92EF92FF920F939C01809137038D
:1065A000813011F080E00EC0C62EDD24EE24FF24E1
:1065B00089E697E0B90140E050E021E003E80E945D
:1065C000443081E00F91FF90EF90DF90CF900895DD
:1065D000CF92DF92EF92FF920F939C01809137034D
:1065E000813011F080E00EC0C62EDD24EE24FF24A1
:1065F00089E697E0B90140E050E021E007E80E9419
:10660000443081E00F91FF90EF90DF90CF9008959C
:10661000CF92DF92EF92FF920F939C01809137030C
:10662000813011F080E00EC0C62EDD24EE24FF2460
:1066300089E697E0B90140E050E021E006E80E94D9
:10664000443081E00F91FF90EF90DF90CF9008955C
:10665000CF92DF92EF92FF920F939C0180913703CC
:10666000813011F080E015C06770862F806E442362
:1066700011F0862F886EC82EDD24EE24FF2489E6D3
:1066800097E0B90140E050E021E005E80E94443085
:1066900081E00F91FF90EF90DF90CF900895CF921F
:1066A000DF92EF92FF920F939C018091370381302C
:1066B00011F080E015C06770862F806F442311F0C1
:1066C000862F886FC82EDD24EE24FF2489E697E00C
:1066D000B90140E050E021E005E80E94443081E04B
:1066E0000F91FF90EF90DF90CF900895CF92DF92BF
:1066F000EF92FF920F93282F80E090E060E070E02F
:1067000040E050E002E8CC24DD2476010E944430D1
:1067100081E00F91FF90EF90DF90CF900895CF929E
:10672000DF92EF92FF920F93FC01242F662311F466
:1067300000E801C001E880E090E0BF0140E050E0E7
:10674000CC24DD2476010E94443081E00F91FF903B
:10675000EF90DF90CF900895CF92DF92EF92FF926B
:106760000F939C01C62EDD24EE24FF2480E090E0F0
:10677000B90140E050E021E001E90E94443081E0AD
:106780000F91FF90EF90DF90CF9008952F923F925E
:106790004F925F926F927F928F929F92AF92BF9231
:1067A000CF92DF92EF92FF920F931F93DF93CF93DD
:1067B00000D000D0CDB7DEB71C012A013B01480153
:1067C0005901009709F433C1DC0119968C9190E0CE
:1067D000837090708130910571F08230910524F4BE
:1067E000892B09F417C123C18230910591F10397D8
:1067F00009F01DC198C084269526A626B726C40197
:1068000081709070892B69F0F1016081718180E065
:1068100090E040E050E024E004E0730162010E9457
:1068200044308EE190E0A0E0B0E088229922AA22D4
:10683000BB2281149104A104B10409F4F8C0D10170
:106840006D917C9180E090E040E050E024E005E430
:10685000EAC0D901C80184279527A627B7278983CD
:106860009A83AB83BC8389819A8181709070892BD4
:1068700069F0D1016D917C9180E090E040E050E0C2
:1068800024E004E0730162010E944430B981B1FF49
:106890000DC0F1016081718180E090E040E050E046
:1068A00024E001E4730162010E944430F981F2FFA7
:1068B0000DC0D1016D917C9180E090E040E050E00E
:1068C00024E002E4730162010E94443088E090E019
:1068D000A0E0B0E088229922AA22BB22D301C20103
:1068E00084709070A070B07088169906AA06BB06D6
:1068F00069F0D1016D917C9180E090E040E050E042
:1069000024E003E4730162010E944430B981B4FFC2
:106910008EC0F1016081718180E090E040E050E044
:1069200024E004E480C084269526A626B726D50157
:10693000C4018F719070A070B0700097A105B1056F
:1069400069F0D1016D917C9180E090E040E050E0F1
:1069500024E004E0730162010E944430D501C401C7
:10696000807E9170A070B0700097A105B10569F0AC
:10697000F1016081718180E090E040E050E024E02E
:1069800005E0730162010E944430D501C4018070AA
:106990009E71A070B0700097A105B10569F0D1019A
:1069A0006D917C9180E090E040E050E024E006E0D2
:1069B000730162010E944430D501C4018070907E51
:1069C000AF71B0700097A105B10569F0F101608168
:1069D000718180E090E040E050E024E002E9730142
:1069E00062010E94443080E090E0A0EEBFE1882286
:1069F0009922AA22BB2281149104A104B104B9F006
:106A0000D1016D917C9180E090E040E050E024E085
:106A100003E909C0F1016081718180E090E040E00C
:106A200050E023E004E0730162010E94443081E001
:106A30000F900F900F900F90CF91DF911F910F91BA
:106A4000FF90EF90DF90CF90BF90AF909F908F908E
:106A50007F906F905F904F903F902F900895CF92CE
:106A6000DF92EF92FF920F937C010E946937FC0145
:106A7000009739F18185282F30E023703070213064
:106A80003105FCF02330310584F023303105C9F4A1
:106A90000E94D63C0E97A9F480E090E060E070E0A0
:106AA00040E050E021E002E807C080E090E0B7015C
:106AB00040E050E027E002E0CC24DD2476010E9493
:106AC000443081E00F91FF90EF90DF90CF900895D8
:106AD000CF92DF92EF92FF920F93CF93DF93EC016F
:106AE0000E946937FC01009761F1818583708150B4
:106AF000C084823090F4DD24EE24FF2480E890E00E
:106B0000A0E0B0E0C822D922EA22FB2280E090E097
:106B1000BE0140E050E02BE011C0DD24EE24FF2454
:106B200080E890E0A0E0B0E0C822D922EA22FB226F
:106B300080E090E0BE0140E050E024E003E00E94ED
:106B4000443081E0DF91CF910F91FF90EF90DF9083
:106B5000CF900895CF92DF92EF92FF920F93CF9351
:106B6000DF93EC01C62E0E946937892B61F0DD248A
:106B7000EE24FF2489E697E0BE0140E050E026E0E5
:106B800000E40E94443081E0DF91CF910F91FF90AB
:106B9000EF90DF90CF900895CF92DF92EF92FF9227
:106BA0000F931F93CF93DF938C01C62E0E946937FA
:106BB000EC010097C1F1898590E08370907083307B
:106BC000910534F48130910534F4892B79F02BC090
:106BD000039749F50BC0DD24EE24FF2489E697E0F6
:106BE000B80140E050E024E001E01BC0DD24EE24C9
:106BF000FF2489E697E0B80140E050E022E001E0A0
:106C00000E94443089858F70833069F480E090E081
:106C100060E070E040E050E021E002E8CC24DD24B8
:106C200076010E94443081E0DF91CF911F910F9156
:106C3000FF90EF90DF90CF90089583E08093C90894
:106C40001092CE081092CF081092D0081092D1085E
:106C50008091CE089091CF08A091D008B091D10832
:106C60008093CA089093CB08A093CC08B093CD082A
:106C70008091370790913807A0913907B0913A0772
:106C800088519C4FAF4FBF4F80936B0790936C0719
:106C9000A0936D07B0936E078093190890931A081C
:106CA000A0931B08B0931C08809137079091380778
:106CB000A0913907B0913A078854944FAF4FBF4F16
:106CC00080936F0790937007A0937107B09372073A
:106CD00080931D0890931E08A0931F08B09320086E
:106CE000109273071092740710927507109276072E
:106CF0001092210810922208109223081092240862
:106D000085EA90E0909335038093340380E00E94FD
:106D10003C310E940C67809338031092360381E067
:106D20000E94A03081E00E94F230E2E6F0E0808133
:106D3000846080830895CF92DF92EF92FF920F9349
:106D40007C01062F0E94913783708150823060F45D
:106D500089E697E0B70140E050E0202F02E0CC2424
:106D6000DD2476010E94443081E00F91FF90EF9086
:106D7000DF90CF900895CF92DF92EF92FF920F9322
:106D80001F93CF93DF93EC018B01C42E0E949137A8
:106D90008370833011F080E00CC0DD24EE24FF24EA
:106DA00080E090E0BE01A80124E004E90E944430A4
:106DB00081E0DF91CF911F910F91FF90EF90DF90D5
:106DC000CF90089520E030E08F708950823010F429
:106DD00021E030E0C901089520E030E08F70855057
:106DE000823010F421E030E0C9010895EF92FF9263
:106DF0000F931F93CF93DF937C0102ED18E0C0E067
:106E0000D0E00BC02196E114F10429F0C801F7018C
:106E10000995882329F0055F1F4FC034D10591F7EC
:106E2000CE01DF91CF911F910F91FF90EF900895C8
:106E30008091520308959091920B992319F420E0C8
:106E400030E011C0809151038F5F80935103891707
:106E500010F010925103909151038BE0989F900194
:106E600011242E52374FC9010895CF92DF92EF922D
:106E70000F931F93CF93DF93EC01162F69014423E7
:106E800061F00E940C678823E1F0CE01612FA6011A
:106E9000202F0E2D0E94303205C0A901202F0E2D6B
:106EA0000E946C32EE2069F484E00E94763360E048
:106EB000111161E0CE0141E00E948F338AE00E940F
:106EC0007633DF91CF911F910F91EF90DF90CF90AC
:106ED0000895CF93DF93EC010E942E12873019F4AE
:106EE00023E533E01AC02097B1F03091920BE2ED28
:106EF000F8E020E00EC0808191813B968C179D07C1
:106F000039F48BE0289F900111242E52374F05C091
:106F10002F5F231780F320E030E0C901DF91CF918C
:106F200008950E946937FC01009711F480E00895EC
:106F300081858F7008958F929F92AF92BF92CF926A
:106F4000DF92EF92FF920F931F93DF93CF9300D0C6
:106F500000D000D0CDB7DEB74C01062F0E942E1214
:106F6000873009F447C0C4010E9469375C0100976B
:106F700009F440C07E010894E11CF11CC701B40172
:106F80000E94606AF5012481358146815781002382
:106F9000B9F0C701BA01A9010E946C6A8FEF6DE0D8
:106FA000A7010E94166BF501248135814681578126
:106FB0009A0144275527C401B9010E949F3D1AC078
:106FC000C701F501608500E00E94856A8FEF6AE0E5
:106FD000A7010E94166BF501C480D580E680F7807A
:106FE0008701222733270170C4016085A601202F65
:106FF0000E94C73D26960FB6F894DEBF0FBECDBFE8
:10700000CF91DF911F910F91FF90EF90DF90CF9084
:10701000BF90AF909F908F9008951F93CF93DF9371
:10702000C2EDD8E010E01BC08A85989FC0011124F2
:107030008035910534F0888590E08F779070892BAA
:1070400061F0888580788887888199810E94683579
:107050008881998160E00E949B371F5F2B969091F9
:10706000920B191708F3DF91CF911F9108958F921A
:107070009F92AF92BF92CF92DF92EF92FF920F93C7
:107080001F93DF93CF930F92CDB7DEB74C017A01F8
:107090008B01922F81149104E1F1F401A480B58059
:1070A000C680D780A416B506C606D70691F124304F
:1070B00061F429830E942E129981873031F5F40101
:1070C000E482F5820683178324C0F4011286992393
:1070D00029F0818580628187913031F0F4018185CA
:1070E00080648187943021F0F401818580618187FB
:1070F000F401E482F58206831783C401B801A70175
:10710000960185010E94C63304C0F401818584FF85
:10711000DCCF0F90CF91DF911F910F91FF90EF90F7
:10712000DF90CF90BF90AF909F908F900895EF9297
:10713000FF920F931F93CF93DF93EC01162F042F31
:10714000009709F492C0443051F40E942E12873007
:1071500009F087C0188789C08F7E898786C0898596
:107160000E94D63C482F5985812F90E08F779070F0
:10717000242F30E02817390714F41078142B688571
:10718000611709F472C01A86002329F0898580628C
:107190008987013029F0898580648987043019F056
:1071A000898580618987E62EFF24812F862787FFC6
:1071B00034C097012F7730702115310509F0107810
:1071C000852F8370833011F08823D1F4232B29F08D
:1071D000888199810E94683510C089858C708830BB
:1071E00061F4812F90E08F779070892B31F4612FBB
:1071F0006160888199810E94CC35888199810BC01A
:1072000088819981232B39F00E94CC35888199811E
:107210000E94683502C00E942F351887212F30E068
:10722000C9018F779070892BB1F089858F70855057
:10723000823088F410FD03C0612F6F5F08C008948E
:10724000E108F1082E153F0531F4612F6150888166
:1072500099810E94AA3588819981612F0E94CC353D
:1072600004C0898584FF7BCF77CFDF91CF911F91B9
:107270000F91FF90EF9008950F931F93CF93DF939B
:107280000E942E12873041F4809152038F5F8093C9
:107290005203C3E5D3E01DC09091920B992319F4DA
:1072A000C0E0D0E04EC0809150038F5F80935003C8
:1072B000891738F0809152038F5F809352031092A8
:1072C0005003909150038BE0989FE0011124CE521F
:1072D000D74F8091520390E087709070892BA1F472
:1072E0006885262F30E0C9018F779070892B61F077
:1072F00089858F708550823038F460FD05C06F5FDE
:10730000888199810E94AA358091520387708430C8
:1073100099F489858370813079F44C815D816E8127
:107320007F810EE110E020E030E0042715272627BA
:107330003727CE010E94C6338A858F3F11F08F5FB9
:107340008A87CE01DF91CF911F910F91089580EC34
:1073500092E0E2EDF8E0DF019C011D922150304007
:10736000E1F710925103109250031092920B08957E
:107370009F92AF92BF92CF92DF92EF92FF920F93C4
:107380001F93DF93CF9300D00F92CDB7DEB76C0180
:10739000962E009719F400E010E028C020E2E22EBB
:1073A000F12C00E010E05E010894A11CB11CA8952E
:1073B000C501B70143E050E00E9482A369817A8150
:1073C000CB0101978F5F9F4340F4892D4B8120E0D3
:1073D00030E0F60109950F5F1F4F84E090E0E80E62
:1073E000F91E9CEDE9169FE0F90609F7C8010F9018
:1073F0000F900F90CF91DF911F910F91FF90EF9021
:10740000DF90CF90BF90AF909F900895AF92BF92C2
:10741000CF92DF92EF92FF920F931F93DF93CF9360
:10742000CDB7DEB727970FB6F894DEBF0FBECDBF3E
:107430008FEF9FEFAFEFBFEF8C839D83AE83BF8352
:1074400000E210E05E010894A11CB11C34E0C32EE0
:10745000D12CCC0EDD1EF02EE12EC501B80143E08B
:1074600050E00E9482A389819A818F5F9F4F19F417
:107470008B818F3F39F0C6016F2D7E2D44E050E0A7
:107480000E949AA30E9435120C5F1F4F8FE00C3DA3
:10749000180709F727960FB6F894DEBF0FBECDBFC9
:1074A000CF91DF911F910F91FF90EF90DF90CF90E0
:1074B000BF90AF900895CF92DF92EF92FF920F931B
:1074C0001F93DF93CF9300D00F92CDB7DEB78C011F
:1074D000009709F441C0FC018081918101978F5F81
:1074E0009F4310F540E2E42EF12C6E010894C11C7C
:1074F000D11CA895C601B70143E050E00E9482A3C9
:1075000029813A81F801808191812817390719F47E
:107510008B818F7020C084E090E0E80EF91E9CED16
:10752000E9169FE0F90629F7F80180819181F8E2D8
:1075300080309F0718F0F80111860EC08F3F91052B
:1075400009F028F488E00E941267882311F087E090
:1075500001C082E0F80181870F900F900F90CF91CA
:10756000DF911F910F91FF90EF90DF90CF900895E2
:10757000FF920F931F93CF93DF938C01F62E0E94FF
:107580002E128730E9F480915303909154038017B1
:10759000910709F455C0109354030093530383E5F6
:1075A00093E00E945B3A80915C0390E0837090705E
:1075B0000197029708F444C082E080935C0340C0C6
:1075C000C80101978F5F9F4318F0C0E0D0E03CC036
:1075D000C8010E946937AC010097A9F52091920B70
:1075E000203450F48BE0289FE0011124CE52D74F75
:1075F0002F5F2093920B10C0E2EDF8E0EF0192852F
:107600008A85891708F4EF013B968BE0E239F80789
:10761000B1F78A858823B9F019830883CE010E94C7
:107620005B3A80E888871C821D821E821F821B8233
:107630001A821A86FF2041F0C8010E94B58004C05A
:10764000C3E5D3E001C0EA01CE01DF91CF911F91E4
:107650000F91FF900895CF92DF92EF92FF921F93C8
:10766000CF93DF936B015FEFE52E5FE7F52EE82206
:10767000F922C70160E00E94B83AEC010097E1F0FE
:1076800018851078D7FC10588FEF9FE7C822D922B1
:10769000C60160E00E94B83AFC01009769F080855D
:1076A0008F77182B1087DB82CA821A86F382E282D8
:1076B0001286C7010E94FC7FDF91CF911F91FF903E
:1076C000EF90DF90CF90089561E00E94B83A08955E
:1076D000CF93DF93EC010E94777F0BC0CE010E9415
:1076E000643BFC01009739F0C281D381138212827E
:1076F0001286209799F7DF91CF910895CF93DF936A
:10770000C2EDD8E08A819B81892B21F08881998103
:107710000E94683B8BE0C738D80711F02B96F2CF58
:10772000DF91CF910895DF92EF92FF920F931F9315
:107730007A018B01D22E0E94643B009729F0B80198
:10774000A7012D2D0E9437381F910F91FF90EF90C8
:10775000DF9008951F93CF93DF93EB01142F0E94C6
:10776000643BFC010097A1F0AE0160E070E0BA015B
:107770005527442784819581A681B781A070B07078
:10778000482B592B6A2B7B2BCF01212F0E94373896
:10779000DF91CF911F9108951F93CF93DF93EB015A
:1077A000142F0E94643BFC01009789F0AE0160E059
:1077B00070E084819581A681B78180709070482B9C
:1077C000592B6A2B7B2BCF01212F0E943738DF9159
:1077D000CF911F9108950E94643BFC01009729F40A
:1077E00020E030E040E050E004C024813581468153
:1077F0005781B901CA0108950E94643BFC010097BA
:1078000011F480E0089580850895FF920F931F93EF
:10781000CF93DF93EC01062FF42E0E942E128330BB
:1078200041F00E942E12873021F084E0F81609F40E
:107830000078CE010E94643BEC010097C1F01885EE
:10784000602F4F2D0E9497388A819B81009779F095
:1078500060E00E94B83AFC01009749F08085182743
:1078600017FD0058CF01602F4F2D0E949738DF91F0
:10787000CF911F910F91FF9008958F929F92BF9289
:10788000CF92DF92EF92FF920F931F93DF93CF93EC
:1078900000D00F92CDB7DEB76C01B62E2FE0B2222A
:1078A00051F482E00E941267882329F482E00E944A
:1078B00097690E94716900E210E0EE24EA94FE2CC0
:1078C0004E010894811C911CA895C401B80143E0A5
:1078D00050E00E9482A389819A818C159D0511F444
:1078E00078010FC02FEFE2162FEFF20621F480503F
:1078F000904408F078010C5F1F4F8FE00C3D180793
:1079000019F729813A812C153D0541F08FEFE816D2
:107910008FEFF80619F42FEF3FEF17C08B818B150F
:1079200019F42C153D0579F0BB82DA82C982A8953D
:10793000CE010196B70144E050E00E949AA3C6012F
:107940006B2D0E94E27E20E030E0C9010F900F9085
:107950000F90CF91DF911F910F91FF90EF90DF90EB
:10796000CF90BF909F908F9008951F93CF93DF93F8
:10797000EC01162F0E94643BFC01009799F0412F07
:107980004F706185862F90E08F709070242F30E0CB
:107990008217930739F0607F642B61871286CE01CE
:1079A0000E943D3CDF91CF911F910895E82FF0E0B8
:1079B000EF70F070E85EFB4FE4918E2F90E0089539
:1079C00090E083709070009731F0039711F48CE190
:1079D000089584E008958FE0089583E693E0089584
:1079E00080917F0382FF05C08091650390916603BB
:1079F00008958091630390916403089580917F03BB
:107A000081FD0CC08260877F80937F031092830387
:107A100080E090E060E070E00E94021E08958823FC
:107A2000E9F082E06EE671E00E94A41F83E066E761
:107A300071E00E94A41F84E06EE771E00E94A41F21
:107A400085E066E871E00E94A41F86E06EE871E0C0
:107A50000E94A41F87E066E971E01CC082E06EE22C
:107A600071E00E94A41F83E06EE371E00E94A41FF6
:107A700084E06EE471E00E94A41F85E066E571E099
:107A80000E94A41F86E06EE571E00E94A41F87E0BB
:107A900066E671E00E94A41F08958091620383301E
:107AA00014F010926203809162038F5F80936203EF
:107AB0008150813041F0823061F0882379F481E097
:107AC00066E372E003C081E06EE272E00E94A41FF0
:107AD000089581E066E272E00E94A41F0895882361
:107AE00021F082E066EB71E003C082E06EEA71E0B3
:107AF0000E94A41F0895882321F081E066EA71E0C6
:107B000003C081E06EE971E00E94A41F0895809394
:107B100093030E943112089520917F0321FD0EC02E
:107B20002B7F216020937F039093660380936503EE
:107B300070936E0360936D030E9431120895E0917B
:107B40006303F09164038E179F0711F0EF2BF1F49C
:107B50009B0140E050E0A90133272227809169036F
:107B600090916A03A0916B03B0916C03A070B07008
:107B7000282B392B4A2B5B2B2093690330936A0304
:107B800040936B0350936C030E9431120895FC01E3
:107B90008091630390916403E817F90711F510923F
:107BA00082036093810360E070E0809169039091AB
:107BB0006A03A0916B03B0916C0380709070482BA6
:107BC000592B6A2B7B2B222311F0616001C06E7F41
:107BD0004093690350936A0360936B0370936C0343
:107BE0000FC08091650390916603E817F90751F47F
:107BF000109282036093810350936E0340936D0350
:107C00000E94311208951F93182F80E06CE00E94AB
:107C1000C31E112309F100D000D00F92EDB7FEB7BB
:107C2000319682E0ADB7BEB711968C938BEB93E0A3
:107C3000928381838091830390E08F779070948307
:107C400083830E943D200F900F900F900F900F9014
:107C500080E00E947A1E05C082E066EB73E00E941D
:107C600097201F910895EF92FF920F931F93182F63
:107C700080FF02C083E001C085EA0E947A1EE12EE7
:107C800011FF02C084E001C085EA0E947A1EE2FE74
:107C900002C085E001C085EA0E947A1EE3FE02C0B0
:107CA00086E001C085EA0E947A1EE4FE02C087E0F9
:107CB00001C085EA0E947A1E1F910F91FF90EF90FC
:107CC000089560916F03709170038091710390919A
:107CD0007203611571058105910561F00E94D0184C
:107CE000882341F010926F03109270031092710379
:107CF0001092720360917303709174038091750305
:107D000090917603611571058105910571F00E94CE
:107D1000D018882351F010927303109274031092BC
:107D20007503109276030E9431126091770370916F
:107D300078038091790390917A036115710581052B
:107D4000910561F00E94D018882341F010927703CA
:107D5000109278031092790310927A038091820333
:107D600018166CF42091810330E02F7730708091E9
:107D7000840390E02817390714F010928203809151
:107D8000820387FF09C08091810390E08F77907014
:107D9000892B11F4109282038091820320915E035B
:107DA00030915F034091600350916103882381F417
:107DB000211531054105510511F00E943112109233
:107DC0005E0310925F0310926003109261030895A6
:107DD000211531054105510539F0CA01B9010E944B
:107DE000D018882309F46CC080918203181644F4DB
:107DF0000E942E12833049F4809181038F5F03C06B
:107E0000809181038150809381038091820381302E
:107E100059F08F3F49F0823061F08E3F51F028E8F1
:107E200033E140E050E009C020E335E740E050E0B6
:107E300004C020EE3EE240E050E0809184038E37A3
:107E400081F48091370790913807A0913907B0915C
:107E50003A07E7E05695479537952795EA95D1F784
:107E600021C08E3081F48091370790913807A0911E
:107E70003907B0913A0774E056954795379527959D
:107E80007A95D1F70FC08091370790913807A0916C
:107E90003907B0913A0765E056954795379527958C
:107EA0006A95D1F7280F391F4A1F5B1F20935E0385
:107EB00030935F0340936003509361030E9431123B
:107EC000089580917F0380FD25C060916F037091BC
:107ED00070038091710390917203611571058105A2
:107EE000910521F00E94D0188823A1F0109266031A
:107EF000109265031092860310928503109264031A
:107F00001092630310927F03109287030E94311234
:107F100081E0089580E00895DF92EF92FF920F9341
:107F20001F9310919303112399F081E060E00E9468
:107F3000C31E812F81500E94B866BC0182E00E945E
:107F400097201092930388EE93E00E94961902C046
:107F5000882319F00E94B71E04C080E060E00E94F0
:107F6000C31E8091630390916403892BF9F00E94F2
:107F70000567FC0140916303509164038281938102
:107F80008417950749F42185328580918503909166
:107F900086032817390751F0538342838091850364
:107FA00090918603928781870E9471692091630373
:107FB0003091640321153105C9F4109269031092C0
:107FC0006A0310926B0310926C031092820310925A
:107FD0006E0310926D0310928103109283038091BF
:107FE0007F038F7E80937F031092800380917F03B5
:107FF00082FD0DC080917B0390917C03A0917D0355
:10800000B0917E030097A105B10531F430C082E044
:1080100065E174E00E9497208DB79EB707970FB671
:10802000F8949EBF0FBE8DBFEDB7FEB7319682E0CC
:10803000ADB7BEB711968C9382E094E092838183B2
:1080400080917B0390917C03A0917D03B0917E038E
:1080500083839483A583B6830E943D20EDB7FEB74A
:1080600037960FB6F894FEBF0FBEEDBF51C0211575
:10807000310531F482E06BEF73E00E94972021C05C
:1080800000D000D00F92EDB7FEB7319682E0ADB7C9
:10809000BEB711968C9386EF93E0928381833483ED
:1080A00023830E943D2080917F030F900F900F90BB
:1080B0000F900F9080FF02C081E001C080E20E941B
:1080C0007A1E109180030E942E12682F863008F0CD
:1080D0006150633091F48091630390916403892B24
:1080E00061F0612F70E06370707013E0660F771FAE
:1080F0001A95E1F76A5A7C4F08C070E0B3E0660F4A
:10810000771FBA95E1F76A587C4F82E00E9497206A
:1081100080E06CE00E94C31E80917F0383FF12C049
:1081200000D000D00F92EDB7FEB7319682E0ADB728
:10813000BEB711968C9382EF93E0928381838091F6
:10814000830311C000D000D00F92EDB7FEB7319677
:1081500082E0ADB7BEB711968C938EEE93E092831A
:1081600081838091810390E08F77907094838383E3
:108170000E943D200F900F900F900F900F908091D4
:10818000630390916403892B89F08091800383704D
:10819000813081F487E10E94E01C882339F080E07F
:1081A0000E947A1E80E06EEE71E05BC080E20E9469
:1081B0007A1E59C080E00E947A1E0E940567FC0169
:1081C000808185FF43C08091810387FF04C080E0E8
:1081D00062EF70E003C080E066EF70E040E024E012
:1081E0000E946D1F809182038823E1F018163CF0F5
:1081F0008E3F81F08F3F94F48D3FA9F507C0823008
:10820000C9F082309CF0833071F518C080E062E1E3
:1082100071E017C080E06EE071E013C080E06AE0BA
:1082200071E00FC080E06AEF70E00BC080E06EEF9D
:1082300070E007C080E062E071E003C080E066E0CB
:1082400071E044E024E00E946D1F0DC08091810325
:1082500087FF04C080E062EE70E003C080E06AEE59
:1082600070E00E94A41F0E942E12813049F489E020
:108270000E94D566AC0181E060E00E941D1F03C230
:1082800080917F0383FD06C080E060E040E050E025
:108290000E94CC1E80917F0387FD03C000E010E0A8
:1082A00014C08091650390916603892B19F001E059
:1082B00010E00BC0809180030E94E03C20E030E0A1
:1082C000853010F021E030E08901F02E81E060E09F
:1082D0000E94C31E80917B0390917C03A0917D033B
:1082E000B0917E030097A105B10509F429C18DE085
:1082F0000E94E01C882329F48EE00E94E01C882361
:1083000081F100D00F9282E0EDB7FEB7818382EE5B
:1083100093E0938382830E943D200F900F900F90F3
:108320008DE00E94E01C882369F081E066EA71E03C
:108330000E94A41F82E06EEA71E00E94A41F8BE7F6
:108340009DE30CC081E06EE971E00E94A41F82E011
:1083500066EB71E00E94A41F8FE69DE36CE271E082
:10836000ECC087E00E94D566BC0182E00E949720A5
:1083700087E00E94D5660E94A9A0182F04C080E261
:108380000E947A1E1F5F1031D0F310918003812F5D
:108390000E94E03C90E0A0E0B0E020917B033091AF
:1083A0007C0340917D0350917E0382179307A407BD
:1083B000B5070CF44DC081E06BE00E94C31E6091D4
:1083C0007B0370917C0381E090E0A0E0B0E0062E9A
:1083D00004C0880F991FAA1FBB1F0A94D2F72091CF
:1083E000690330916A0340916B0350916C038223BF
:1083F0009323A423B5230097A105B10519F425EA19
:1084000030E002C023E030E08DB79EB707970FB68B
:10841000F8949EBF0FBE8DBFEDB7FEB7319682E0D8
:10842000ADB7BEB711968C9389ED93E092838183AB
:10843000CB0163839483368325830E943D20EDB76F
:10844000FEB737960FB6F894FEBF0FBEEDBFC0C0A3
:108450001370133009F0BCC08FE00E94E01C882329
:1084600051F480E10E94E01C882329F48CE00E94F2
:10847000E01C882369F180E10E94E01C882321F040
:1084800081E066E272E003C081E06EE172E00E948A
:10849000A41F81E06FE00E94C31E00D000D00F92A5
:1084A000EDB7FEB7319682E0ADB7BEB711968C93AB
:1084B00086ED93E09283818381E090E094838383CF
:1084C0000E943D200F900F900F900F900F90DBC0F7
:1084D00081E066E272E00E94A41F81E06BE00E94EE
:1084E000C31EEDB7FEB739970FB6F894FEBF0FBEA7
:1084F000EDBF319682E0ADB7BEB711968C938DEC8F
:1085000093E09283818386E090E09483838387E085
:1085100090E09683858381E090E0908787830E9436
:108520003D20EDB7FEB739960FB6F894FEBF0FBEEB
:10853000EDBF8DE49DE368EC70E00E94021EA3C0D5
:1085400020916503309166032115310539F100D082
:1085500000D00F92EDB7FEB7319682E0ADB7BEB74F
:1085600011968C9388EC93E09283818334832383E8
:108570000E943D200F900F900F900F900F908091D0
:108580006D038F710E94333E002321F08CE30E9423
:108590007A1E2DC080E20E947A1E1CC000D000D03E
:1085A0000F92EDB7FEB7319682E0ADB7BEB7119628
:1085B0008C938FEB93E09283818387E893E094839D
:1085C00083830E943D200F900F900F900F900F908B
:1085D000FF2069F48091730390917403A091750357
:1085E000B09176030097A105B10509F444C08091CC
:1085F000650390916603892BF1F5809180030E94B9
:10860000E03C8530C0F181E060E00E94C31E86E45A
:108610000E947A1EA2E0EA2EF12C012D112DDD24FC
:10862000D3948091690390916A03A0916B03B091F8
:108630006C038E219F21A023B1230097A105B105D2
:1086400049F0B9E0BD1518F08D2D805D04C08D2D69
:10865000885001C085EA0E947A1ED394E0E1DE16BC
:1086600029F0EE0CFF1C001F111FDBCF80E20E94DF
:108670007A1E81E006C0809169038F710E94333EAB
:1086800080E00E940F3D1F910F91FF90EF90DF90CF
:108690000895CF93DF93EB0180938003E82FF0E000
:1086A000EF70F070E85EFB4FE491E0938403611596
:1086B000710559F0CB0160E070E047E853E00E949B
:1086C000DE7DD0938603C09385030E943112DF9133
:1086D000CF9108951F93FC01009769F410927F03D6
:1086E00010926F0310927003109271031092720334
:1086F0000E94613F64C070917F0371FD60C0609310
:108700008103CA01A0E0B0E02091690330916A03BF
:1087100040916B0350916C0320703070822B932B2F
:10872000A42BB52B8093690390936A03A0936B03EA
:10873000B0936C038091370790913807A091390767
:10874000B0913A0788519C4FAF4FBF4F81608093E3
:108750006F0390937003A0937103B093720372FF41
:1087600025C071607B7F70937F03F0936603E09375
:108770006503CF010E946937FC01009761F0809189
:1087800081039085892787FF06C0609165037091FA
:108790006603706804C06091650370916603809100
:1087A0006303909164030E942B3B07C07E7F70930C
:1087B0007F03F0936403E09363030E9431121F91DF
:1087C0000895AC0180917F038C7F80937F0310928A
:1087D000860310928503662309F045C01092870333
:1087E00020916303309164032115310521F030930A
:1087F0006803209367031092690310926A03109232
:108800006B0310926C0310926E0310926D03109222
:108810006603109265031092640310926303109232
:108820008203109280031092930B4115510551F170
:108830008FEFBA010E94536980917F0381FD22C0AE
:108840001092690310926A0310926B0310926C03EA
:1088500010926603109265031092640310926303F2
:10886000109280030DC01092930B6091630370917E
:1088700064038FEF0E94D16880917F0381FD02C065
:1088800090E001C091E080917F038B7F82608093B4
:108890007F03892F0895CF93DF93EC01288D398DC5
:1088A0004A8D5B8D203088E2380780E0480780E001
:1088B00058071CF08C8D86FF5DC0203080E438079F
:1088C00080E0480780E058070CF054C06A817B8143
:1088D000211531054105510509F443C061157105A4
:1088E000E1F088819981A0E0B0E082179307A407A6
:1088F000B50741F0CB01A0E0B0E082179307A407D1
:10890000B50759F48C8D8E7F8C8F888199810E9458
:10891000683B1B821A821982188288819981A0E0A3
:10892000B0E0288D398D4A8D5B8D82179307A4079F
:10893000B50729F48C8D91E089278B7F16C081E0E3
:1089400060E00E94C31E80E00E94D566BC0182E008
:108950000E9497206C8D6470888D998D0E94E143F0
:1089600005C0672B19F48C8D84608C8F188E198E3E
:108970001A8E1B8EDF91CF910895DF92EF92FF92B6
:108980000F931F939C018531910509F465C38631CE
:10899000910524F58C30910509F480C18D30910545
:1089A000A4F48A30910544F4813091050CF0AAC3F7
:1089B000009709F45BC3F0C38A30910509F4D4C36E
:1089C0008B30910509F0E8C3C6C3813191050CF0E5
:1089D00054C28F3091050CF0BFC206C28A3891058F
:1089E00009F4BEC38B389105C4F48B31910564F44E
:1089F000893191053CF58631910509F4E1C2873151
:108A0000910509F0C9C30FC18132910509F4D0C2A3
:108A10008332910509F0C0C3B6C38F3891054CF479
:108A20008D3891050CF0E0C18C38910509F0B4C384
:108A3000B5C1813991050CF4ADC28739910509F0B2
:108A4000ABC3A8C380917F0383FF03C0109183034E
:108A500002C01091810300E02931310509F401E0E1
:108A6000E09084030E940567FC01F7800E9405677F
:108A7000FC01808184FF35C017FD05C080E0002324
:108A800009F481E0082F002311F001E02CC0812FB0
:108A900090E08F779070892B79F480917703909193
:108AA0007803A0917903B0917A030097A105B105ED
:108AB00019F4212F2058ADC08091370790913807C5
:108AC000A0913907B0913A07845D9E4FAF4FBF4FD9
:108AD0008093770390937803A0937903B0937A03FC
:108AE00024C0002311F10E940567FC01808185FFED
:108AF00007C08091820383300CF08AC08F5F21C051
:108B00000E942E12833009F083C0812F90E08F776E
:108B100090702E2D30E0821793070CF079C0FEE79D
:108B2000EF16E1F5FF20E1F439C00E940567FC0172
:108B3000808185FF09C0809182038E3F0CF468C05C
:108B400081508093820364C0812F90E08F77907072
:108B5000892B09F45DC04EE7E41641F5FF2031F1A1
:108B600081E0F81619F460E820E00EC0E2E0FE169D
:108B700019F46EE324E108C0F3E0FF1619F466E18E
:108B80002AE002C060E820E8812F90E030E0002376
:108B900041F08F779070821793075CF4212F2F5F3D
:108BA00038C08F779070281739071CF0212F21507B
:108BB00030C0462F50E0812F90E08F77907048179B
:108BC00059071CF0212F2E7F04C0212F261B2C7F3C
:108BD000260F211719F0002319F41BC0002361F0A0
:108BE000822F90E08F7790708417950714F482E0BD
:108BF00001C084E0280F0DC0822F90E08F77907025
:108C00004817590714F082E001C084E0281B01C016
:108C1000212F80917F0383FF03C02093830320785B
:108C200020938103B7C290917F0397FF21C088E012
:108C3000892780937F0383FF0EC0809181038093F7
:108C400083038078809381031092820383E09EE304
:108C500060E971E00AC080918303809381031092E0
:108C6000830380E090E060E070E00E94021E92C208
:108C7000809180038370813029F480E06EEE71E092
:108C80000E94A41F80918103805880788093810383
:108C90001092820380917F03877F72C28091650367
:108CA00090916603009709F049C0E0907B03F09033
:108CB0007C0300917D0310917E031E141F04100697
:108CC0001106E4F5D09080038D2D0E94E03C90E0E9
:108CD000A0E0B0E08E159F05A007B1071CF181E070
:108CE00090E0A0E0B0E004C0880F991FAA1FBB1F4E
:108CF000EA94D2F72091690330916A0340916B03A3
:108D000050916C0382279327A427B527809369038A
:108D100090936A03A0936B03B0936C0380917F03DD
:108D200080683BC143E0D422D41609F033C280915D
:108D3000630390916403B70141E026C160917F0312
:108D400067FF10C0892B71F080916D0390916E03C5
:108D500021E030E08227932790936E0380936D0388
:108D6000606119C08091690390916A03A0916B03BF
:108D7000B0916C0321E030E040E050E0822793277F
:108D8000A427B5278093690390936A03A0936B038C
:108D9000B0936C036F7E60937F03FCC18091650389
:108DA00090916603892B29F480917F038F778093BC
:108DB0007F0380917F0385FFEDC120917B0330917C
:108DC0007C0340917D0350917E0312161306140616
:108DD00015060CF0DFC08091630390916403B90124
:108DE00040E00E94BB36D6C080917B0390917C030B
:108DF000A0917D03B0917E030097A105B105D9F143
:108E0000893FE7E09E07E0E0AE07E0E0BE070CF038
:108E1000C1C1AC0141505040440F551FC9018F776B
:108E200090700E9709F4416027FF1FC0CA0160E0EF
:108E300044E00E94868680917F0383FD05C080E028
:108E400090E060E070E004C083E09EE360E971E0E0
:108E50000E94021E81E066E271E00E94A41F82E08F
:108E60006EE271E00E94A41F9AC0CA0161E044E072
:108E70000E9486868FC127FD8DC1022F0D50109153
:108E80007F0317FF0AC08091650390916603892BC9
:108E900021F4213131050CF40C5F809180030E9494
:108EA000E03C081708F076C10430A0F08091370745
:108EB00090913807A0913907B0913A078C509E4F96
:108EC000AF4FBF4F8093730390937403A0937503C8
:108ED000B093760317FF1DC08091650390916603E0
:108EE000892BB9F082E090E0A0E0B0E004C0880FE8
:108EF000991FAA1FBB1F0A95D2F720916D033091CD
:108F00006E032827392730936E0320936D03106179
:108F100020C082E090E0A0E0B0E004C0880F991F7C
:108F2000AA1FBB1F0A95D2F72091690330916A03EB
:108F300040916B0350916C0382279327A427B52798
:108F40008093690390936A03A0936B03B0936C03BF
:108F50001F7E10937F031EC1E0907B03F0907C0383
:108F600000917D0310917E03E114F10401051105C8
:108F700009F483CF809163039091640340E02F3024
:108F8000310509F441E0B7010E94BB3680917F03AF
:108F90008062F6C080917F038F7D80937F03109263
:108FA0007B0310927C0310927D0310927E03F2C02B
:108FB00080916303909164036CE30E949B36EAC046
:108FC00080917B0390917C03A0917D03B0917E03FF
:108FD0000097A105B10571F180917F0382FD2AC040
:108FE0000E942E12833019F580918403282F30E0DF
:108FF00040E050E080917B0390917C03A0917D0341
:10900000B0917E03281739074A075B0744F4209381
:109010007B0330937C0340937D0350937E038091C8
:109020008103807890917B03892B80938103109238
:109030008203B5CFF89483E00E94491287E10E9431
:10904000E01C882339F080916303909164036BE402
:109050000E949B3678949EC080917F0387FF02C058
:1090600082E001C080E00E94491294C080917F0399
:1090700087FF12C08091670390916803009709F4FD
:109080008BC0A0E0B0E080937B0390937C03A0931F
:109090007D03B0937E031EC082FF21C080917B03BD
:1090A00090917C03A0917D03B0917E030097A10570
:1090B000B105A9F489E00E94149D80917B039091F1
:1090C0007C03A0917D03B0917E030097A105B105BB
:1090D00009F462C083E693E00E944B445DC0809136
:1090E0007B0390917C03A0917D03B0917E03009758
:1090F000A105B10539F48FEF0E94149D81E00E9413
:109100008C3F4AC079010027F7FC0095102F609131
:109110007B0370917C0380917D0390917E032AE014
:1091200030E040E050E00E94E19EE60EF71E081F8E
:10913000191FF0E0EF16F0E8FF06F0E00F07F0E08F
:109140001F0754F5E0927B03F0927C0300937D03AC
:1091500010937E031FC083E693E00E944B441AC025
:1091600080917F038F770CC010927B0310927C0359
:1091700010927D0310927E0380917F038B7F806825
:1091800080937F0307C0809181038078809381035F
:10919000109282030E9431121F910F91FF90EF9065
:1091A000DF900895FC01EC5BFF4F2081E454F04018
:1091B0002223C1F0E95BFF4F8081E754F0409481A6
:1091C00080FD08C0983511F0983761F4223020F402
:1091D00081E00895892F01C085818095881F8827A7
:1091E000881F089580E0089580E008950F931F93ED
:1091F000CF93DF93182FEB01622F9E0170E02EC0FA
:10920000CA018095909528233923DA01AC23BD2328
:10921000109711F0A1E0B0E06A30B8F46117A8F43B
:10922000862F90E0FC01E295F295F07FFE27E07F2B
:10923000FE27E81BF90BEB5DFB4F8685882329F0A1
:10924000808191818230910508F0CD01892B11F048
:10925000242B352B7F5F440F551F6F5F701780F2F3
:10926000C901DF91CF911F910F910895E82F4423F9
:10927000E9F088E4E89FF0011124EB56FC4F80915F
:109280003304882371F08091250490912604823064
:10929000910538F4892B29F0E95BFF4F80818160CB
:1092A00004C0E95BFF4F80818E7F808381E0089559
:1092B000653069F1663070F4623001F1633028F492
:1092C0006623B1F06130B1F516C06330D1F064307F
:1092D00089F51AC0683021F1693028F46630D1F080
:1092E000673041F51AC06930F1F0603119F51EC0E0
:1092F00064E777E01DC06EE677E01AC06AE677E0C3
:1093000017C067E677E014C061E677E011C06AE550
:1093100077E00EC06FE477E00BC068E477E008C048
:1093200060E477E005C061E377E002C069E277E0DE
:109330000E94972081E0089568E179E00E949720DB
:1093400081E0089561E579E00E94972081E0089529
:109350006EE679E00E94972081E008951F93182F10
:1093600061EE79E00E949720812F62EC79E00E9403
:109370009720812F65EA79E00E94972081E01F9174
:109380000895CF93DF93EC01009719F16FE177E037
:109390000E94A0A0892B11F481E01CC0CE016BE1DA
:1093A00077E00E94A0A0892B11F482E013C0CE01C7
:1093B00067E177E00E94A0A0892B11F483E00AC046
:1093C000CE0164E177E00E94A0A0892B11F480E037
:1093D00001C08FEFDF91CF9108952F923F924F926E
:1093E0005F926F927F928F929F92AF92BF92CF9235
:1093F000DF92EF92FF920F931F93DF93CF9300D0F2
:10940000CDB7DEB79A83898386E9E5E2F4E0DF0130
:109410001D928A95E9F749805A80F201908199233B
:1094200099F09C3289F0943279F0953269F0892F65
:1094300080538A3048F0892F992787FD90950E94A4
:1094400091A0892B09F4DFC095E2692E94E0792E72
:10945000AA24A3941E010894211C311CADC00F5FE7
:109460001F4F1A83098309811A81D801BC908B2D63
:10947000992787FD90950E9491A0892B81F7BB20A9
:1094800009F4AAC0BCE2BB1609F48DC0E7E2BE161F
:1094900029F0F2E2BF1611F0BB2404C00F5F1F4F8A
:1094A0001A83098382E0882E912C860C971CC98030
:1094B000DA80EE24FF2409C0D4011D934D010894E5
:1094C000C11CD11C0894E11CF11CBBE0EB16F1049B
:1094D0009CF4F6011081112379F0BB2019F01B15C3
:1094E00059F70AC01C3241F0812F992787FD9095CA
:1094F0000E9491A0892B01F3D4011C92E981FA8189
:109500008081843241F4CF0101969A838983B1012D
:1095100040E150E013C0853269F4CF0101969A838F
:109520008983B10142E050E00E94339FD3016D93E3
:109530007C9309C0CF01B1014AE050E00E94339F03
:10954000F30171836083E1E0D3011E96EC9304C0C4
:109550000F5F1F4F1A83098309811A81D801FC907C
:10956000FF2081F08F2D992787FD90950E9491A073
:10957000892B41F4BCE2FB1659F704C00F5F1F4F63
:109580001A83098309811A81F801F080FF2079F09C
:109590008F2D992787FD90950E9491A0892B71F7B7
:1095A000FCE2FF1621F40F5F1F4F1A830983A39477
:1095B0008FE090E0680E791EFA2CFA94E981FA8126
:1095C0008081882321F09BE0A91609F04CCF41143B
:1095D000510411F0D2011C928F2D90E00F900F904A
:1095E000CF91DF911F910F91FF90EF90DF90CF907F
:1095F000BF90AF909F908F907F906F905F904F90B3
:109600003F902F9008950894411C511C5A82498222
:1096100002CF0F931F93082F162F603418F064ECBD
:1096200075E002C06CEB75E00E9497201A30A1F142
:109630001B3080F4163021F1173030F41130C1F0B6
:10964000123009F045C018C0183011F1193009F076
:109650003FC01AC01E3071F11F3028F41B3001F1D9
:109660001D30B1F521C0113449F1123489F52AC0F9
:10967000802F6CEA75E01BC0802F68E975E017C089
:10968000802F6BE875E013C0802F68E775E00FC08E
:10969000802F65E675E00BC0802F6DE575E007C093
:1096A000802F6BE475E003C0802F62E475E00E94B8
:1096B000972014C0802F6BE275E0F9CF802F60E215
:1096C00075E003C0802F65E175E00E94972002C01D
:1096D000103420F0802F6DE00E94BD1F81E01F91AB
:1096E0000F910895782F6A30C8F46417B8F4862F64
:1096F00090E0FC0144E0EE0FFF1F4A95E1F7E81B04
:10970000F90BEB5DFB4F8685882341F04081518149
:109710002417350718F04115510531F4872F62E001
:109720000E94094B40E050E0CA0108950F931F9337
:10973000082F142F0E949720802F60E20E94BD1FE7
:10974000112319F469EE76E002C06CEE76E0802F0A
:109750000E949720802F6DE00E94BD1F1F910F91E6
:109760000895DF92EF92FF920F931F93CF93DF93B1
:10977000082F7B01EA01D22E10E012C0802F60E298
:109780000E94BD1FCE018E219F21892B11F460E321
:1097900001C061E3802F0E94BD1F1F5FCC0FDD1F42
:1097A0001D1560F3DF91CF911F910F91FF90EF9006
:1097B000DF90089560E00E94BD1F8FEF08950F9322
:1097C0001F93182FFB010181002311F482E011C0C7
:1097D00060E00E94BD1FE02FF0E0E852F34F60818F
:1097E0006095812F0E94BD1F812F60E00E94BD1FE8
:1097F0008FEF1F910F9108950E948E3184E06EEBE0
:1098000071E00E94A41F85E066EC71E00E94A41F35
:1098100081E794E968EC70E00E94021E80E060E05D
:109820000E94C31E0E94063A0E947E7B0E94CC6961
:109830000E944C6781E008950F931F93082F142F07
:1098400082E00E941267882329F482E00E949769CF
:109850000E947169112379F080913304882359F0B3
:1098600060912504709126046115710531F080E442
:109870006030780710F060E070E08FEF0E945B7757
:109880009B01AC01611571058105910501F1ADB731
:10989000BEB717970FB6F894BEBF0FBEADBFEDB7FA
:1098A000FEB7319611960C9384ED95E092838183F7
:1098B00023833483458356830E943D20EDB7FEB752
:1098C00037960FB6F894FEBF0FBEEDBF12C000D0A2
:1098D0000F92ADB7BEB711960C9311978EEC95E031
:1098E00013969C938E9312970E943D200F900F9099
:1098F0000F9081E01F910F910895982F442309F450
:1099000040C0809133048823E1F160912504709177
:10991000260461157105A9F120E46030720788F50D
:10992000272F33272F73307020543F4FAB015070D7
:10993000ADB7BEB71F970FB6F894BEBF0FBEADBF91
:10994000EDB7FEB7319611969C9381E997E092832B
:10995000818374836383768365833087278332872B
:10996000218754874387568745870E943D2081E0A1
:10997000EDB7FEB73F960FB6F894FEBF0FBEEDBF32
:109980000895892F61E00E9458490895682F442363
:1099900071F080913304882351F0809125049091D7
:1099A0002604803C910518F0883E910510F080E077
:1099B00090E0582F423060F080914204882341F0BB
:1099C00020913404309135042F3F310519F010F007
:1099D00020E030E0852F805C883228F0862F61E01F
:1099E0000E945849089500D000D00F92EDB7FEB7FD
:1099F0003196ADB7BEB711966C938CEC97E092831D
:109A00008183852F90E08F739070982F8827820F25
:109A1000911D948383830E943D2081E00F900F90DD
:109A20000F900F900F9008956EE079E00E949720BC
:109A300082E00E94491280E0089583E00E9449126A
:109A400080E0089580E00E94491280E0089560E07F
:109A50000E94BD1F82E00E9449128FEF089580E0AE
:109A60000E9449120E94739D81E008951F93182F50
:109A70000E942E128430D1F0853038F4823071F09B
:109A8000833080F4882331F01EC08730B8F08730EF
:109A9000D1F410C0812F62E778E013C0812F6AE60D
:109AA00078E00FC0812F63E678E00BC0812F67E577
:109AB00078E007C0812F6BE478E003C0812F65E474
:109AC00078E00E94972081E01F910895EF92FF9225
:109AD0000F931F93182F7B01042F83E00E944912DC
:109AE000812FB701402F0E94364D1F910F91FF909B
:109AF000EF900895EF92FF920F931F93182F7B0121
:109B0000042F80E00E944912812FB701402F0E944C
:109B1000364D1F910F91FF90EF9008951F93182FCE
:109B20000E942E12833041F0873031F0823011F4E0
:109B300068E103C060E001C068E0812F0E94BD1FA2
:109B40008FEF1F910895AF92BF92CF92DF92EF9265
:109B50000F931F93CF93DF93182F042F0E942E1281
:109B6000882319F4812F66E016C0002391F08091BC
:109B70003304882371F0A0902504B0902604A1142A
:109B8000B10439F020E0A21628E2B20610F4023047
:109B900028F4812F62E00E94094B58C08091420452
:109BA0008823B9F3C0903404D0903504C114D10493
:109BB00081F331E0C31634E0D30658F7023061F088
:109BC00080915104882341F0C0914304D091440412
:109BD000CF3FD10519F010F0C0E0D0E0C5010E94E0
:109BE00091378370833019F0812F6AE0D4CF9601CA
:109BF00021503040C50160E041E000E0EC2E0E94C1
:109C000035378DB79EB709970FB6F8949EBF0FBE34
:109C10008DBFEDB7FEB73196ADB7BEB711961C93A9
:109C20008AED95E092838183B482A382D682C58235
:109C3000D087C7830E943D2081E02DB73EB7275FC4
:109C40003F4F0FB6F8943EBF0FBE2DBFDF91CF91AF
:109C50001F910F91EF90DF90CF90BF90AF9008953C
:109C6000AF92BF92CF92DF92EF92FF920F931F932A
:109C7000CF93DF93B82E7B0180914204882309F4AF
:109C80007DC080915104423008F478C000913404C2
:109C9000109135040115110509F470C024E001305C
:109CA000120708F47AC06AC0423029F480E090E0DC
:109CB00020E030E019C020914304309144042F3F4C
:109CC000310519F010F020E030E0443058F0809178
:109CD0006004882339F080915204909153048138B4
:109CE000910510F080E090E0D22EC82EC7016EE8FA
:109CF00077E00E94A0A0892B39F0C7016BE877E0DC
:109D00000E94A0A0892B01F5809133048823B1F132
:109D1000C0912504D091260481E0CF3FD80770F58B
:109D2000C70168E877E00E94A0A0892B11F062E0EB
:109D300001C061E0219701501040CE01B3E0880FCF
:109D4000991FBA95E1F711C0809133048823B1F0CF
:109D50008091250490912604009781F020E48030C2
:109D6000920760F40150104060E04A2D98010D2DDB
:109D7000EC2C0E9435378B2D60E002C08B2D61E00A
:109D80000E945849DF91CF911F910F91FF90EF9062
:109D9000DF90CF90BF90AF900895AA24882309F058
:109DA00083CFAA24A394CC24DD24A0CFEF920F93D9
:109DB000FB01828190E087709070582F4427818149
:109DC00090E0482B592B6381848197E0483F5907E5
:109DD00000F590E087709070382F2227862F90E052
:109DE000282B392B2150304083E02F3F380788F44F
:109DF0008081893D29F4CA0162E040E0058104C008
:109E0000CA0162E041E000E0EE240E94353780E0C4
:109E100001C082E00F91EF9008951F93182F442303
:109E200059F080913304882339F080912504909172
:109E300026048830910510F08FEF90E0883010F400
:109E40000E94A3690E940C6700D000D00F92EDB76A
:109E5000FEB73196ADB7BEB711961C9327EE35E02D
:109E600032832183838314820E943D200F900F90C0
:109E70000F900F900F9081E01F9108951F93CF9343
:109E8000DF93142F80E00E94491288EE93E00E9435
:109E90009619112371F080913304882351F0C091F9
:109EA0002504D0912604209721F0CF3FD10519F049
:109EB00010F0CEE4D0E0F89487E00E944912CE0181
:109EC0000E94643BCE0166E90E949B36789481E053
:109ED000DF91CF911F910895875E934091F5613096
:109EE00069F0613028F06230A9F0633051F51EC08E
:109EF0000E940567FC0180818F731DC00E94056769
:109F0000FC0180818F7780830E940567FC0180813E
:109F1000806411C00E940567FC0180818068808395
:109F20000E940567FC0180818F7B05C00E94056748
:109F3000FC018081806C80830E94716920E030E0A8
:109F400002C02FEF3FEFC9010895FB01928180E02D
:109F5000218130E0822B932B63810E946C4F892FEB
:109F6000881F8827881F880F08951F9381309105C7
:109F700031F0875E9340A9F02FEF3FEF26C00E949B
:109F80000567FC018181882311F484E608C08430D0
:109F900011F485E604C08150843008F08150282FE8
:109FA00013C00E940567FC01808190E036E0969521
:109FB00087953A95E1F7182F11700E940567FC010B
:109FC000808187FD1260212F30E0C9011F91089523
:109FD0001F93CF93DF93182F4423A9F1809133046B
:109FE000882341F0209125043091260483E0283E07
:109FF000380710F02FEF3FEF423039F580914204DF
:10A00000882341F0C0913404D0913504CF3FD1056D
:10A0100019F010F0C0E0D0E0C9016C2F0E946C4F25
:10A0200097FD19C000D000D00F92EDB7FEB7319662
:10A03000ADB7BEB711961C938EED97E092838183E6
:10A04000C38314821EC02FEF3FEFC9010E94B54F9A
:10A050009C0197FF05C0812F62E00E94094B19C047
:10A0600000D000D00F92EDB7FEB73196ADB7BEB7B6
:10A0700011961C938BED97E092838183307034832B
:10A0800023830E943D2081E00F900F900F900F904E
:10A090000F90DF91CF911F9108951F93CF93DF937E
:10A0A000182FFB01928180E0218130E0822B932BDD
:10A0B0000E94B54FEC0197FF02C082E009C0812FDA
:10A0C00060E00E94BD1F812F6C2F0E94BD1F8FEF8B
:10A0D000DF91CF911F9108950F931F93CF93DF933B
:10A0E000082F142F0E940567DC0118968C91C82F49
:10A0F000D0E0CC0FDD1F112361F080913304882361
:10A1000041F080912504909126048134910508F452
:10A11000EC010E940567FE01EF5F2E2F2695DC0102
:10A1200018962C930E94056700D000D00F92EDB7CF
:10A13000FEB73196ADB7BEB711960C932DEE37E052
:10A1400032832183DC0118968C9190E0880F991F4F
:10A15000948383830E943D200F900F900F900F9067
:10A160000F9081E0DF91CF911F910F9108950F9390
:10A170001F93CF93DF93082F142F0E940567EC01E4
:10A18000112351F14B8580913304882339F02091BC
:10A190002504309126042531310518F0842F90E0F4
:10A1A0009C012B878C85282F30E0220F331F123023
:10A1B00078F080914204882359F080913404909182
:10A1C00035048230910520F041E08F3F940708F07C
:10A1D000C901969587958C870E9471698DB79EB746
:10A1E00007970FB6F8949EBF0FBE8DBFEDB7FEB7B1
:10A1F0003196ADB7BEB711960C938CE198E092837F
:10A2000081838B85838314828C8590E0880F991FCE
:10A21000968385830E943D208DB79EB707960FB623
:10A22000F8949EBF0FBE8DBF81E0DF91CF911F914B
:10A230000F9108950F931F93FB0102818181882361
:10A2400019F08330C1F40CC00936A8F410E00F5F98
:10A250001F4F159507950E940567FC01008709C0EF
:10A260008091640C002311F0816001C08E7F809387
:10A27000640C80E001C082E01F910F9108950F935C
:10A280001F93082FFB018181882321F0833041F047
:10A2900082E012C00E940567FC011085110F03C007
:10A2A0001091640C1170802F60E00E94BD1F802F00
:10A2B000612F0E94BD1F8FEF1F910F910895EF92A4
:10A2C000FF920F931F93CF93DF93082F142F0E94B9
:10A2D00005677C0180913304882389F087E294E04C
:10A2E00060EF75E00E94A0A0F7012081892B11F496
:10A2F0002B7F02C02460F70120830E940C308091E4
:10A300004204882379F0123008F453C08091340459
:10A3100090913504893C910508F04BC097FD49C0E8
:10A32000F701868380915104882379F085E494E0D5
:10A330006DEE75E00E94A0A0F7012081892B11F439
:10A34000277F02C02860F701208380916004882362
:10A3500059F080915404F7012081893511F421606E
:10A3600002C02E7FF701208380916F04882369F05B
:10A370001530F8F080916104909162048533910565
:10A38000C0F497FD16C0F701808780917E04882372
:10A39000F1F0163070F0C0917004D0917104F4E0C7
:10A3A000C03BDF0730F081EEC130D80710F410E079
:10A3B00006C0802F62E00E94094B0CC01F5F812FF6
:10A3C0000E946B148C179D07C8F3F70111830E943C
:10A3D000716981E0DF91CF911F910F91FF90EF9014
:10A3E00008950F931F93082F142F86E394E06AEFCC
:10A3F00075E00E94A0A0892B19F063E070E002C014
:10A4000061E070E090913304992341F4809142041B
:10A41000882321F0CB010E9485842DC0112361F097
:10A42000992351F020912504309126042F3F3105C6
:10A4300009F010F437FF05C0802F62E00E94094B3D
:10A440001BC080914204A3E0220F331FAA95E1F7BD
:10A45000882371F4C9010E940484019719F063EF05
:10A4600075E002C067EF75E0802F0E94972003C05F
:10A47000C9010E94358481E01F910F9108951F93B7
:10A48000182F68E378E00E949720812F62E378E03C
:10A490000E9497200E9419672DB73EB72750304081
:10A4A0000FB6F8943EBF0FBE2DBFEDB7FEB7319685
:10A4B000ADB7BEB711961C9325E238E032832183F5
:10A4C00063837483858396830E943D202DB73EB7B6
:10A4D000295F3F4F0FB6F8943EBF0FBE2DBF81E0FE
:10A4E0001F9108958F929F92AF92BF92CF92DF9269
:10A4F000EF92FF920F931F93DF93CF93CDB7DEB709
:10A5000066970FB6F894DEBF0FBECDBFE82ECE0122
:10A5100001960E94E87B8D819E8127E0822E912CFE
:10A520008C0E9D1E09E0A02EB12CAC0EBD1E14EEAB
:10A53000C12E16E0D12E53C0B4E0880F991FBA95F2
:10A54000E1F760E1A40120E00E94E67A8501FF24A2
:10A55000D8018D919C910097E1F19C013F77B0E487
:10A5600020303B07B0F5FF2019F480E091E002C0F5
:10A5700081E091E0EDB7FEB737970FB6F894FEBFD4
:10A580000FBEEDBF3196ADB7BEB71196EC92D28239
:10A59000C18294838383368325830E943D20EDB757
:10A5A000FEB737960FB6F894FEBF0FBEEDBFFF2083
:10A5B00049F0D8018D919C9197FF04C08E2D61E2E6
:10A5C0000E94BD1FF3940E5F1F4FB7E0FB1609F00A
:10A5D000BFCF8E2D6DE00E94BD1F8F8198850097A3
:10A5E00009F0AACF66960FB6F894DEBF0FBECDBFB6
:10A5F000CF91DF911F910F91FF90EF90DF90CF905F
:10A60000BF90AF909F908F9008951F93182F0E9436
:10A610007252812F6EE077E00E94972081E01F91B7
:10A620000895EF92FF920F931F93CF93DF93F82E2D
:10A630008B01E42EE901842F0E94D63C2DB73EB752
:10A64000275030400FB6F8943EBF0FBE2DBFEDB778
:10A65000FEB73196ADB7BEB71196FC9227E037E052
:10A660003283218314830383968385830E943D2054
:10A670002E2D30E0C9018370907001974DB75EB701
:10A68000495F5F4F0FB6F8945EBF0FBE4DBF029794
:10A6900078F4C9018C7090708430910519F48F2D75
:10A6A00061E604C0089721F48F2D62E60E94BD1F69
:10A6B0008F2D64E077E00E9497204E2D50E043708C
:10A6C00050704130510569F0423051051CF4452B62
:10A6D000A1F018C04230510541F04330510591F4CA
:10A6E00008C08F2D60E077E00BC08F2D6CEF76E017
:10A6F00007C08F2D68EF76E003C08F2D65EF76E001
:10A700000E9497202097D1F088818823B9F000D04B
:10A7100000D00F92EDB7FEB73196ADB7BEB7119628
:10A72000FC9280EF96E092838183D483C3830E945E
:10A730003D200F900F900F900F900F908F2D6DE098
:10A740000E94BD1FDF91CF911F910F91FF90EF905D
:10A7500008959F92AF92BF92CF92DF92EF92FF92B5
:10A760000F931F93DF93CF93CDB7DEB72D970FB61F
:10A77000F894DEBF0FBECDBF982E80E090E00E941F
:10A78000777C7C018C0132E0C32ED12CCC0EDD1EF7
:10A790005E010894A11CB11C14C0C801B501A6013A
:10A7A0000E94DE7DBC01009779F0892D49819601D8
:10A7B0000E941153C8010E94777C8C018E159F0561
:10A7C00019F00115110549F72D960FB6F894DEBF63
:10A7D0000FBECDBFCF91DF911F910F91FF90EF90F2
:10A7E000DF90CF90BF90AF909F900895AF92BF92AF
:10A7F000CF92DF92EF92FF920F931F93CF93DF934D
:10A80000082F0E9405676C01802F6CED76E00E9496
:10A810009720802F63ED76E00E949720802F6DECCB
:10A8200076E00E949720802F6DE00E94BD1F00D02F
:10A8300000D00F92EDB7FEB73196ADB7BEB7119607
:10A840000C938EEB96E0928381838DE090E094836D
:10A8500083830E943D200F900F900F900F900F90D8
:10A86000802F6FEA76E00E9497200E941967EDB76B
:10A87000FEB737970FB6F894FEBF0FBEEDBF319607
:10A88000ADB7BEB711960C9323EA36E0328321832D
:10A8900063837483858396830E943D20EDB7FEB762
:10A8A00037960FB6F894FEBF0FBEEDBF802F6BE951
:10A8B00076E00E94972081E193E5602F0E94B839ED
:10A8C000802F0E94A953802F6EE876E00E94972087
:10A8D000802F0E947252802F64E876E00E949720B9
:10A8E000C0E0D0E0EE24FF244FE7A42E46E0B42ED3
:10A8F000C7010E940484182F00D000D00F92EDB73A
:10A90000FEB73196ADB7BEB711960C93B282A18255
:10A91000D483C3830E943D200F900F900F900F901F
:10A920000F90113019F068E776E002C06CE776E02E
:10A93000802F0E949720802F6DE00E94BD1F2196DE
:10A94000E8E0F0E0EE0EFF1ECF3FD10589F6802F44
:10A950006EE676E00E949720D6014C914170802FE0
:10A9600064E676E00E94964BF60140814470802FA9
:10A9700066E576E00E94964BD6014C914870802F98
:10A980006BE476E00E94964B00D000D00F92EDB7BA
:10A99000FEB73196ADB7BEB711960C938DE396E036
:10A9A00092838183D60116968C91838314820E94B0
:10A9B0003D20EDB7FEB73196ADB7BEB711960C93FB
:10A9C0008EE296E092838183D60118968C918383E0
:10A9D00014820E943D20EDB7FEB73196ADB7BEB7E9
:10A9E00011960C938FE196E092838183D6011B969A
:10A9F0008C9122E3829FC0011124948383830E945F
:10AA00003D20EDB7FEB73196ADB7BEB711960C93AA
:10AA100080E196E092838183D6011C968C9124E696
:10AA2000829FC0011124948383830E943D200F9054
:10AA30000F900F900F900F90F60181810E946B1480
:10AA400000D000D00F92EDB7FEB73196ADB7BEB7CC
:10AA500011960C9323E036E0328321839483838321
:10AA60000E943D200F900F900F900F900F90802F1D
:10AA70006DEF75E00E94972081E0DF91CF911F91EB
:10AA80000F91FF90EF90DF90CF90BF90AF9008951F
:10AA90001F93182F0E94A953812F63E277E00E9431
:10AAA000972081E01F9108951F93182F1F7701F1C0
:10AAB0001150862F0E94D63C8B3141F08C3171F0C1
:10AAC0008E30B1F4812F90E008960DC083E0189F7E
:10AAD000C00111240B966EE070E007C0812F90E05A
:10AAE000880F991F079669E070E00E94209F162F3B
:10AAF000812F1F9108951F93182F1F7711F480E065
:10AB00001DC0862F0E94D63C8B3151F08C3171F0E4
:10AB10008E3091F4E12FF0E0EA53F74F84910EC0AC
:10AB2000E12FF0E0EB52F74F849108C0E12FF0E005
:10AB3000EF50F74F849102C0812F8F5F1F910895CE
:10AB4000EF92FF920F931F93CF93DF93182F8823D9
:10AB500019F0E0E4FE2E02C070E2F72EC2EDD8E05C
:10AB600000E0EF2CE09430C069858F2D862351F1F1
:10AB700088850E947B55682F812F0E94BD1F2C81E4
:10AB80003D814E815F815695479537952795812F59
:10AB9000622F0E94BD1F812F68810E94BD1F6981A5
:10ABA0006F738C8180FD6064888587FD6068812F6C
:10ABB0000E94BD1F68856F77812F0E94BD1F898508
:10ABC0008E2189870F5F2B968091920B081760F278
:10ABD00080E8DF91CF911F910F91FF90EF90089542
:10ABE0000E947E3B81E00895FF920F931F93CF93C5
:10ABF000DF93042F442309F441C080913304882358
:10AC0000E9F1C0912504D09126042097B9F180E4A0
:10AC1000C030D80798F511E0BFE0FB2E2DC01A30E8
:10AC2000C0F4812F90E0FC01A4E0EE0FFF1FAA9575
:10AC3000E1F7E81BF90BEB5DFB4F8685882349F0B4
:10AC4000608171816115710531F080E460307807B1
:10AC500010F060E070E01F9DF0011124E95DFB4FF2
:10AC600001C031968081882319F08132D1F70DC05F
:10AC7000CE010E942B3B1F5F101788F281E0DF910D
:10AC8000CF911F910F91FF9008957068F1CF0E94AE
:10AC9000063A02C00E94447C80E090E00E94777CEB
:10ACA0000097C1F781E008951F93182F60E02FEF00
:10ACB0003FE30E94724B009769F10E946937FC01E3
:10ACC000009721F4812F61EB78E022C0818590E02C
:10ACD000837090708130910581F0823091051CF471
:10ACE000892B39F017C08230910559F0039791F400
:10ACF0000CC0812F6EEA78E00BC0812F61EA78E00A
:10AD000007C0812F64E978E003C0812F60E978E013
:10AD10000E94972081E01F9108950F931F93CF9376
:10AD2000DF93182FFB01042F928180E0218130E016
:10AD3000282B392BC90101978F5F9F4338F0812F52
:10AD400062E00E94BD1FC0E0D0E015C0002321F0EA
:10AD5000C9010E94643B03C0C9010E946937EC012C
:10AD6000009749F4002319F0812F6BE002C0812F76
:10AD70006AE00E94BD1FCE01DF91CF911F910F911C
:10AD800008951F93CF93DF93182F41E00E948D56B3
:10AD9000EC01009719F1812F60E00E94BD1F2C810A
:10ADA0003D814E815F8191E1569547953795279575
:10ADB0009A95D1F7812F622F0E94BD1F2C813D8172
:10ADC0004E815F8189E156954795379527958A95FC
:10ADD000D1F72F70812F622F0E94BD1F8FEFDF915F
:10ADE000CF911F9108951F93CF93DF93182F41E0C8
:10ADF0000E948D56EC01009799F0812F60E00E942F
:10AE0000BD1F2C813D814E815F8169E0569547953C
:10AE1000379527956A95D1F7812F622F0E94BD1F24
:10AE20008FEFDF91CF911F9108951F93CF93DF9301
:10AE3000182F41E00E948D56EC01009781F0812F80
:10AE400060E00E94BD1F2C813D814E815F8156953F
:10AE5000479537952795812F622F0E94BD1F8FEF51
:10AE6000DF91CF911F9108951F93CF93DF93182FF8
:10AE700041E00E948D56EC01009741F1812F60E086
:10AE80000E94BD1F888569850E947B55682F812F90
:10AE90000E94BD1F8C819D81AE81BF819C01AD014F
:10AEA0005695479537952795622F6F7081709070F2
:10AEB000892B09F06061888587FD6062812F0E947F
:10AEC000BD1F68856F77812F0E94BD1F8FEFDF91B7
:10AED000CF911F910895CF93DF93EB0141E00E9442
:10AEE0008D56FC01009711F48FEF2DC08B818130BE
:10AEF00069F18130E0F0823019F0833019F50AC031
:10AF000022E025C06B3111F4246015C06C31D1F4FE
:10AF1000286011C06C816E3011F423E00CC06C31DC
:10AF200011F427E008C06E3769F42BE004C08C816F
:10AF30008E3741F420E080819181622F0E94B53CE0
:10AF400080E001C082E0DF91CF91089521E06C8123
:10AF50006E30C1F6F0CF1F93CF93DF93182FEB0124
:10AF60006115710559F18F3F51F11370CB010E94AA
:10AF700062A08F3708F08EE7133018F4113020F4F8
:10AF80001BC01330E1F40DC08B3199F4CE0162E4A3
:10AF900070E00E94C7A0009711F0186010C0146004
:10AFA0000EC08C3111F417E00AC08E3711F41BE08B
:10AFB00006C08E3019F403C08E3709F01FEF812FC1
:10AFC000DF91CF911F9108950F931F93CF93DF933C
:10AFD000082F442301F1809133048823E1F0C091CC
:10AFE0002504D09126042097B1F080E4C030D80722
:10AFF000E8F111C080915104882369F085E494E060
:10B000000E94C1498F3F39F066E374E00E94AB575C
:10B01000182F8F3F29F4802F62E00E94094B21C036
:10B02000CE010E946937892B21F0CE01612F0E9449
:10B03000B53CCE01612F0E943D3CCE010E94B97CFF
:10B040009C0180916004882341F0C901BE01412F19
:10B0500024E534E00E94267E03C0C9010E94447C9E
:10B0600081E0DF91CF911F910F910895809142046B
:10B07000882309F0BFCFCFCF1F93CF93DF93182F33
:10B08000442361F180913304882341F1C091250468
:10B09000D0912604209711F180E4C030D80748F100
:10B0A0001DC0812F6BE00E94094B1FC061858091FC
:10B0B0004204882339F086E394E00E94C149682F56
:10B0C0008F3F61F080915104882359F0862F65E409
:10B0D00074E00E94AB57682F8F3F19F4812F62E014
:10B0E000E2CFCE010E94B53C81E0DF91CF911F916C
:10B0F0000895CE010E94643BFC010097B9F6D1CFC0
:10B10000EF92FF921F93CF93DF93182F442351F1B7
:10B1100080913304882331F1C0912504D091260415
:10B12000C038D105F8F080E4C030D807D8F47E01EB
:10B130006F2D606C80E190E00E94B77699233CF01F
:10B1400081E190E06C2F0E94B77697FF03C0812FBA
:10B1500067E00DC08CE190E065E041E00E94CD76B3
:10B1600097FF03C0812F61E002C0812F60E00E9441
:10B170005849DF91CF911F91FF90EF9008950F9361
:10B180001F93CF93DF93182F80E190E00E94AD765C
:10B1900097FD10C0082F805C883228F0812F61E075
:10B1A0000E94584932C081E190E00E94AD76EC01E6
:10B1B00097FF03C0812F67E0F3CF8CE190E065E05B
:10B1C00041E00E94CD7697FDE9CF00D000D00F92EC
:10B1D000EDB7FEB73196ADB7BEB711961C9387E7B2
:10B1E00097E092838183802F90E08F739070982FE7
:10B1F00088278C0F911D948383830E943D2081E0DA
:10B200000F900F900F900F900F90DF91CF911F91A3
:10B210000F9108951F93182FFB01809142048823FA
:10B2200009F461C0442309F45EC08091330488238B
:10B2300009F459C0209125043091260421153105C7
:10B2400009F451C084E02130380708F45AC04BC0DB
:10B2500060913404709135046F3F710519F010F05E
:10B2600060E070E083818434B1F085341CF4823472
:10B27000D1F516C0803551F08235A9F52930310558
:10B2800090F5822F81500E94967630C0C9010197B7
:10B290000E9480762BC0C90101970E94B77626C014
:10B2A000423038F060913404709135046830710593
:10B2B00010F06FEF70E06F3FB1F0433058F08091C5
:10B2C0005104882339F040914304509144044230A2
:10B2D000510510F04FEF50E04F3F29F0C9010197A1
:10B2E0000E94CD7603C0812F61E007C0892B19F041
:10B2F000812F67E002C0812F60E00E9458491F91B2
:10B300000895423008F0A4CFABCFFF920F931F9364
:10B31000CF93DF93082FFB01442311F18091330475
:10B320008823F1F080912504909126040097C1F0C4
:10B3300024E08130920708F459C012C08930910589
:10B3400078F481500E948B7607C001970E94767630
:10B3500003C001970E94AD76EC0197FF09C003C0BE
:10B36000802F61E002C0802F67E00E94584938C0FA
:10B370008DB79EB707970FB6F8949EBF0FBE8DBFCF
:10B38000EDB7FEB73196ADB7BEB711960C938AE70D
:10B3900097E092838183D483C383D683C5830E943D
:10B3A0003D20FC2E8DB79EB707960FB6F8949EBF32
:10B3B0000FBE8DBF802F65E20E94BD1F10E8C0E068
:10B3C000D0E0812F8F2111F460E301C061E3802F71
:10B3D0000E94BD1F16952196C830D10591F781E0D6
:10B3E000DF91CF911F910F91FF9008956381643495
:10B3F00009F4AFCF653424F4623409F0B1CFA9CF9A
:10B40000603509F4A2CF623509F0AACF97CF1F9318
:10B41000182F442319F5813031F481E067EE77E08D
:10B420000E9497201DC00E94991400D000D00F9256
:10B43000EDB7FEB73196ADB7BEB711961C9324EEAB
:10B4400037E032832183948383830E943D2081E00F
:10B450000F900F900F900F900F900FC0813011F44C
:10B4600081E00BC061EE77E00E9497208091250477
:10B47000909126040E942D1480E01F910895EF9270
:10B48000FF920F931F93CF93DF93F82E442371F015
:10B4900080913304882351F02091250430912604B3
:10B4A0002115310529F02533310510F020E030E079
:10B4B000122F222309F44FC000D000D00F92EDB715
:10B4C000FEB73196ADB7BEB71196FC9283EF97E009
:10B4D00092838183238314820E943D20E12EEA948B
:10B4E0000F900F900F900F900F908E2D60E00E94A4
:10B4F000AF79EC0100E011E0812F90E08C239D23D7
:10B50000892B19F08F2D61E302C08F2D60E30E941B
:10B51000BD1F0F5F083011F0110FEECF8F2D60E2CD
:10B520000E94BD1F8E2D61E00E94AF79EC0100E00A
:10B5300011E0812F90E08C239D23892B19F08F2D12
:10B5400061E302C08F2D60E30E94BD1F0F5F0830D2
:10B5500011F0110FEECF81E0DF91CF911F910F918C
:10B56000FF90EF9008950F931F93082FFB01118117
:10B570001150143310F082E014C060E00E94BD1F2F
:10B58000812F60E00E94AF79682F802F0E94BD1F3D
:10B59000812F61E00E94AF79682F802F0E94BD1F2C
:10B5A0008FEF1F910F9108951F93182F4423A9F037
:10B5B0008091640C282F30E021703070809133042A
:10B5C000882341F0809125049091260482309105D2
:10B5D00008F49C01822F0E94BA7900D000D00F920B
:10B5E000EDB7FEB73196ADB7BEB711961C9386E1A5
:10B5F00098E0928381838091640C90E081709070D8
:10B60000948383830E943D200F900F900F900F90A2
:10B610000F9081E01F910895CF92DF92EF92FF92F9
:10B620000F931F93CF93DF93D82E8B0121E0281720
:10B6300008F45AC0FB01828190E087709070D82F87
:10B64000CC27818190E0C82BD92B2197F7E0C83F08
:10B65000DF0710F082E049C00E942E12982F82501E
:10B66000823020F0973011F086E03FC07E01EE0C72
:10B67000FF1CF801628167FD04C081E090E0E82AC8
:10B68000F92A88E4D89EE0011124CB56DC4F862F9E
:10B6900090E0B6E096958795BA95E1F7CC24C394EF
:10B6A000C8228E010B5B1F4FF80180819181FFEF53
:10B6B0008F3F9F0749F060E04D2D0E9486868FEFF7
:10B6C0009FEFF80191838083C7016C2D4D2D0E945F
:10B6D0008686882311F489E008C0CC2029F0FE0179
:10B6E000EB5BFF4FF182E08280E0DF91CF911F9111
:10B6F0000F91FF90EF90DF90CF9008950F931F93DD
:10B70000CF93DF93082FFB01828190E087709070C8
:10B71000D82FCC27818190E0C82BD92B219787E0A7
:10B72000C83FD80710F082E01BC0CE010E94D6832C
:10B73000873621F0873411F010E001C014E0CE010B
:10B74000880F991F0E940484039709F41160802FC9
:10B7500060E00E94BD1F802F612F0E94BD1F8FEFF0
:10B76000DF91CF911F910F910895AF92BF92DF9219
:10B77000EF92FF920F931F93CF93DF93D82E142F46
:10B780000E942E12882319F48D2D66E061C08D2D44
:10B7900060E0412F28EF37E00E94724B5C01009778
:10B7A00009F49CC021E02D1508F498C0123008F46B
:10B7B00059C088E4D89E7001112485E993E0E80E11
:10B7C000F91EE701CB5BDF4F88819981AFEF8F3F97
:10B7D0009A0741F060E04D2D0E9486868FEF9FEF23
:10B7E0009983888380913604873411F490E012C0E5
:10B7F000823511F491E00EC080914204882339F023
:10B8000080913404909135048230910510F082E0EB
:10B8100090E0982F123059F080915104882339F02C
:10B8200000914304109144040230110510F000E02F
:10B8300010E0E5012197CC0FDD1FC90FD11DCE010E
:10B84000602F4D2D0E948686882329F48D2D69E076
:10B850000E94094B44C0002329F0F701EB5BFF4F26
:10B86000D183C083C50101970E94D683082F112779
:10B8700007FD1095C8010E9498A07C01C8010E9494
:10B8800080A02DB73EB7295030400FB6F8943EBF88
:10B890000FBE2DBFEDB7FEB73196ADB7BEB711964F
:10B8A000DC922AE738E032832183B482A382F682D5
:10B8B000E58220E030E0892B11F021E030E0308794
:10B8C00027830E943D2081E02DB73EB7275F3F4F81
:10B8D0000FB6F8943EBF0FBE2DBF01C081E0DF91CF
:10B8E000CF911F910F91FF90EF90DF90BF90AF909D
:10B8F0000895EF92FF920F931F93CF93DF93182F2A
:10B90000042F60E02FEF3FE30E94724BEC010097A1
:10B9100009F45BC00E9469377C01009771F4023022
:10B9200018F4812F6AE011C0CE010E94643B7C01B3
:10B93000009729F4812F6BE008C00230F0F00E94DC
:10B94000AE21882329F0812F68E00E94094B3EC078
:10B95000D70114966D917C911597802F40E052E0AD
:10B9600021E008E00E94F648BC01CE01412F0E9470
:10B97000CC3BCE0160E00E949B370E942E128823B0
:10B9800021F4812F62E40E94094B00D000D00F9275
:10B99000EDB7FEB73196ADB7BEB711961C9385E8EB
:10B9A00098E092838183D483C3830E943D200F90CB
:10B9B0000F900F900F900F90F70164817581812F88
:10B9C00040E052E028E00E94B14B81E0DF91CF914E
:10B9D0001F910F91FF90EF900895EF92FF920F93B8
:10B9E0001F93CF93DF93182F042F60E02FEF3FE3D7
:10B9F0000E94724BEC01009709F45BC00E9469370A
:10BA00007C01009771F4023018F4812F6AE011C0B4
:10BA1000CE010E94643B7C01009729F4812F6BE0EA
:10BA200008C00230F0F00E94AE21882329F0812F57
:10BA300068E00E94094B3EC0D70114966D917C913D
:10BA40001597802F42E050E021E008E00E94F64880
:10BA5000BC01CE01412F0E94CC3BCE0160E00E9490
:10BA60009B370E942E12882321F4812F62E40E94CA
:10BA7000094B00D000D00F92EDB7FEB73196ADB7AD
:10BA8000BEB711961C938BE898E092838183D48390
:10BA9000C3830E943D200F900F900F900F900F9046
:10BAA000F70164817581812F42E050E028E00E9417
:10BAB000B14B81E0DF91CF911F910F91FF90EF90FB
:10BAC0000895DF92EF92FF920F931F93CF93DF932E
:10BAD000D82E142F60E02FEF3FE30E94724B7C01C1
:10BAE000009709F4E8C00E946937EC01009771F4EF
:10BAF000123018F48D2D6AE012C0C7010E94643B19
:10BB0000EC01009731F48D2D6BE009C0123008F480
:10BB100081C00E94AE21882329F08D2D68E00E940B
:10BB2000094BCAC08C819D81AE81BF81BC016E7FF3
:10BB3000AC0141705070123059F08091510488234B
:10BB400039F020914304309144042230310508F04B
:10BB50009A01232B09F06160812F42E050E024E03C
:10BB600004E00E94F648BC01C7014D2D0E94CC3B69
:10BB7000888569850E947B55482F809142048823DF
:10BB800039F020913404309135042038310508F023
:10BB9000242F80915404863411F411E01AC08235A8
:10BBA00011F410E016C040E050E0888587FF02C025
:10BBB00041E050E0143058F080916004882339F05F
:10BBC00080915204909153048230910508F0CA018B
:10BBD000182F213029F4C7010E94683500E005C004
:10BBE000822F69850E945455082F111100686885BD
:10BBF000802F862787FF05C06078C7014D2D0E94E2
:10BC0000053CC701602F4D2D0E94053CC70160E037
:10BC10000E949B370E942E12823019F48D2D61E410
:10BC200006C00E942E12833021F08D2D62E40E9406
:10BC3000094B888569850E947B55682F8C8180FD22
:10BC400003C040E350E002C041E350E0888587FD37
:10BC500003C022E730E002C026E630E08DB79EB791
:10BC60000B970FB6F8949EBF0FBE8DBFEDB7FEB712
:10BC70003196ADB7BEB71196DC9288EB98E092830F
:10BC80008183F482E38265831682508747833287FB
:10BC900021870E943D208DB79EB70B960FB6F89472
:10BCA0009EBF0FBE8DBF6C817D818D2D42E050E027
:10BCB00024E00E94B14B81E0DF91CF911F910F9161
:10BCC000FF90EF90DF900895AF92BF92CF92DF92F6
:10BCD000EF92FF920F931F93CF93DF93C82E882389
:10BCE00049F0A4E9AA2EABE0BA2EFBE6EF2EFCE069
:10BCF000FF2E08C0ECEFAE2EEBE0BE2E75E6E72E71
:10BD00007CE0F72EDD2433C0F8940D2D10E0C70140
:10BD1000B8010E943789882341F1F801EE0FFF1F17
:10BD2000D501AE0FBF1FEF58F34FCD91DC911197A6
:10BD300080819181C82BD92B1D921C928081918189
:10BD4000C817D90721F4C701B8010E942189789446
:10BD50006D2D6F5F8C2D0E94BD1F8C2D6D2F0E944D
:10BD6000BD1F8C2D6C2F0E94BD1F7894D3940E9410
:10BD70000567FC018085D81638F28C2D60E00E94A2
:10BD8000BD1F8FEFDF91CF911F910F91FF90EF902B
:10BD9000DF90CF90BF90AF900895CF92DF92EF9257
:10BDA000FF920F931F93DF93CF93CDB7DEB7C254AB
:10BDB000D0400FB6F894DEBF0FBECDBFC82EDD2435
:10BDC0007E010894E11CF11C8C2D0E94EF878C01F0
:10BDD0008FEF0F3F180719F1C8010E94D683282F53
:10BDE000C8010196F7018083892F877081832734EA
:10BDF00011F0273629F48068F7018183273411F088
:10BE0000223521F4F701818180648183D394F0E2AB
:10BE1000DF1629F082E090E0E80EF91ED5CF8C2DD8
:10BE20006D2D0E94BD1FED2CFF24EE0CFF1C8E011A
:10BE30000F5F1F4FD02E06C0F80161918F018C2D2E
:10BE40000E94BD1F802F8D1990E08E159F05A4F3D1
:10BE50008FEFCE5BDF4F0FB6F894DEBF0FBECDBFC6
:10BE6000CF91DF911F910F91FF90EF90DF90CF90D6
:10BE700008951F93CF93DF93182F0E949788692FFF
:10BE8000629566956695617095FD646080FD686059
:10BE900097FD6062EC01CE7FDF71209709F060684A
:10BEA000812F0E94BD1F2097A1F0CE019695879506
:10BEB000682F6170C2FD6064C97F209709F06068D7
:10BEC000812F0E94BD1FCD2B21F0812F60E00E94A9
:10BED000BD1F8FEFDF91CF911F910895CF92DF9219
:10BEE000FF920F931F93DF93CF93CDB7DEB7609789
:10BEF0000FB6F894DEBF0FBECDBFF82E64E00E94EF
:10BF0000BD1F8F2D62E00E94BD1F8F2D60E00E943B
:10BF1000BD1F8F2D60E00E94BD1F8F2D60E20E942B
:10BF2000BD1F8F2D64E00E94BD1F0E9419672DB7B1
:10BF30003EB7285030400FB6F8943EBF0FBE2DBF1D
:10BF4000EDB7FEB731968E010F5F1F4FADB7BEB78D
:10BF500012961C930E9311972BEF39E033832283B3
:10BF600064837583868397830E94F9A0EDB7FEB73B
:10BF700038960FB6F894FEBF0FBEEDBF39E0C32E62
:10BF8000D12CCC0EDD1ED8016C916295607F11968C
:10BF90008C918053682B0E5F1F4F8F2D0E94BD1F09
:10BFA0000C151D0581F780E060960FB6F894DEBF92
:10BFB0000FBECDBFCF91DF911F910F91FF90DF900A
:10BFC000CF9008950E94C47980E008950F931F9345
:10BFD000CF93DF938B01823030F5FB01828190E0BB
:10BFE00087709070D82FCC27818190E0C82BD92BF7
:10BFF0002197F7E0C83FDF0710F082E015C00E94EC
:10C000002E12982F8250823020F0973011F086E067
:10C010000BC0F8016281669566956695CE01880F22
:10C02000991F0E94AC3380E0DF91CF911F910F9157
:10C030000895CF93DF93EB0140E00E948D56FC0101
:10C04000009711F48FEF1CC081858370833011F04D
:10C0500082E016C04B816C8170E07695762F662762
:10C0600077956795842F90E08F779070682B792B68
:10C07000441F4427441F808191810E94BB3680E089
:10C08000DF91CF910895FF920F931F93CF93DF938A
:10C09000F82EEB0141E00E948D568C01009711F4BF
:10C0A0008FEF35C0FC0184819581A681B781A17095
:10C0B000B07E4B8150E060E070E031E1440F551FED
:10C0C000661F771F3A95D1F7482B592B6A2B7B2B8C
:10C0D0008C8190E0A0E0B0E08F709070A070B070A4
:10C0E00029E1880F991FAA1FBB1F2A95D1F7482B5A
:10C0F000592B6A2B7B2B808191812F2D0E94933BA2
:10C10000F8018081918161E00E949B3780E0DF919E
:10C11000CF911F910F91FF900895FF920F931F935E
:10C12000CF93DF93F82E8B0141E00E948D56EC01F6
:10C13000009711F48FEF21C08C819D81AE81BF816A
:10C140009170AE7FF801438150E060E070E0E9E07B
:10C15000440F551F661F771FEA95D1F7482B592BBF
:10C160006A2B7B2B888199812F2D0E94933B88819C
:10C17000998160E00E949B3780E0DF91CF911F9111
:10C180000F91FF900895FF920F931F93CF93DF932A
:10C19000F82E8B0141E00E948D56EC01009711F4BE
:10C1A0008FEF1EC08C819D81AE81BF8181709E7F8B
:10C1B000F801438150E060E070E0440F551F661FB6
:10C1C000771F482B592B6A2B7B2B888199812F2D28
:10C1D0000E94933B8881998160E00E949B3780E0B8
:10C1E000DF91CF911F910F91FF900895CF92DF9231
:10C1F000EF92FF920F931F93CF93DF93C82E8B0183
:10C20000F42E41E00E948D56EC01009711F48FEF5F
:10C2100078C00E94AE21882311F088E072C0D80156
:10C220001396DC90FF2071F0B1E0DB1631F48881C9
:10C2300099810E946835DD2405C08D2D69850E9495
:10C240005455D82EF8016481262F30E065FF02C0D6
:10C25000F0E8DF2AEC80FD800E811F818EEF9FEFDA
:10C26000AFEFBFEFE822F9220A231B2324FF08C007
:10C2700081E090E0A0E0B0E0E82AF92A0A2B1B2B2D
:10C2800067FF15C081EE9FEFAFEFBFEFE822F92205
:10C290000A231B232F703070220F331FC901AA27D6
:10C2A00097FDA095BA2FE82AF92A0A2B1B2B68853F
:10C2B0008D2D862787FF06C06078888199814C2D57
:10C2C0000E94053C888199816D2D4C2D0E94053C72
:10C2D00088819981B801A7012C2D0E94933B888108
:10C2E000998160E00E949B370E942E12833041F0BA
:10C2F000873031F0823011F082E403C081E401C064
:10C3000080E0DF91CF911F910F91FF90EF90DF9030
:10C31000CF90089540E00E94F660089541E00E94A9
:10C32000F66008951F93CF93DF93182FEB010E94BF
:10C330002E12833011F082E43EC0812FBE0141E015
:10C340000E948D56FC01009711F48FEF34C01186C6
:10C3500013821282148215821682178210866C81D3
:10C3600070E080E090E0982F872F762F66272D8150
:10C3700030E040E050E0A90133272227622B732BE5
:10C38000842B952B2B8130E040E050E0622B732B07
:10C39000842B952B2E8130E040E050E0522F442733
:10C3A00033272227622B732B842B952B40815181BD
:10C3B0000E94F33180E0DF91CF911F9108951F9388
:10C3C000CF93DF93182F41E00E948D56EC01009728
:10C3D00001F1812F60E00E94BD1F69856370812F8C
:10C3E0000E94BD1F89850E94E236892B19F0812F9A
:10C3F0006CE105C089850E94D63C682F812F0E9480
:10C40000BD1F812F6FEF0E94BD1F812F6FEF0E9414
:10C41000BD1F8FEFDF91CF911F910895CF92DF92D3
:10C42000EF92FF920F931F93CF93DF93D82EEB01E0
:10C43000C42E21E0281708F4F9C028817FE1F72EE7
:10C44000F222422F50E0CA01807E90708034910524
:10C4500009F49AC08134910534F4009789F08097EB
:10C4600009F0E4C050C08038910509F4B5C0803CA3
:10C47000910509F4C7C08036910509F0D7C0A4C062
:10C4800081E08C1508F0D4C00981802F90E00E94D3
:10C49000643BFC01009709F4C9C064817581F4FE16
:10C4A00003C0EB01C16002C0EB01CE7F1F2D1F70E6
:10C4B000F0841F3021F46F2D6095607817C081855E
:10C4C000112389F00E94D63C8C3139F08E3739F037
:10C4D0008B3149F4110F115006C0110F04C089E0CF
:10C4E000189F102D11246F2D6078612B802F90E004
:10C4F0004D2D0E94053C802F90E0BE014D2D0E94E5
:10C50000CC3B802F5CC088E4D89E70011124E5E903
:10C51000F3E0EE0EFF1E237F288387010B5B1F4F86
:10C52000F80180819181FFEF8F3F9F0749F060E024
:10C530004D2D0E9486868FEF9FEFF80191838083B7
:10C540002881203209F472C0233209F46FC0F1E06F
:10C55000FC1508F06DC06981213231F4C62FD0E09E
:10C560002197CC0FDD1F05C0C62FD0E0CC0FDD1FFB
:10C570002197CE0161E04D2D0E948686F701EB5B8D
:10C58000FF4FD183C08352C021E02C1508F050C06A
:10C590001981812F90E00E94EB3B9B01AC01217E31
:10C5A0008F2D90E08F709070880F991F282B392B5A
:10C5B000812F90E0B9014D2D0E94CC3B812F90E05E
:10C5C00060E00E949B3732C020FF02C080E001C0C3
:10C5D00083E00E9449122AC0FF2011F480E015C0B8
:10C5E00000E0802F6D2D0E949679182F8D2D692FD8
:10C5F0000E94BD1F8D2D612F0E94BD1F0F5F0F1563
:10C6000080F314C0FF2021F481E00E94BA790EC0AB
:10C610008F2D81506D2D0E949679182F8D2D692FA9
:10C620000E94BD1F8D2D612F0E94BD1F81E001C0A2
:10C6300080E0DF91CF911F910F91FF90EF90DF90FD
:10C64000CF900895BF92CF92DF92EF92FF920F9317
:10C650001F93CF93DF93B82E81E08B1508F419C395
:10C6600088E4B89E70011124E5E9F3E0EE0EFF1EA8
:10C67000E701C95BDF4F888187FD0BC38B2D0E94CB
:10C68000A91F8C01FFEF8F3F9F0709F402C3888128
:10C6900080688883E4E4CE2ED12CCE0CDF1CF6011A
:10C6A00080818823F1F0F70160817181828193811B
:10C6B00068537F4F8F4F9F4F0E94D018882389F077
:10C6C000F6018081882349F0888180FD0AC0F70146
:10C6D0008481883531F0883721F0F701EC5BFF4F1A
:10C6E00010828091370790913807A0913907B09157
:10C6F0003A07F70180839183A283B383EC5BFF4FFA
:10C700008081803408F01082C7010E94D2488823BB
:10C71000B1F00830110551F4F701EC5BFF4F808157
:10C72000882309F4A8C281508083A5C20115110590
:10C7300009F4A1C20D30110511F400E010E0F70179
:10C74000EC5BFF4F8081D701A80FB11D14960C93AD
:10C75000D82ED394D082DD2091F0F701E95BFF4F12
:10C76000808190E0EC01C170D07080FD8BC2F70138
:10C770008481883509F486C2883709F483C2B701F9
:10C780006C5F7F4F8B2D4D2D0E940E62882309F028
:10C790006EC271C2012B09F06EC2F701EC5BFF4F54
:10C7A000108287010C5F1F4FF701E95BFF4F80810B
:10C7B00080FD03C087010B5F1F4FF8018081882334
:10C7C00009F425C2C80161E175E043E050E00E9430
:10C7D000B2A0892B59F4C6E3D9E4C80103960E949C
:10C7E000E7A0C8010E94ED49D82E0AC2C8010E94E4
:10C7F000E7A0C8010E94ED49D82EC8016FE075E09E
:10C800000E94A0A0892B39F0C8016DE075E00E945C
:10C81000A0A0892B19F4CEEAD9E4F2C1C8016AE0DC
:10C8200075E00E94A0A0892B19F4C8EAD9E4E8C1F8
:10C83000C80167E075E00E94A0A0892B19F4C2EA44
:10C84000D9E4DEC1C80164E075E00E94A0A0892B94
:10C8500019F4CCE9D9E4D4C1C80162E075E00E94C2
:10C86000A0A0892B39F0C8016DEF74E00E94A0A050
:10C87000892B19F4CAE7DDE4C3C1C8016BEF74E08A
:10C880000E94A0A0892B39F0C80168EF74E00E94D3
:10C89000A0A0892B19F4C6E6DDE4B2C1C80163EF9C
:10C8A00074E00E94A0A0892B19F4C4E1DDE4A8C1C2
:10C8B000C80161EF74E00E94A0A0892B19F4C1E6C1
:10C8C000DDE59EC1C8016EEE74E00E94A0A0892B38
:10C8D00019F4C4E5D6E594C1C8016CEE74E00E9479
:10C8E000A0A0892B19F4CDEEDCE58AC1C80169EE60
:10C8F00074E00E94A0A0892B19F4C9E7DCE580C18F
:10C90000C80167EE74E00E94A0A0892B19F4C5EB62
:10C91000DBE576C1C80165EE74E00E94A0A0892B1A
:10C9200019F4C6E3DDE46CC1C80163EE74E00E9453
:10C93000A0A0892B19F4CFE3D2E562C1C80160EE53
:10C9400074E00E94A0A0892B19F4C7EBD0E558C170
:10C95000C8016DED74E00E94A0A0892B19F4C4ED0C
:10C96000DAE54EC1C8016AED74E00E94A0A0892BEF
:10C9700019F4CFE3DAE544C1C80167ED74E00E9421
:10C98000A0A0892B19F4CCE6D0E53AC1C80164ED2A
:10C9900074E00E94A0A0892B19F4CCE4D7E630C142
:10C9A000C80162ED74E00E94A0A0892B19F4C7E0D1
:10C9B000DAE526C1C8016FEC74E00E94A0A0892BC3
:10C9C00019F4C8EEDFE41CC1C8016CEC74E00E94ED
:10C9D000A0A0892B19F4C6ECDCE412C1C80169ECF3
:10C9E00074E00E94A0A0892B19F4CDE7DCE408C113
:10C9F000C80166EC74E00E94A0A0892B39F0C80140
:10CA000063EC74E00E94A0A0892B19F4C0E3DEE47B
:10CA1000F7C0C8016EEB74E00E94A0A0892B51F111
:10CA2000C80169EB74E00E94A0A0892B69F1C801DC
:10CA300064EB74E00E94A0A0892BE1F0C8016FEACA
:10CA400074E00E94A0A0892BF9F0C8016AEA74E0A2
:10CA50000E94A0A0892B71F0C80165EA74E00E94D1
:10CA6000A0A0892B89F0C80160EA74E00E94A0A010
:10CA7000892B19F4C5E8D9E5C3C0C8016BE974E096
:10CA80000E94A0A0892B19F4CAE0D9E5B9C0C80159
:10CA900066E974E00E94A0A0892B19F4CFEBD8E5D9
:10CAA000AFC0C80161E974E00E94A0A0892B19F40D
:10CAB000C0E8D8E5A5C0C8016EE874E00E94A0A057
:10CAC000892B19F4CCE3D8E59BC0C80166E874E073
:10CAD0000E94A0A0892B19F4C8E4D5E591C0C80133
:10CAE0006FE774E00E94A0A0892B19F4C4EED7E58B
:10CAF00087C0C80166E774E00E94A0A0892B19F4E2
:10CB0000C7E4D6E57DC0C8016EE674E00E94A0A02F
:10CB1000892B19F4C5E0D3E573C0C80167E674E05A
:10CB20000E94A0A0892B19F4C4EFD5E569C0C80103
:10CB30006EE574E00E94A0A0892B19F4C0EFD5E542
:10CB40005FC0C80166E574E00E94A0A0892B19F4BB
:10CB5000C6EFD3E555C0C8016FE474E00E94A0A001
:10CB6000892B19F4C1EFD1E54BC0C80168E474E02A
:10CB70000E94A0A0892B19F4CFE5D1E541C0C801DE
:10CB800064E474E00E94A0A0892B19F4CEE3DFE4F2
:10CB900037C0C80161E474E00E94A0A0892B19F499
:10CBA000CDE0DFE42DC0C8016DE374E00E94A0A0D9
:10CBB000892B19F4C3EADDE423C0C80164E374E0FF
:10CBC0000E94A0A0892B19F4CFE2DDE419C0C801AE
:10CBD00060E374E00E94A0A0892B19F4CCE1DCE4AE
:10CBE0000FC0C8016BE274E00E94A0A0892B19F469
:10CBF000CCEFDBE405C08B2D61E00E94094B05C042
:10CC00008B2DB8014D2DFE0109958823A1F18B2DA7
:10CC100068E274E00E9497202EC0CD2B31F0B7015E
:10CC20006C5F7F4FF701948106C0B7016B5F7F4F48
:10CC3000DA94F7019581E4E0F1E012C0891779F404
:10CC40008181D816C0F00280F381E02D309779F011
:10CC50008B2D0995682F8F3F51F08B2D06C0349690
:10CC60008081882359F78B2D61E00E94BD1FF70159
:10CC7000EC5BFF4F1082F701E95BFF4F80818F77FC
:10CC8000808307C0C7010E94D248882309F082CD63
:10CC9000C4CFDF91CF911F910F91FF90EF90DF9064
:10CCA000CF90BF9008956F5F7F4F42E00E940E6269
:10CCB0008FEF08956F5F7F4F41E00E940E628FEF0C
:10CCC00008958230C0F4282F30E088E490E0289F57
:10CCD000F001299FF00D389FF00D1124EB56FC4F09
:10CCE000EC5BFF4F1082339610828FEF9FEF929391
:10CCF00082930E94458808951F93182F823118F05F
:10CD000021E83EE032C00E940567FC012581243005
:10CD100039F0253079F0812F90E02130F1F414C002
:10CD2000212F30E054E0220F331F5A95E1F72F5F97
:10CD3000354F1BC0212F30E044E0220F331F4A95AE
:10CD4000E1F72F5D344F11C09C0194E0220F331F97
:10CD50009A95E1F72F5B334F08C09C0184E0220FC6
:10CD6000331F8A95E1F72F59324FC9011F9108955A
:10CD7000882319F026ED3EE016C00E940567FC01ED
:10CD80008581843029F0853031F0813051F406C03E
:10CD900022E93EE008C023EA3EE005C024EB3EE085
:10CDA00002C025EC3EE0C90108951F93182F83327D
:10CDB00018F022E338E126C00E940567FC01858156
:10CDC000843029F0853051F08130B1F40EC081E11A
:10CDD000189F900111242A51314F14C081E1189FEE
:10CDE00090011124275C3E4E0DC081E1189F9001F7
:10CDF000112424573C4E06C081E1189F9001112454
:10CE000021523A4EC9011F9108958BEB94E0089589
:10CE10008091BC0490E008958091CA0408958091A7
:10CE2000BB0408959091BB04982309F091E0892FE9
:10CE300008952CEF3FEF41E050E04BBFF9012791FF
:10CE40003791479156915070B901CA0108958FEFFB
:10CE50009FEFA1E0B0E0ABBFFC018791823029F4E5
:10CE6000079902C080E8089582E00895EBEDF4E0B0
:10CE700080819181892B29F08381882311F411828B
:10CE800010828381882311F081508383349684E05B
:10CE9000EB3EF80769F708950E948E31F89488E117
:10CEA00081BD8BE081BDFFCF0E946937DC01009717
:10CEB000C1F0EBEDF4E0208131818D919C911197CF
:10CEC0002817390739F012968D919C9113972817DE
:10CED000390711F411821082349684E0EB3EF80792
:10CEE00051F708957F928F929F92AF92BF92CF9207
:10CEF000DF92EF92FF920F931F93DF93CF9300D0B7
:10CF000000D000D0CDB7DEB7782E5B01042FFE0134
:10CF1000319686E0DF011D928A95E9F7CF010E94E4
:10CF2000606AEBEDF4E014E088249924143029F4CD
:10CF300080819181892B09F4182D808191818A1536
:10CF40009B0509F0E5C0F401EE0FFF1FEE0FFF1F78
:10CF5000E552FB4F88E08383F401EE0FFF1FEE0FD5
:10CF6000FF1FE352FB4F80818F5F8083833008F483
:10CF700003C1C5010E94643B6C01009709F4FCC029
:10CF8000BFEF7B16B1F5FC0144815581002319F0F8
:10CF9000C501BA0129C0C501D60118966C910E943D
:10CFA0006A43F6011185C5010E94B97CBC01812F3D
:10CFB0000E944943D60114962D913D914D915C916B
:10CFC00017979A0144275527C501B9010E949F3D33
:10CFD000F60182819381009749F00E94643BFC0135
:10CFE00064817581808191810E948C3D0E94FE3C0C
:10CFF00082C0DC0114962D913D914D915C91179763
:10D00000002369F07E010894E11CF11CC70160E077
:10D0100000E00E94856A872D68E0A7016AC000E0F1
:10D02000FC0182819381892B09F001E07E01089443
:10D03000E11CF11CC701D60118966C910E94856A0B
:10D04000872D67E0A7010E94166BF60181858F7717
:10D050008B8382819381892B41F4C5010E94B97C25
:10D06000BC01CE0104960E94606A0E94C26B8823B4
:10D07000E1F3872D69E08E010F5F1F4FA8010E9429
:10D08000166BD60114964D915D916D917C91179719
:10D09000C8010E946C6A0E94C26B8823E1F3872D4D
:10D0A0006DE05E010894A11CB11CA5010E94166BE5
:10D0B000F601828193810E9469378C010097D9F033
:10D0C000DC016D917C91C5010E94606AF8012481A8
:10D0D000358146815781C50160E000E00E94856A84
:10D0E0000E94C26B8823E1F3872D68E0AE014F5F99
:10D0F0005F4F0E94166B880C991C880C991C8BED55
:10D1000094E0880E991ED4011D921C9281E035C0D6
:10D110000894811C911C3496B4E08B16910409F09C
:10D1200005CF143041F48FEF66E0AE014F5F5F4FE3
:10D130000E94166B21C00E94F03C8A159B0519F4D1
:10D140000E94613F07C08FEF65E0AE014F5F5F4F08
:10D150000E94166BE12FF0E0EE0FFF1FEE0FFF1F96
:10D16000DF01A552BB4F1196BC92AE92E352FB4F2A
:10D17000108288E013968C9380E026960FB6F89480
:10D18000DEBF0FBECDBFCF91DF911F910F91FF90FA
:10D19000EF90DF90CF90BF90AF909F908F907F9057
:10D1A00008957F928F929F92AF92BF92CF92DF921B
:10D1B000EF92FF920F931F93DF93CF9300D000D095
:10D1C00000D0CDB7DEB7782E4B017A01CB010E949B
:10D1D000643B5C01009709F452C0C7010E94643BA4
:10D1E0006C01009709F44BC0D50119968C910E94EF
:10D1F000D63C8C01F60181850E94D63C9801281B03
:10D20000390BC90137FF03C0909581959F4F029755
:10D21000B4F03FEF731621F481E00E94873D2FC0E8
:10D22000FE01319686E0DF011D928A95E9F781E0E3
:10D230008983872D61E2AF010E94166B20C000E058
:10D24000872DB70141E00E947267882389F0F601BB
:10D250008085D50118969C91892787FF04C0E0E05E
:10D26000F0E8EE2AFF2AC401B7010E942B3B07C059
:10D270000E94C26B8823E1F30F5F043109F7269601
:10D280000FB6F894DEBF0FBECDBFCF91DF911F91D7
:10D290000F91FF90EF90DF90CF90BF90AF909F9055
:10D2A0008F907F9008951F93CF93DF93EB016115CB
:10D2B000710599F08F3F71F410E08FEFBE0140E0EF
:10D2C0000E9472670E94C26B8823E1F31F5F1A30CD
:10D2D000A1F703C040E00E947267DF91CF911F91D8
:10D2E0000895CF93DF93C0E0D0E0CE010E9492A3D7
:10D2F000FE01E554FB4F6081861719F0CE010E94B4
:10D30000A4A3A8952196C032D10579F7DF91CF91DA
:10D310000895982F90952091BB0492239093BB047D
:10D3200082FF02C00E940C300E94716908959091A2
:10D33000BB04982B9093BB0482FF02C00E940C3068
:10D340000E94716908951F93182F82FD136011FDCB
:10D3500011601093CA040E947169812F0E94F62205
:10D360001F9108951F93182F883008F017E08091BF
:10D37000BC04181751F01093BC040E947169812FEE
:10D3800068E04EE421E00E9496131F910895809377
:10D39000C0040E94716908959091C004973008F00C
:10D3A00091E080E1EBEBF4E0DF011D928A95E9F773
:10D3B00088E18093BF049093C00497E09093BC04ED
:10D3C00084E18093C10482E08093C60482E3809369
:10D3D000C7048CE08093BB049093CA0483E090E080
:10D3E0000E9485840E94716908950E948E3184E0B4
:10D3F0006EEB71E00E94A41F85E066EC71E00E9474
:10D40000A41F81E794E968EC70E00E94021E80E0AE
:10D4100060E00E94C31E83E00E94D566BC0182E0EA
:10D420000E9497200E94063A0E947E7B0E94CC694F
:10D430000E944C6708958BEB94E060E070E040E25E
:10D4400050E00E9482A38091BD049091BE048F5F42
:10D450009F4F11F40E94CC698091BC04883018F071
:10D4600087E08093BC048091C8049091C904885FD0
:10D47000974020F01092C9041092C8048091C00413
:10D48000873010F01092C0048AEF9FEFA1E0B0E067
:10D49000ABBFFC019791892F81508E3F10F4909380
:10D4A0006F000895682780E097E067FF03C0660F6C
:10D4B000692701C0660F8F5F8830B9F7862F0895FE
:10D4C000FC01862F8F778083660F672F661F770B8F
:10D4D00071956F7761830895FC01CB01AA27BB2763
:10D4E0008F77828327E176956795579547952A959B
:10D4F000D1F7842F8F77838397E07695679557953B
:10D5000047959A95D1F7448308950F93FC01862F90
:10D510008F778283DA01C9017AE0B695A79597954E
:10D5200087957A95D1F78F7366956074862B838380
:10D53000DA01C90163E0B695A795979587956A9535
:10D54000D1F78F778483822F82958077858340FF00
:10D5500002C088608583002319F0858181608583FE
:10D560000F910895CF92DF92EF92FF921F93CF9386
:10D57000DF93782F162F7A01A895209110058091BE
:10D58000110530E090E001972817390709F445C0EC
:10D5900080911005833021F4809111058823E9F1F1
:10D5A0009091100589E0989FE0011124C451DB4F50
:10D5B000672F6068688380E00E94526A1983612F38
:10D5C0000E94526A982FE2E0CE2ED12CCC0EDD1EA6
:10D5D000E60110E0E114F10431F0F70181917F01DF
:10D5E0008F77888301C01882892F69910E94526ABF
:10D5F000982F1F5F163071F787FD9095F60196837F
:10D60000809110058F5F8093100580911005843004
:10D6100010F01092100581E001C080E0DF91CF9101
:10D620001F91FF90EF90DF90CF9008950F931F937D
:10D63000CF93DF93082F162FEA0102C00E94351204
:10D64000802F612FAE010E94B26A8823B9F3DF9167
:10D65000CF911F910F910895DF93CF9300D000D009
:10D6600000D0CDB7DEB7FE01319696E0DF011D9206
:10D670009A95E9F74983AF010E94166B26960FB67B
:10D68000F894DEBF0FBECDBFCF91DF9108950F9309
:10D690001F93CF93DF93EC01162F009709F46CC012
:10D6A00086E0DE011D928A95E9F70E9405672091C8
:10D6B00013053091140504E0220F331F0A95E1F79A
:10D6C000FC01858596858217930720F41092140536
:10D6D000109213051F77DE011D93E0911305F09161
:10D6E00014058E2F8F7789839D012F5F3F4FCF01C8
:10D6F000880F892F881F990B91958F7711968C939E
:10D70000A9014F5F5F4FEE0FFF1FDF01A752B34F1D
:10D710008C918F77E9018983EA012196E652F34FD4
:10D720008081880F8E779C91991F9927991F892B4B
:10D73000DA0111968C938E010F5F1F4F80818295C5
:10D74000869586958370898382E00E94126788237C
:10D7500029F089818460898381E001C080E00E9492
:10D760009E89E801219680911305909114050196F8
:10D770009093140580931305CE01DF91CF911F91F3
:10D780000F9108952F923F924F925F926F927F92E6
:10D790008F929F92AF92BF92CF92DF92EF92FF92C1
:10D7A0000F931F93DF93CF93CDB7DEB7EB970FB6F1
:10D7B000F894DEBF0FBECDBFA2E06A2E712C6C0EB6
:10D7C0007D1EF8E04F2E512C4C0E5D1E8824839454
:10D7D0009E01295E3F4F3FAB2EABC30102969DAB2E
:10D7E0008CABDE019996B9AFA8AFFE01BD96FBAF39
:10D7F000EAAFFDC587FF05C010921B05FFEFF09350
:10D800001D0520911B05293040F4E22FF0E0E45E75
:10D81000FA4F80832F5F20931B0580911B05893071
:10D8200009F0E5C580911C0587FFE1C50CE115E015
:10D8300090E0D8016D918D01892F0E94526A982F36
:10D84000B5E004321B07A9F787FD90958091240568
:10D85000981709F0C7C538C7EFE79E2E9822209188
:10D860001F05C22EDD24D694DC2CCC24D794C7947B
:10D87000B0901E058B2D90E0C82AD92AF30136E01E
:10D8800011923A95E9F790911D05933109F477C209
:10D89000943158F59930B0F4973008F0A8C093301F
:10D8A00009F457C0943038F4913009F4ADC1923086
:10D8B00009F098C5B5C2953009F4C4C2963008F095
:10D8C0007DC0ABC19E3009F4B6C09F3038F49B30A8
:10D8D00009F420C19D3009F085C56EC1903109F46D
:10D8E000B1C1903108F47EC533C29B3109F4AEC298
:10D8F0009C3170F4973159F1983118F4963118F140
:10D9000024C0993109F43FC29A3108F04EC2D4C103
:10D91000913409F431C5923450F4943209F4B9C207
:10D92000903409F437C5903209F05CC563C1933473
:10D9300009F4E2C4933408F408C5903709F052C5DD
:10D940000EE115E03EC510E0BBC180E0B7C180E04C
:10D95000B4C1C114D10409F43CC5109120058091D3
:10D960002105282F30E086FD1068322F2227330F43
:10D97000330F6091220570E06F77707053E0660F8F
:10D98000771F5A95E1F78091230590E0807790709A
:10D9900044E0959587954A95E1F7682B792B622BA2
:10D9A000732BC60144E00E94CC3BC601612F44E0CA
:10D9B0000E94053CC6010E9454670BC5809120055A
:10D9C0008295880F880F807C8FA71EA64EA55FA525
:10D9D0004C295D2980912105882319F0CA0161E055
:10D9E00002C0CA0160E044E00E948686F2C48091D1
:10D9F0002105E82FF0E0609123056F7740E0983033
:10DA000009F441E09F01277030703695322F2227AC
:10DA1000379527958091200590E0282B392BE074CD
:10DA2000F070EE0FFF1F009122050E2BC601EE24B1
:10DA30000E943537CEC4C6010E9469377C01009729
:10DA400099F48BE0AEA9BFA91D928A95E9F7D88E0B
:10DA5000CF8A80E88F8FCE0147960E945B3AB7E16C
:10DA6000EB2EF12CEC0EFD1EF701228133812115E6
:10DA70003105D9F0822F8F778A83220F232F221F1F
:10DA8000330B3195822F8F778B83828193810E9414
:10DA9000EB3B9B01AC01C30160E000E00E94856AA2
:10DAA000892D6FE0A3010E94166B8C2D8F778A83DE
:10DAB000CC0CCD2CCC1CDD08D1948C2D8F778B8396
:10DAC000D70119968C918C83892D69E0A3010E945E
:10DAD000166BF701248135814681578100E08281F0
:10DAE0009381892B09F001E0C301D70118966C914D
:10DAF0000E94856A892D6EE0A3010E94166BF701D2
:10DB00004481558166817781C3010E946C6A892DA9
:10DB10006DE094C02091200530E040E050E0E091BD
:10DB200023058091210590E09695982F8827979559
:10DB300087957C010027F7FC0095102F8091220526
:10DB4000382E3294330C330C60EC36222224C1017F
:10DB5000AA2797FDA095BA2FE82AF92A0A2B1B2B92
:10DB6000E22AF32A042B152B8E2F90E0A0E0B0E0E0
:10DB700087709070A070B07025E1880F991FAA1F60
:10DB8000BB1F2A95D1F7E82AF92A0A2B1B2BD801AB
:10DB9000C7010197A109B1098F5F9F4FAF4FB040F7
:10DBA00008F017C4E695E695E695C801B701A60109
:10DBB0002E2F0E9412810DC48091200590E060916B
:10DBC000210570E07695762F6627779567952091E9
:10DBD00022052295220F220F207C29AB18AA28A902
:10DBE00039A9622B732B682B792BC60144E00E9464
:10DBF000AA3BEFC30E942E12843009F4EAC380913D
:10DC00001E050E944912E5C3C114D10409F4E1C301
:10DC1000892DB6010E945369DCC3C60160912005BD
:10DC20000E94B53C80911E058A8380911F058B83DD
:10DC3000C6010E9491378C83892D69E0A3010E945F
:10DC4000166BC7C3C6016CA97DA9AE014E5D5F4FBF
:10DC50000E94DE7D282F2F772A83880F892F881F27
:10DC6000990B91958F778B838AA18D838BA18E835E
:10DC70001F82892D61E1A3010E94166BFE01B496FB
:10DC80008301D30181918D9388AD99ADE817F90790
:10DC9000C9F7892D62E1A3010E94166BFE01B996B6
:10DCA0008191D8018D938D012AAD3BADE217F30729
:10DCB000B9F7892D63E1C2CF83E08D5F182F1D5F17
:10DCC000943199F480912105682F70E07695762F34
:10DCD0006627779567958091200590E0682B792BD2
:10DCE0008091220589831AA223C0C601BE016F5FFD
:10DCF0007F4FAE014E5D5F4F0E94DE7DBC01A0E212
:10DD0000B5E00DC0E2E2F0E0EC0FFD1FE10FF11D08
:10DD10008D9180831F5F35E0A332B30711F01B3074
:10DD200088F3E2E2F0E0EC0FFD1FE10FF11D10823D
:10DD3000C60149819E012E5D3F4F0E94267E282FFD
:10DD40002F772A83880F892F881F990B919512C0EE
:10DD5000913121F4C6010E94777C03C0C6010E9464
:10DD6000477C9C018F778A83220F232F221F330B3E
:10DD70003195822F8F778B83892D60E15FCFC6012C
:10DD80000E94447C26C38C2D8F778A83C601880F1E
:10DD9000892F881F990B91958F778B83C6010E94DD
:10DDA000D6838C83892D69E149CF80912105082F85
:10DDB00010E01695102F00271795079580912205E2
:10DDC0008295880F880F807C8BAB1AAA8AA99BA9A1
:10DDD000082B192B8091200590E0082B192B760138
:10DDE00094E0EE0CFF1C9A95E1F781E0C82ED12C4F
:10DDF000B0E1AB2EB12CAE0CBF1C60E0C60180239D
:10DE00009123892B09F061E0C7010E94CC84CC0CDE
:10DE1000DD1C0894E11CF11CEA14FB0471F7D9C263
:10DE20004091210550E05695542F4427579547952A
:10DE30008091200590E0482B592B892DB6010E9436
:10DE4000D168C7C2C6010E94683BC3C24091230586
:10DE50006091210570E06F7770707695762F662758
:10DE600077956795842F90E08170907090E4899FFA
:10DE7000902D88271124682B792B8091200590E024
:10DE8000682B792B441F4427441FC6010E94BB36D0
:10DE9000A0C2D201E6E01D92EA95E9F70E9405676B
:10DEA0008C01F6E0BF1609F4A4C0FB15A8F022E02F
:10DEB000B21609F449C02B1538F0BB2041F131E00E
:10DEC000B31609F086C22CC084E0B81609F470C0FD
:10DED0008B1508F47AC04FC099E0B91609F4D2C086
:10DEE0009B1548F0A7E0BA1609F489C0B8E0BB1644
:10DEF00009F06FC2BBC0EBE0BE1609F40CC1BE1640
:10DF000008F467C2F4E1FB1508F463C211C1188676
:10DF10000E940F678F7089870E940C67877046C0C8
:10DF200080911F058F700E9497690E940C679091E5
:10DF30002005982B892F87700E94A36980911F0567
:10DF400086FFE5CF81E014C080911F058F700E948D
:10DF500089690E940C679091200590959823892FDC
:10DF600087700E94A36980911F0586FFD0CF80E053
:10DF70000E94BA79CCCF80911F05882369F08091E7
:10DF8000210587958827879590912005892BD801B1
:10DF900016968C930E947169B3E0B887F801868168
:10DFA0008F7789878681881F8827881F8A87A0C1E5
:10DFB00080911F05853318F4D80118968C93B4E02E
:10DFC000B887F8018085898793C180911F0564E037
:10DFD0000E9496799C01F5E0F8878F778987C901BF
:10DFE000880F892F881F990B91958F778A87832FA8
:10DFF0007AC180911F0564E00E94AF79EBCF8091D8
:10E000002005082F10E01695102F0027179507956B
:10E0100080911F0590E0082B192B2FE0003F12077D
:10E0200028F03FE30F3F130709F0D3C160912105AA
:10E03000633011F0613069F48FE30F3F180729F462
:10E04000862F90E00E94858404C0C80170E00E9481
:10E05000358487E0888780911F0589878091200516
:10E060008A87C8010E9404848F7741C180911F056F
:10E07000882319F00E94FB8202C00E94688188E018
:10E08000888736C18886892D65E2A2010E94166BB9
:10E090006091200570E07695762F662777956795D5
:10E0A00080911F0590E0682B792B892D0E945B776A
:10E0B0007B018C011886892D65E2A2010E94166BF6
:10E0C000B8868E2D8F77898797E016950795F794F8
:10E0D000E7949A95D1F78E2D8F778A8787E01695EA
:10E0E0000795F794E7948A95D1F78E2D8F778B87D4
:10E0F000B7E016950795F794E794BA95D1F78E2D6A
:10E100008F778C87A7E016950795F794E794AA95E3
:10E11000D1F7ED86EDC0B886892D64E2A2010E9498
:10E12000166B82E390E00E9496190E94F56951C136
:10E1300080E00E9449128886892D65E2A2010E9432
:10E14000166B90E1B91609F474C09B1580F0ADE030
:10E15000BA1679F1AB1520F0BCE0BB16B9F419C0C2
:10E16000EEE0BE16F1F1FFE0BF1681F44DC022E1F2
:10E17000B21609F472C0B21608F461C033E1B316E6
:10E1800009F47BC084E1B81609F48FC000E010E008
:10E1900097C08091200590E09695982F88279795B5
:10E1A000879520911F0530E0822B932B0E94AD763E
:10E1B00086C08091200590E09695982F88279795A6
:10E1C000879520911F0530E06091220567956627AD
:10E1D000679540912105642B822B932B0E94B77683
:10E1E0006EC08091200590E09695982F882797958E
:10E1F000879520911F0530E0609121056770822B83
:10E20000932B0E94C2765BC08091200590E096958A
:10E21000982F88279795879520911F0530E060916A
:10E2200021056770822B932B409122050E94CD76A9
:10E2300046C080911F058F700E948B7640C08091F0
:10E240001F056091210567956627679590912005C8
:10E25000692B8F700E94967632C08091200590E0E5
:10E260009695982F88279795879520911F0530E0E0
:10E27000822B932B0E94767622C08091200590E01D
:10E280009695982F88279795879520911F0530E0C0
:10E290006091220567956627679540912105642B5B
:10E2A000822B932B0E9480760AC08091200587954F
:10E2B0008827879590911F05892B0E94A2768C0153
:10E2C0001886892D65E2A2010E94166B85E1888778
:10E2D000802F8F778987C801880F892F881F990B16
:10E2E0008F778A87812F82958695869583708B8715
:10E2F000892D64E2A201A3CC00E010E0902EF80189
:10E30000EB5DFA4F80818823B1F4F02E802F64E01A
:10E310004EE155E00E94166B80911505801710F4B0
:10E32000009315059FE39F1560F00B5D1A4FEEE11A
:10E33000D801EC9306C093940F5F1F4F0034110572
:10E34000E9F6F4E0F093160544C080911605833099
:10E3500008F03FC023E02093160580911E058093AE
:10E36000170580911F0580931805809120058093E3
:10E37000190510921A052DC080911605823048F5B6
:10E3800032E030931605B0921705209318051092CD
:10E3900019051FC0809116058823D9F480921605AF
:10E3A00080911E05809317051092180512C08A30BF
:10E3B00019F48DE00E94CF15D8018D918D010E9436
:10E3C000CF15F8018081882321F0F5E004321F0782
:10E3D00071F72FE3291530F0E92DF0E0EB5DFA4FEE
:10E3E0003EE1308310921B058FEF80931D050E9444
:10E3F0002D18AFEF8F3F9A0709F0FCC90E94C01794
:10E400000A970CF444C1909110058091110598175A
:10E4100019F19091110589E0989F70011124ECEE9B
:10E42000F4E0EE0EFF1E00E010E0D7018D917D01BB
:10E430000E94D1170F5F1F4F09301105B1F780916E
:10E4400011058F5F8093110580911105843008F4C8
:10E450001EC1109211051BC18091EB04882311F09D
:10E46000DD2418C181E08093EB0490911205903473
:10E4700029F080911605882309F475C08FEF8E87E7
:10E48000809116058130B1F0813030F0823021F179
:10E49000833009F056C036C080E48F87809117051D
:10E4A000982F9770988B8F5F8093170521E1E22E4C
:10E4B000F12C4CC081E48F87809117058770888B81
:10E4C00080911805982F9F77998B8F5F80931805FF
:10E4D0009E012E5E3F4F2FC082E48F8780911705EB
:10E4E0008770888B809118058F77898B80911905AB
:10E4F000982F9F779A8B8F5F809319059E012D5ED1
:10E500003F4F19C083E48F87809117058770888BF0
:10E51000809118058F77898B809119058F778A8B69
:10E5200080911A05982F9F779B8B8F5F80931A0598
:10E530009E012C5E3F4F87FF02C0109216057901A5
:10E5400007C0109216059FE0E92EF12CEC0EFD1E7F
:10E5500080911605882329F4809112058F5F80939E
:10E560001205DD2472C0913409F043C08FEF8E870D
:10E5700083E08F870E942E12682FCE0140960E9462
:10E58000476B7C01809112058F5F809312050E947A
:10E59000ED3C8C01FC01848D81FF28C0D8018D9158
:10E5A0009C9111975E966C9144E00E94053CF801A5
:10E5B00046815781608571858081918124E00E9428
:10E5C000933BD80112968D919C911397009739F047
:10E5D0001A966D917C911B9744E00E94CC3BF80108
:10E5E000808191810E9454670E943667DD24D39414
:10E5F0002CC0903410F01092120590911205892FC2
:10E6000080688E8782E08F87903448F4E92FF0E0AD
:10E61000EB5DFA4F8081882311F0815080838091D7
:10E6200012058F5F80931205909115059E01205F62
:10E630003F4F981718F480E480931205DD24790188
:10E6400004C0D7011D927D0102C0CE014696E81696
:10E65000F906B8F3FF248E01025F1F4F86E1A82E52
:10E66000B12CAC0EBD1E8F2DF80160810E94526A44
:10E67000F82ED8018D918D010E94D1170A151B0526
:10E6800090F3F7FCF0948F2D0E94D11701C0DD2488
:10E690001092EB048D2DEB960FB6F894DEBF0FBEF3
:10E6A000CDBFCF91DF911F910F91FF90EF90DF9041
:10E6B000CF90BF90AF909F908F907F906F905F9022
:10E6C0004F903F902F90089580911C0587FF8ACE30
:10E6D000C3C80F931F93DF93CF9300D000D000D017
:10E6E000CDB7DEB7682F8E010F5F1F4FC8010E94A4
:10E6F000476B8FEF63E0A8010E94166B26960FB65A
:10E70000F894DEBF0FBECDBFCF91DF911F910F9167
:10E710000895EF92FF920F931F93CF93DF93182FDB
:10E7200080E00E94491282E390E00E94961984E002
:10E730000E944912112319F00E94853102C00E94E3
:10E74000C13184EF91E00E9496190E94F6250E9443
:10E75000FD2284E690E00E9496191123D9F00E94D0
:10E7600018238C0180E090E060E040E00E942833B4
:10E7700080E090E060E041E00E94283383E090E098
:10E780000E94C17484E690E00E9496190E941823AA
:10E79000EC015FC04AE0E42EF12C0E94FD220E94B1
:10E7A000F62560E070E080E090E040E20E941132E7
:10E7B00004C084E190E00E9496190E94DF2F882314
:10E7C000C1F30E9418238C010E94FD2260E070E0DA
:10E7D00080E090E841E00E94113260E070E080E06B
:10E7E00090E041E00E94113204C084E190E00E9478
:10E7F00096190E94DF2F8823C1F384E690E00E94DF
:10E8000096190E941823EC010531110534F0C80156
:10E81000880F991FC817D907C4F48E2D8A508230EB
:10E8200060F0C7010E94A13104C084E190E00E9421
:10E8300096190E94DF2F8823C1F30894E11CF11C74
:10E8400020E1E216F10409F0A8CF80E090E00E94F8
:10E85000A1310E94F625C8014497855A9B40B0F02B
:10E8600081E060E00E94C31E0431110514F48DE1C3
:10E8700001C08EE10E94D566BC0182E00E94972013
:10E8800080E00E94491288EE93E002C086E990E0A1
:10E890000E949619C801880F991F8C179D0754F480
:10E8A00081E0C53FD80734F098012C0F3D1F359506
:10E8B00027950AC024E0C13BD2071CF428EE33E0C0
:10E8C00003C09E01285C3040C901DF91CF911F91A8
:10E8D0000F91FF90EF900895DF93CF9300D000D079
:10E8E00000D0CDB7DEB716B886B187B90E940567EC
:10E8F000DC0114968C910E943A1EFE01319686E04E
:10E90000DF011D928A95E9F781E089838FEF62E24A
:10E91000AF010E94166BE2E6F0E080818D7F80837C
:10E9200026960FB6F894DEBF0FBECDBFCF91DF9114
:10E930000895DF93CF9300D000D000D0CDB7DEB7DD
:10E94000E2E6F0E080818260808380E00E943A1EEF
:10E95000FE01319686E0DF011D928A95E9F78FEF7F
:10E9600062E2AF010E94166B83EC87B98FEE86B925
:10E9700026960FB6F894DEBF0FBECDBFCF91DF91C4
:10E9800008950F931F93CF93DF93EC0101C0A895D7
:10E990000E94DF2F8823D9F311C0A89504C081E01D
:10E9A00090E00E9496190E94DF2F8823C1F380E037
:10E9B00090E060E041E00E948F3321970E94F922AD
:10E9C000882311F4209749F70E94F922082F15E0B7
:10E9D0000FC080E090E060E043E00E948F330E942F
:10E9E000FD2201C0A8950E94DF2F8823D9F3115082
:10E9F0000E94F922882319F0112359F707C0112327
:10EA000029F0802F002319F081E001C080E0DF9120
:10EA1000CF911F910F910895EF92FF920F931F9343
:10EA2000CF93DF937C01C0E0D0E0C7016C2F0E9440
:10EA3000E83280E090E00E94C174882319F40FEF5F
:10EA40001FEF02C00C2F10E0CF3FD10551F4E801B9
:10EA500083E090E00E94C174882349F00FEF10E03A
:10EA60000AC021968FEF0F3F1807F9F204C08FEF0D
:10EA70000F3F1807C1F0102FC701612F0E94E83225
:10EA800083E090E00E94C174882319F4CFEFDFEF98
:10EA900002C0C12FD0E0112331F08FEFCF3FD80754
:10EAA00011F41150E9CFCE01DF91CF911F910F9159
:10EAB000FF90EF9008952F923F924F925F926F9246
:10EAC0007F928F929F92AF92BF92CF92DF92EF92FE
:10EAD000FF920F931F93CF93DF93D82E7B01C42E09
:10EAE000A22E302E0E949974C7019695879596950F
:10EAF0008795482E4394CFEFDFEFBB2437E0632E9A
:10EB0000712C6E207F2023E0822E912C8E209F205E
:10EB10005A2C222481E00E9489730E9407230E94BC
:10EB2000FD220E942E12843009F0C7C083E0D8165F
:10EB300009F446C08D1530F081E0D81631F18D15FD
:10EB4000F8F00EC085E0D81640F086E08D1508F08C
:10EB500057C088E08D1508F072C0CFEFDFEF9FC07F
:10EB6000C7016C2D4A2D0E944F338FE090E00E9428
:10EB7000C174882309F493C0852D922DEC0189C0BE
:10EB8000C7016C2D0E94C8324BC0C7016C2D40E0FC
:10EB90000E94283383E090E00E94C174882309F02A
:10EBA000A2C0C7016C2D41E00E94283383E090E0B1
:10EBB0000E94C174882309F472C0C1E0D0E069C02A
:10EBC00010E000E00695C701612F40E00E94283365
:10EBD00083E090E00E94C174882309F400681F5FFD
:10EBE000183081F7C701602F0E94A83283E090E0BF
:10EBF0000E94C174882309F452C0C02FD0E049C0DC
:10EC000085E090E061E00E9408338FE090E00E9490
:10EC1000C17485E0D81661F4C3016C2D0E940833DD
:10EC20008FE090E00E94C174882309F05CC037C077
:10EC3000C3010E940C75EC0193E0B92E28C085E059
:10EC400090E0642D0E9408338FE090E00E94C17430
:10EC500087E0D81669F4C4016C2D0E9408338FE058
:10EC600090E00E94C174882349F0C0E0D0E006C063
:10EC7000C4010E940C75EC0183E0B82E85E090E0A1
:10EC800061E00E9408338FE090E00E94C174D7FDDC
:10EC900006C0332021F08CE291E00E94961980E0BA
:10ECA0000E944912D7FF09C08CE291E00E94961998
:10ECB000B39482E08B1508F02DCF0E946C74CE01C6
:10ECC000DF91CF911F910F91FF90EF90DF90CF9048
:10ECD000BF90AF909F908F907F906F905F904F907C
:10ECE0003F902F900895C0E0D0E0D3CF0F93BC01A8
:10ECF00088E040E020E000E00E945B750F910895FD
:10ED00000F939C01462F87E0B90120E001E00E94AB
:10ED10005B750F9108950F93682F86E070E040E0D7
:10ED200020E000E00E945B750F9108950F93982FEB
:10ED3000462F85E0692F70E020E001E00E945B75BE
:10ED40000F9108950F93482F85E060E070E020E078
:10ED500001E00E945B750F9108950F93BC0183E061
:10ED600040E020E000E00E945B750F9108950F9352
:10ED70009C01462F82E0B90120E001E00E945B7512
:10ED80000F9108950F939C01462F81E0B90120E077
:10ED900000E00E945B750F9108950F93FC01962F80
:10EDA000242F80E0BF01492F01E00E945B750F9185
:10EDB0000895DF92EF92FF920F931F9320913707F0
:10EDC000309138074091390750913A077C0100E0B3
:10EDD00010E0E20EF31E041F151F10C081E090E04A
:10EDE0000E9496190E94FD22C801B7010E94D01806
:10EDF000882391F40E94F922882311F0DD2401C0B8
:10EE0000D3940E94DF2F882349F30E94F92288239C
:10EE100029F789E08D1510F70E94DF2F882319F458
:10EE200080E090E008C00E94F92290E0811191E01A
:10EE300081E09827892F1F910F91FF90EF90DF902D
:10EE40000895EF92FF920F931F932091370730910F
:10EE500038074091390750913A077C0100E010E0F3
:10EE6000E20EF31E041F151F01C0A8950E94DF2F9C
:10EE70008823D9F301C0A8950E94F922882331F490
:10EE8000C801B7010E94D0188823A9F30E94DF2F80
:10EE9000882319F480E090E009C00E94F92290E0F4
:10EEA000882309F491E081E09827892F1F910F9121
:10EEB000FF90EF9008952F923F924F925F926F9242
:10EEC0007F928F929F92AF92BF92CF92DF92EF92FA
:10EED000FF920F931F93DF93CF93CDB7DEB7679762
:10EEE0000FB6F894DEBF0FBECDBF8B8B7D8B6C8BC6
:10EEF0000E94997480E00E9489738E8B9F8B8C890D
:10EF00009D890E94643B9A8B898B009771F0DC018C
:10EF100019961C92E989FA89148215821682178241
:10EF20008C899D8960E00E943D3C0E942E128430B5
:10EF300021F0CC24DD247601D9C118861F8288EE09
:10EF400093E00E94D97601E0CC24DD247601812C67
:10EF5000912CA12C60E8B62E09870E94041D0A9707
:10EF600009F4B5C1FB89FF3F51F581E060E00E94E3
:10EF7000C31E2DB73EB7295030400FB6F8943EBFA0
:10EF80000FBE2DBFEDB7FEB7319622E0ADB7BEB7CD
:10EF900011962C934DE558E15283418303831482EB
:10EFA000C582D682E782F0860E943D208DB79EB74B
:10EFB00009960FB6F8949EBF0FBE8DBF37C09AE07A
:10EFC00099838C2D8F778A83D701C60157E0B69538
:10EFD000A795979587955A95D1F78F778B83D7010A
:10EFE000C6014EE0B695A795979587954A95D1F7B6
:10EFF0008F778C83D701C60135E1B695A795979594
:10F0000087953A95D1F78F778D83D701C6012CE18B
:10F01000B695A795979587952A95D1F78E838B8975
:10F0200064E2AE014F5F5F4F0E94166B023028F41E
:10F0300020E030E040E050E80EC0802F90E00197E3
:10F0400020E030E040E050E804C056954795379501
:10F0500027958A95D2F72D873E874F87588B8E89C3
:10F060009F899C0119012601370135E03C87C101C8
:10F070000E94072384E690E00E94D976C301B20182
:10F08000402F0E9411328AE090E00E942177811186
:10F0900081E0182F0E9418239B878A878D859E8583
:10F0A000AF85B889482659266A267B2684E690E0F3
:10F0B0000E94D976C301B201402F0E9411328AE02A
:10F0C00090E00E942177811112600E941823AA8586
:10F0D000BB858A1B9B0B97FF03C0909581959F4F23
:10F0E0008059914014F484E005C0112311F01330CD
:10F0F000CCF0812FEC85E150EC87EE2391F0882352
:10F1000029F428E33FEF220E331E06C0833021F49A
:10F1100048EC50E0240E351E84E690E00E949619DB
:10F12000A6CF182F812F815031F0813051F4C8289B
:10F13000D928EA28FB28B694A794979487940F5F60
:10F1400015C0023028F0880C991CAA1CBB1C015069
:10F15000D501C40180959095A095B095C822D9227B
:10F16000EA22FB2284E690E00E94961959855F5FAF
:10F170005987503621F0013208F4EFCE03C0013236
:10F1800008F499C0C114D104E104F10409F493C056
:10F190008FEFC8168FEFD8068FEFE8068FEFF806CF
:10F1A00009F495C09B899F3F41F581E060E00E9492
:10F1B000C31EADB7BEB719970FB6F894BEBF0FBE4A
:10F1C000ADBFEDB7FEB7319622E011962C9341E525
:10F1D00058E1528341838F81988594838383C582CC
:10F1E000D682E782F0860E943D20ADB7BEB7199661
:10F1F0000FB6F894BEBF0FBEADBFE989FA89EF2BF9
:10F2000009F468C02C893D892115310509F462C0D3
:10F21000C701B601A9010E94F33188EE93E00E9474
:10F220009619BB2489899A8941E050E060E070E03A
:10F2300000E010E020E030E00E94C6330E94DF2FA3
:10F240008823E1F384E690E00E943319B39435E01B
:10F25000B31641F784E690E00E94D976C701B60163
:10F260004C895D890E94D5318AE090E00E94217727
:10F27000882381F54B894F3FF1F481E060E00E94E3
:10F28000C31E00D000D00F92EDB7FEB7319622E03A
:10F29000ADB7BEB711962C934FE358E1528341832B
:10F2A0008F819885948383830E943D200F900F90D7
:10F2B0000F900F900F9088EE93E00E949619AF8107
:10F2C000B8851196B887AF83159709F038CECC244E
:10F2D000DD24760180E00E944912C114D104E104CA
:10F2E000F10421F488EE93E00E9496190E946C7458
:10F2F00080E00E944912B601C70167960FB6F894E4
:10F30000DEBF0FBECDBFCF91DF911F910F91FF9058
:10F31000EF90DF90CF90BF90AF909F908F907F90B5
:10F320006F905F904F903F902F900895662319F053
:10F3300024E93BE002C02CEF3BE0F894E82FF0E03A
:10F34000EE0FFF1FE20FF31F208191818091640C6B
:10F3500080FF02C0118210827894822F0895E82FD6
:10F36000F8947894F0E0EE0FFF1FEF58F34F808190
:10F37000918108959091640C882311F0916001C0EF
:10F380009E7F9093640C0895BF92CF92DF92EF928C
:10F39000FF920F931F93CF93DF93882339F03BE6BF
:10F3A000C32E3CE0D32EC4E9DBE006C025E6C22E26
:10F3B0002CE0D22ECCEFDBE00E940567FC01B0848C
:10F3C00001E71CE07E01C0E0D0E018C0F894F8012D
:10F3D00080819181F70191838083F80180819181FF
:10F3E000892B21F0C601BE010E940C8978942196D8
:10F3F0000E5F1F4F82E090E0E80EF91ECB1530F350
:10F40000DF91CF911F910F91FF90EF90DF90CF9000
:10F41000BF90089584E0809374001092710083E09F
:10F420008093700008951F920F920FB60F920BB643
:10F430000F9211248F939F93EF93FF93809171000C
:10F4400090E0887F90708032910509F485C0813208
:10F4500091055CF480319105D1F08831910509F472
:10F4600042C0089709F07AC016C080349105A9F10E
:10F470008134910524F4889709F070C03EC080352E
:10F480009105D9F08835910509F068C00AC08091CE
:10F49000650587FF02C080EA01C081EA809373009E
:10F4A00059C0E0916B05F0916C05809173008193D8
:10F4B000F0936C05E0936B0546C0E0916B05F0910D
:10F4C0006C05809173008193F0936C05E0936B055C
:10F4D0008091660581508093660580916605823033
:10F4E000CCF185EC3FC08091690590916A059093BD
:10F4F00073008FEF809365052DC08091650587FFB0
:10F5000009C08091690590916A05809373001092FB
:10F51000650520C0809167058823F1F0809166051C
:10F52000882389F0E0916B05F0916C0581918093BF
:10F530007300F0936C05E0936B0580916605815034
:10F540008093660507C084E98093740081E080930E
:10F5500068050AC085E806C085EA04C08FEF80937D
:10F56000680584E980937400FF91EF919F918F91DA
:10F570000F900BBE0F900FBE0F901F9018958091AB
:10F58000740020E090E087709070892B09F021E0F2
:10F59000822F08956093660590936A0580936905AC
:10F5A0002093670550936C0540936B058EEF809315
:10F5B00065051092680585EA80937400089520918E
:10F5C0006805332727FD3095C901089560936605C6
:10F5D00090936A05809369052093670550936C05A5
:10F5E00040936B058EEF809365051092680585EA60
:10F5F0008093740001C0A895809168058823D9F391
:10F6000020916805332727FD3095C9010895CF92D1
:10F61000DF92EF92FF920F931F93DF93CF9300D06F
:10F62000CDB7DEB77C011A8219826E010894C11C25
:10F63000D11C09811A81C80124E0880F991F2A95DD
:10F64000E1F762E0A60120E00E94E67AA8958981B0
:10F650009A81009721F08E159F0559F704C0EF2875
:10F6600011F000E010E0C8010F900F90CF91DF91F2
:10F670001F910F91FF90EF90DF90CF900895EF9240
:10F68000FF920F931F93DF93CF9300D0CDB7DEB7D8
:10F690008C0101978F5F934000F5C80144E0880F0B
:10F6A000991F4A95E1F762E07E010894E11CF11C84
:10F6B000A70120E00E94E67AC8010E94077B24E0AF
:10F6C0008030920750F434E0880F991F3A95E1F7A3
:10F6D00062E0A70121E00E94E67A0F900F90CF919F
:10F6E000DF911F910F91FF90EF900895AC0180E0A2
:10F6F00090E066E021E00E94E67A0895BF92CF9202
:10F70000DF92EF92FF920F931F93DF93CF93CDB7CA
:10F71000DEB766970FB6F894DEBF0FBECDBF1E8270
:10F720001D821A82198281E090E09C838B83A895C8
:10F7300080E090E066E0AE014F5F5F4F21E00E9405
:10F74000E67A8E01095F1F4FC8016FEF70E040E15C
:10F7500050E00E94C0A061E0E62EF12C50E1C52EE1
:10F76000D12CB02E012F8FEFE81683E0F80649F078
:10F770000894E11CF11CF886EF820894E108F10876
:10F7800002C018861F820E943512C60160E14B2D0F
:10F79000502F21E00E94E67A0894E11CF11C80E1E0
:10F7A00090E0C80ED91E90E0E91694E0F906D9F66B
:10F7B00066960FB6F894DEBF0FBECDBFCF91DF9136
:10F7C0001F910F91FF90EF90DF90CF90BF90089521
:10F7D000AC0180E090E066E020E00E94E67A0895C7
:10F7E000CF92DF92EF92FF920F931F93DF93CF930D
:10F7F000CDB7DEB766970FB6F894DEBF0FBECDBFAC
:10F800006C0101978F5F934080F5C6010E943F7B9A
:10F8100080E090E066E07E010894E11CF11CA70105
:10F8200020E00E94E67A8E01095F1F4FC8016FEF4A
:10F8300070E040E150E00E94C0A08B819C819887DD
:10F840008F83C60174E0880F991F7A95E1F760E114
:10F85000A80121E00E94E67ADC82CB8280E090E081
:10F8600066E0A70121E00E94E67A66960FB6F8945A
:10F87000DEBF0FBECDBFCF91DF911F910F91FF90E3
:10F88000EF90DF90CF9008950E94F07B0895DF9372
:10F89000CF9300D000D000D0CDB7DEB724E08130C8
:10F8A000920718F020E030E018C0009761F480E083
:10F8B00090E066E0AE014F5F5F4F20E00E94E67A85
:10F8C00029813A810AC00E94077B9C01009729F494
:10F8D00080E090E00E94077B9C01C90126960FB64C
:10F8E000F894DEBF0FBECDBFCF91DF9108950F9387
:10F8F0001F93DF93CF93CDB7DEB766970FB6F8941B
:10F90000DEBF0FBECDBF8C0144E08130940718F0FC
:10F9100020E030E022C080E090E066E0AE014F5F82
:10F920005F4F20E00E94E67A01151105A1F0C801A1
:10F93000E4E0880F991FEA95E1F760E1AE01495FC5
:10F940005F4F20E00E94E67A2F813885C901019738
:10F950008E5F9F4F10F029813A81C90166960FB6DC
:10F96000F894DEBF0FBECDBFCF91DF911F910F91F5
:10F970000895CF92DF92EF92FF920F931F93DF9340
:10F98000CF93CDB7DEB766970FB6F894DEBF0FBE44
:10F99000CDBF7C01009741F180E090E066E0AE01D0
:10F9A0004F5F5F4F20E00E94E67A09811A81A7E04D
:10F9B000CA2ED12CCC0EDD1E12C0C801F4E0880F77
:10F9C000991FFA95E1F764E0A60120E00E94E67A2B
:10F9D00089859A858E159F0549F00F811885C80184
:10F9E00001978E5F9F4F48F300E010E0C8016696D4
:10F9F0000FB6F894DEBF0FBECDBFCF91DF911F9140
:10FA00000F91FF90EF90DF90CF900895EF92FF92CB
:10FA10000F931F93DF93CF9300D000D000D0CDB7CA
:10FA2000DEB780E090E066E07E010894E11CF11C06
:10FA3000A70120E00E94E67A0B811C8101151105C7
:10FA4000A1F0C801B4E0880F991FBA95E1F762E010
:10FA5000AE014D5F5F4F20E00E94E67A80E090E0CB
:10FA600066E0A70121E00E94E67AC80126960FB65B
:10FA7000F894DEBF0FBECDBFCF91DF911F910F91E4
:10FA8000FF90EF900895CF92DF92EF92FF920F9345
:10FA90001F93DF93CF93CDB7DEB766970FB6F89479
:10FAA000DEBF0FBECDBF80E090E066E0AE014F5FED
:10FAB0005F4F20E00E94E67A89E00E94E01C8823E4
:10FAC00029F08EE00E94E01C882351F48B819C81F8
:10FAD0008F5F9F4F21F589819A818F5F9F4FF9F446
:10FAE00084E06EEB71E00E94A41F85E066EC71E09B
:10FAF0000E94A41F81E794E968EC70E00E94021E56
:10FB000080E060E00E94C31E83E00E94D566BC01D5
:10FB100082E00E9497200E947E7B0E944C670981B0
:10FB20001A8137E0C32ED12CCC0EDD1E1BC0C801BC
:10FB300024E0880F991F2A95E1F760E1A60120E0F3
:10FB40000E94E67AFF80E88489859A8501978F5F15
:10FB50009F4318F0C8010E94F07BA8958F2D9E2D21
:10FB60009C018901C80101978F5F934000F38D814B
:10FB70009E818F5F9F4F99F480E090E066E08E0158
:10FB80000F5F1F4FA80120E00E94E67A1E821D82AF
:10FB900080E090E066E0A80121E00E94E67A6696A7
:10FBA0000FB6F894DEBF0FBECDBFCF91DF911F918E
:10FBB0000F91FF90EF90DF90CF900895EF92FF921A
:10FBC0000F931F93DF93CF93CDB7DEB760970FB638
:10FBD000F894DEBF0FBECDBF9C017B018A01019767
:10FBE0008F5F934018F020E030E022C0C90144E06C
:10FBF000880F991F4A95E1F760E1AE014F5F5F4FB3
:10FC000020E00E94E67AE114F10419F08D81F701F9
:10FC100080830115110551F0D801FE0136968BE065
:10FC200001900D928150E1F7F80113862B813C8100
:10FC3000C90160960FB6F894DEBF0FBECDBFCF915D
:10FC4000DF911F910F91FF90EF9008958F929F92F7
:10FC5000AF92BF92CF92DF92EF92FF920F931F93DA
:10FC6000DF93CF93CDB7DEB7A8970FB6F894DEBF7A
:10FC70000FBECDBF8C016B01B42E7901211531056A
:10FC800009F48CC06115710509F488C084E0003066
:10FC9000180708F083C00115110521F0C8010E9462
:10FCA0003F7B06C00E94067D8C01009709F476C058
:10FCB000DC86CB86BD86FE013E969E01275E3F4FC9
:10FCC00004C081930894E11CF11CD7018C91882316
:10FCD00021F0E217F307A9F704C0E217F30708F4CD
:10FCE00010821A83098380E090E066E0AE014D5FE8
:10FCF0005F4F20E00E94E67A0B811C81EE24FF24F6
:10FD0000A9E18A2E912C8C0E9D1EFEE1AF2EB12C06
:10FD1000AC0EBD1EEEE0CE2ED12CCC0EDD1E19C0D9
:10FD2000A895C80174E0880F991F7A95E1F760E102
:10FD3000A40120E00E94E67AC501B6014BE050E044
:10FD40000E94D9A097FF08C07801898D9A8D9C01E7
:10FD500089010115110521F71A870987A89589815D
:10FD60009A8164E0880F991F6A95E1F760E1AE011E
:10FD7000475F5F4F21E00E94E67AC70154E0880F99
:10FD8000991F5A95E1F762E0AE014F5F5F4F21E0A6
:10FD90000E94E67A29813A81C9018C01C801A8969E
:10FDA0000FB6F894DEBF0FBECDBFCF91DF911F918C
:10FDB0000F91FF90EF90DF90CF90BF90AF909F900A
:10FDC0008F900895BF92CF92DF92EF92FF920F93A0
:10FDD0001F93DF93CF93CDB7DEB72D970FB6F8946F
:10FDE000DEBF0FBECDBF7C01B62E0E94B97C8C0158
:10FDF0000097B9F0B2E0CB2ED12CCC0EDD1EBE01A7
:10FE00006F5F7F4FA6010E94DE7DBC018E159F05AE
:10FE100041F489818B1529F0C8014B2D96010E9470
:10FE2000267E2D960FB6F894DEBF0FBECDBFCF91C4
:10FE3000DF911F910F91FF90EF90DF90CF90BF90D7
:10FE40000895FC01A62F9A0180E090E0BF014A2F9F
:10FE50000E94267E0895CF92DF92EF92FF920F9339
:10FE60001F93DF93CF9300D000D000D0CDB7DEB783
:10FE70006C017B01CE0101960E94E87B0D811E8101
:10FE800024E000301207E0F020C0A895C80124E06B
:10FE9000880F991F2A95E1F760E1A70120E00E94F1
:10FEA000E67AF70120E0828193819F778C159D058A
:10FEB00071F02F5F32962730B1F7F7010081118181
:10FEC000C80101978F5F934000F300E010E0C80184
:10FED00026960FB6F894DEBF0FBECDBFCF91DF914F
:10FEE0001F910F91FF90EF90DF90CF900895CF92E8
:10FEF000DF92EF92FF920F931F93DF93CF93CDB7D3
:10FF0000DEB7A0970FB6F894DEBF0FBECDBFBE011F
:10FF10006F5E7F4F0E942B7F7C01009709F45DC0CC
:10FF2000CE010B960E94E87B0F8518890E151F05E0
:10FF3000B1F400E010E020C0A895C80164E0880F8B
:10FF4000991F6A95E1F762E0A60120E00E94E67A37
:10FF50008B819C818E159F0559F08C0105C053E063
:10FF6000C52ED12CCC0EDD1E0115110529F735C08B
:10FF700084E00030180788F589899A899A838983F3
:10FF8000CE0105960E94E87B0115110529F48981AF
:10FF90009A819A8789870DC0C80144E0880F991F0C
:10FFA0004A95E1F762E0AE014F5F5F4F21E00E94AA
:10FFB000E67AA895C70134E0880F991F3A95E1F7D2
:10FFC00062E0AE01495F5F4F21E00E94E67AF88669
:10FFD000EF82CE0105960E94767BA0960FB6F8942C
:10FFE000DEBF0FBECDBFCF91DF911F910F91FF906C
:10FFF000EF90DF90CF9008956F927F928F929F92B3
:020000021000EC
:10000000AF92BF92CF92DF92EF92FF920F931F9326
:10001000DF93CF93CDB7DEB766970FB6F894DEBF08
:100020000FBECDBF4C0180916D05882309F085C0BE
:10003000C4010E9469378C01009709F47EC0DC017D
:1000400012968D919C911397892B09F476C018967E
:10005000BC90C401BE01695F7F4F0E942B7F7C0171
:100060000097C9F40E94067D7C01009709F467C0DF
:10007000CE0101960E94E87B8D819E8198878F83B7
:100080008050944010F018861F82FE82ED82CE01CF
:1000900001960E94767B8EE0FE013996DF011D926B
:1000A0008A95E9F79A868986ABE0CA2ED12CCC0EC8
:1000B000DD1EF7E16F2E712C6C0E7D1EAB2CBB2468
:1000C000A7FCB094AA24BB0CAA1CBB241DC00E9490
:1000D00069378C01009719F1FC0120813181D6012B
:1000E0002D933C9340E050E0808587FF02C041E0C3
:1000F00050E04A155B0521F03068F601318320831A
:1001000082E090E0C80ED91ED80112968D919C9184
:1001100013978815990519F0C614D704C1F6C701BD
:1001200074E0880F991F7A95E1F760E1AE01495FAD
:100130005F4F21E00E94E67A02C0EE24FF24C7014F
:1001400066960FB6F894DEBF0FBECDBFCF91DF919C
:100150001F910F91FF90EF90DF90CF90BF90AF90E5
:100160009F908F907F906F900895CF92DF92EF9243
:10017000FF920F931F93DF93CF93CDB7DEB76097B6
:100180000FB6F894DEBF0FBECDBF9C0180916D0508
:100190008823C1F5C901BE016F5F7F4F0E942B7F8D
:1001A000892B81F181E080936D05EB80FC80C70194
:1001B0000E94643B892B11F18E010B5F1F4FBFE042
:1001C000CB2ED12CCC0EDD1EF801208131813F7762
:1001D000C90101978E5F9F4358F4C9010E94643B97
:1001E000892B61F0F80160817181C7010E942B3B6E
:1001F0000C151D0519F00E5F1F4FE6CF10926D050F
:1002000081E001C080E060960FB6F894DEBF0FBEBB
:10021000CDBFCF91DF911F910F91FF90EF90DF90B5
:10022000CF900895EF92FF920F931F93DF93CF9398
:10023000CDB7DEB728970FB6F894DEBF0FBECDBF9F
:100240007B018C0180916E0590916F05892B99F14E
:10025000E982FA820B831C8318861F82122F20FFEB
:100260000AC058874F83CA0160E070E040E050E068
:100270000E94DE7DAC0111FF05C08F8198859068DA
:1002800098878F8341155105B1F080916E0590914B
:100290006F055E834D8368E0AE014F5F5F4F21E0E5
:1002A0000E94E67A80916E0590916F050896909372
:1002B0006F0580936E0528960FB6F894DEBF0FBECB
:1002C000CDBFCF91DF911F910F91FF90EF900895D7
:1002D0005F926F927F928F929F92AF92BF92CF92D6
:1002E000DF92EF92FF920F931F93DF93CF93CDB7DF
:1002F000DEB76C970FB6F894DEBF0FBECDBF0E947D
:100300002E12582E80E00E94491280E090E060E0BA
:1003100040E050E00E946A43FE01319686E0DF0132
:100320001D928A95E9F710E0FE2E0F2F812F67E0CE
:100330004F2D502F0E94166B84E190E00E94961979
:100340001F5F103499F70E94A7391E861D86A12CC5
:1003500010E4B12EBDE0EB2EF12CEC0EFD1E30C0F2
:10036000C50168E0A70120E00E94E67A8D859E85A0
:10037000BFEF8F3F9B0701F10E94643B8C01009708
:10038000D9F06B896F70FC01808191810E94B53C2E
:100390008F859889D80113969C938E93129789899B
:1003A0009A89A0E0B0E0F80184839583A683B7839F
:1003B0008B899C8990FD108688E090E0A80EB91E7C
:1003C0008D859E858F5F9F4F59F61D8A1E8A1F8AD5
:1003D000188EA5E16A2E712C6C0E7D1EF7E08F2E13
:1003E000912C8C0E9D1EC7C0C50168E0A30120E0C2
:1003F0000E94E67A8D899E89AF89B88D80509040A1
:10040000A040B14008F0B3C0E98CFA8CE114F104CB
:1004100009F4ADC0F0E0EF16F0E4FF0608F0A7C065
:100420008B8D9C8DD92EDD1CDD24DD1CDD0C009711
:1004300011F4870111C08C011F77C80160E070E0E2
:1004400040E050E00E94DE7DE816F90619F421E054
:10045000D22A02C0098D1A8D2D893E894F89588D67
:10046000CD2CDD24211531054105510509F044C08D
:100470000E94ED3C7C01C0FE09C0AC014C5D5F4FA9
:10048000C80160E070E00E94DE7D8C01C8010E941E
:1004900069378C01009711F1DC0114964D915C9144
:1004A00015978D919C91119718966C910E946A43B3
:1004B000F801818560E070E00E944943D8011296FE
:1004C0008D919C9113970E946937FC01009731F040
:1004D00064817581808191810E948C3DC1FE04C040
:1004E000F701848D8160848FD7015C968C915C9735
:1004F00082605C968C933BC0802F8F778F83000F38
:10050000012F001F110B1195802F8F778887822F65
:100510008F77898777E056954795379527957A9510
:10052000D1F7822F8F778A8767E056954795379561
:1005300027956A95D1F7822F8F778B8793E0CC0C24
:10054000DD1C9A95E1F787E05695479537952795F5
:100550008A95D1F7822F87708C298C878FEF6CE07A
:10056000A4010E94166B0E94C26B8823E1F3E8E0AD
:10057000F0E0AE0EBF1E8D899E89AF89B88D805088
:100580009040A040B14008F42FCF09ED1CE0C50118
:1005900068E0A80120E00E94E67A88E090E0A80EDA
:1005A000B91E085F1F4F9DE0093D190781F783E0E1
:1005B0000E94491284E690E00E9496198F859889DE
:1005C0000E94FF86852D0E9449126C960FB6F89402
:1005D000DEBF0FBECDBFCF91DF911F910F91FF9076
:1005E000EF90DF90CF90BF90AF909F908F907F90D3
:1005F0006F905F9008958F929F92AF92BF92CF922B
:10060000DF92EF92FF920F931F93DF93CF93CDB7BB
:10061000DEB728970FB6F894DEBF0FBECDBF00E05F
:1006200010E4FF248BE0882E912C5E010894A11C1D
:10063000B11C2FC08F2D90E0889DF001899DF00D99
:10064000989DF00D1124EE52F74FC080D180A28109
:10065000B38144815581668177818185282F30E07F
:100660002F70307038872F83808587FD03C03160FD
:1006700038872F835E834D83BC83AB83DA82C98244
:10068000C80168E0A50121E00E94E67AF394085FC2
:100690001F4F8091920BF81668F20E9405672FEFAA
:1006A0003FEF3A832983FC01858596859C838B8364
:1006B000C80168E0AE014F5F5F4F21E00E94E67A1B
:1006C0000E94ED3CFC01085F1F4F10936F050093E3
:1006D0006E0542A153A1848D4115510531F080FD75
:1006E00002C021E009C023E007C04081518180FDA4
:1006F00002C020E001C022E060E070E080E090E015
:100700000E94128110E0812F6BE040E050E00E94D7
:10071000166B1F5F1034B9F710E00E94C26B88237C
:10072000E1F31F5F1630C9F76FEF7FEF8FEF9FEF99
:100730004FEF5FEF20E00E941281E0906E05F09095
:100740006F0510926F0510926E0509ED1CE0C70150
:1007500068E0A80121E00E94E67A88E090E0E80ED7
:10076000F91E085F1F4F9DE0093D190781F7289684
:100770000FB6F894DEBF0FBECDBFCF91DF911F91B2
:100780000F91FF90EF90DF90CF90BF90AF909F9030
:100790008F900895E0E7F5E08FEF9FEF91838083DE
:1007A000379626E0E035F207C9F708950F931F93B7
:1007B0008C0189ED9CE0B8010E943789482F98018F
:1007C000220F331F442311F02F5F3F4FE0E7F5E086
:1007D000808191818217930749F4868180FF0CC044
:1007E000442311F487E40DC082E50BC086E0E934B0
:1007F000F80711F03796ECCF442311F487E601C0D7
:1008000082E71F910F9108950F931F932FE0803F70
:10081000920718F02FEF3FEF24C09C0136952795E3
:1008200043E02D3F3407D8F48901169507951695B6
:10083000079526E0969587952A95E1F78452904F83
:100840000E9492A390E00770107002C09595879562
:100850000A95E2F780FD03C021E030E002C023E00A
:1008600030E0C9011F910F910895EF92FF920F930D
:100870001F93CF93DF937B012FE0803F920708F017
:100880003DC06330710519F061307105B9F59C0107
:100890003695279543E02D3F340780F5890116955D
:1008A000079516950795EC0156E0D695C7955A958C
:1008B000E1F7C452D04FCE010E9492A3482F980175
:1008C0002770307083E0E816F10451F481E090E085
:1008D00002C0880F991F2A95E2F7642F682B0AC07F
:1008E00081E090E002C0880F991F2A95E2F7682FF7
:1008F00060956423A895CE010E94A4A3DF91CF91B7
:100900001F910F91FF90EF9008951F93CF93DF9366
:10091000039711F010E001C01FEFCCEDDFE0A895C8
:10092000CE01612F0E94A4A321968FE0CC3FD8076F
:10093000B1F7DF91CF911F910895CF93DF93EC0131
:10094000662331F089ED9CE0BE010E940C8905C050
:1009500089ED9CE0BE010E942189CC0FCD2FCC1FD8
:10096000DD0BD19581E090E002C0880F991FCA95F8
:10097000E2F72091500630915106282B392B309305
:1009800051062093500688EB9BE09093530680938A
:100990005206DF91CF9108951F93CF93DF93EC011F
:1009A000162F8FE0C03FD80708F589ED9CE0BE0107
:1009B0000E943789181761F0CE01612F0E949D8433
:1009C000CE0160E00E943088CE0161E00E94308854
:1009D0000E940567FC01858596858C179D0730F47C
:1009E000C07F2F96D687C5870E947169DF91CF910E
:1009F0001F910895DF92EF92FF920F931F93DF9361
:100A0000CF9300D000D000D0CDB7DEB78C01D62E6A
:100A1000009709F462C0FC01E080F1806623F9F0E0
:100A2000C70161E00E941630882309F456C0809106
:100A3000370790913807A0913907B0913A07F8012C
:100A400082839383A483B5838681816086836E2DA0
:100A50006170C701969587950E949D840BC0C70160
:100A600060E00E9416308823C1F18FEF9FEFF801FC
:100A700091838083F801868183FF06C0C701969524
:100A8000879560E00E943088F801868184FF06C067
:100A9000C7019695879561E00E9430888E2D8F77EB
:100AA0008983C701880F892F881F990B91958F77AC
:100AB0008A838F2D82958695869583708B831C8281
:100AC000DD2011F081E08C838FEF63E2AE014F5F98
:100AD0005F4F0E94166B81E001C080E026960FB642
:100AE000F894DEBF0FBECDBFCF91DF911F910F9164
:100AF000FF90EF90DF9008956F927F928F929F9278
:100B0000AF92BF92CF92DF92EF92FF920F931F931B
:100B1000CF93DF930E94C322882309F4E8C00E9488
:100B200005678C01FC01638570E080E090E022E3C2
:100B300030E040E050E00E94E19E3B014C01F801B2
:100B4000648570E080E090E024E630E040E050E032
:100B50000E94E19E5B016C01C0E7D5E0EE24FF241A
:100B600000E010E048815981FFEF4F3F5F0709F433
:100B70006DC08E8180FF36C082FD0FC06A817B818F
:100B80008C819D81660D771D881D991D0E94D0184E
:100B9000882319F08E8184608E838E8181FF02C04C
:100BA00082FD0DC06A817B818C819D816A0D7B1DD8
:100BB0008C1D9D1D0E94D018882309F447C0011583
:100BC000110509F442C0F801228133814481558125
:100BD0008A819B81AC81BD8182179307A407B507E9
:100BE000A0F134C0BA01B3E076956795BA95E1F704
:100BF000E0E7F5E0208131818FEF2F3F380771F07A
:100C00002417350759F0868180FF08C0A3E0369588
:100C10002795AA95E1F726173707C1F086E0E93452
:100C2000F80709F45FC03796E5CFF70122813381D9
:100C3000448155818A819B81AC81BD818217930754
:100C4000A407B50718F47E0101C08E01F6E0C9348F
:100C5000DF0711F0279686CF0115110519F0C8019D
:100C600060E005C0E114F10421F0C70161E00E94D9
:100C7000FA8480915206909153060097C1F1019732
:100C80009093530680935206892B89F580915006E4
:100C900090915106892B59F101E010E0C0E0DFE7A7
:100CA0002091500630915106C80182239323892B4D
:100CB00089F0C801809590958223932390935106E3
:100CC00080935006AE0147525247CE0160E121E0C9
:100CD0000E94E67A000F111F8FE7C03FD80739F056
:100CE0006096DECFE114F10409F09FCFACCFDF9125
:100CF000CF911F910F91FF90EF90DF90CF90BF9019
:100D0000AF909F908F907F906F9008950F931F9357
:100D1000CF93DF93EC01162F042F2FE0803F920733
:100D200008F067C00E942E12833019F4E0E7F5E066
:100D300007C00E942E12823009F05BC0F7CF3796B1
:100D4000808191818C179D0719F186E0E934F807BD
:100D5000B1F7112309F1E0E7F5E0808191818F5F20
:100D60009F4F81F4D183C0838091370790913807DA
:100D7000A0913907B0913A0782839383A483B58306
:100D8000168206C086E0E934F80799F13796E5CF78
:100D9000309759F4112369F5CE018170682FCE0187
:100DA000969587950E949D8422C0112319F486810F
:100DB00082608683002329F08681886086830130E3
:100DC00019F08681806186830E940567FC011123EA
:100DD00061F0BE017695679585859685861797079C
:100DE00020F4768765870E9471690E947C8581E086
:100DF00001C080E0DF91CF911F910F9108953F9244
:100E00004F925F926F927F928F929F92AF92BF921A
:100E1000CF92DF92EF92FF920F931F93CF93DF93C6
:100E20005C0127E0883F920708F082C00E940567B6
:100E30003C01DC011E96BC92AE921D970E94716926
:100E40008824992400E010E092E0392E25010894CE
:100E5000411C511C7801CC24DD244FC0E701CC0F8C
:100E6000DD1FB601600F711F89ED9CE00E9437897C
:100E7000882331F0219604C08AE090E00E94961900
:100E8000CE0161E044E00E9486868823A9F3CE016A
:100E900060E044E00E94868681E060E00E94C31E1C
:100EA00080E20E94D5660894811C911CEDB7FEB7C4
:100EB00037970FB6F894FEBF0FBEEDBF3196ADB7B2
:100EC000BEB711963C92928381839482838256822C
:100ED00045820E943D20EDB7FEB737960FB6F894D5
:100EE000FEBF0FBEEDBF84E690E00E94961924E09D
:100EF00030E0E20EF31EC20ED31EAE14BF0408F0A3
:100F0000ADCFD3011B968C9190E00E9496190F5F94
:100F10001F4F0430110509F09DCF84E690E00E9438
:100F2000961902C00E9435120E94DF2F8823D1F348
:100F3000DF91CF911F910F91FF90EF90DF90CF90B5
:100F4000BF90AF909F908F907F906F905F904F90E9
:100F50003F90089580E09FE760E449ED5CE020E089
:100F60000E94E67A80E49FE760E449E15DE020E0EA
:100F70000E94E67A80E89FE760E449E55DE020E0D2
:100F80000E94E67A80EC9FE760E449E95DE020E0BA
:100F90000E94E67A0895DC018C91803108F01C9261
:100FA0008C91E82FF0E03196EE0FFF1FEA0FFB1F48
:100FB000718360838F5F8C93803108F01C929C91C9
:100FC00011968C911197981749F4892F8F5F11967C
:100FD0008C931197803110F011961C9208958823FC
:100FE000C1F49091570680915606891751F1E92F67
:100FF000F0E0EE0FFF1FE85AF94F0190F081E02D6D
:10100000892F8F5F809357068031E8F01092570642
:101010001AC09091790680917806891791F0E92F8E
:10102000F0E0EE0FFF1FE658F94F0190F081E02D40
:10103000892F8F5F80937906803128F0109279068E
:1010400002C0EFEFFFEFCF01089590915406982B67
:101050009093540690915506982B909355060895B9
:101060009C0187E0283F380778F4662331F486E551
:1010700096E0B9010E94CB870895613029F488E792
:1010800096E0B9010E94CB8708950F931F93CF93E9
:10109000DF93109255061092540610925706109244
:1010A0005606109279061092780600E010E0C0E033
:1010B000D0E01DC0F894FE01E159F34F8081918189
:1010C000FE01EE56F44F91838083FE01E650F44F0B
:1010D0009183808385E69CE0B8010E9421898BE69C
:1010E0009CE0B8010E94218978940F5F1F4F0E94F5
:1010F00005672296FC01808590E008171907D4F255
:101100009091920BE2EDF8E08BE0989F9001112412
:101110002E0F3F1F04C081858F7981873B96E21790
:10112000F307C9F7DF91CF911F910F910895EF92C7
:10113000FF920F931F93CF93DF93882371F48091D5
:101140005406082F10E010925406E6E5F6E065E636
:10115000E62E6CE0F62E60E20DC080915506082F59
:1011600010E010925506E8E7F6E05BE6E52E5CE05D
:10117000F52E60E490818181981310688091920B24
:10118000482F50E0EBEDF8E020E030E009C080812E
:1011900086233B96882311F0106405C02F5F3F4FD4
:1011A00024173507A4F3C0E0D0E009C0F701EC0F25
:1011B000FD1F8081882311F010620FC021960E94CC
:1011C0000567FC01808590E0079643E0959587953B
:1011D0004A95E1F7C817D9074CF3C801DF91CF91C1
:1011E0001F910F91FF90EF9008951F93162F20E409
:1011F0008030920778F40E946937FC01009751F023
:10120000112329F0818580628187113019F0818551
:10121000806481871F910895FB0123E0F595E79590
:101220002A95E1F7E80FF91F6770707081E090E090
:1012300002C0880F991F6A95E2F72081282B20832E
:101240000895FB0133E0F595E7953A95E1F7E80F4E
:10125000F91F6770707081E090E002C0880F991FDD
:101260006A95E2F780952081282320830895FB0169
:1012700043E0F595E7954A95E1F7E80FF91F80817E
:1012800090E06770707002C0959587956A95E2F757
:1012900081700895FB0157FD02C021E004C0509504
:1012A00041955F4F20E08330910541F184309105F5
:1012B00034F48130910501F1029751F523C0843057
:1012C000910519F0059721F50AC081818F5F81830F
:1012D00090E084179507E4F0222351F00DC081813E
:1012E0008150818390E08417950794F0222321F0A8
:1012F000842F815081830CC011820AC01282138214
:10130000168A06C090E08281882309F491E09283D6
:1013100080E090E008958230910519F0039751F430
:1013200003C02FEF3FEF08C083E090E040E050E0C3
:101330000E944A8920E030E0C90108951F93182FC8
:101340000E94ED3CFC01848D112311F0806401C0EA
:101350008F7B848F1F9108951F93CF93DF93EC01B0
:101360008A81882309F470C081E060E00E94C31E76
:1013700000D000D00F92EDB7FEB7319612E0ADB7B6
:10138000BEB711961C9380E099E1928381838C8192
:101390009D81948383830E943D200F900F900F9036
:1013A0000F900F908B81843079F400D00F92EDB7BD
:1013B000FEB711838CEF98E1938382830E943D20D6
:1013C0000F900F900F9018C000D000D00F92EDB783
:1013D000FEB73196ADB7BEB711961C9388EF98E172
:1013E000928381838885838314820E943D200F909D
:1013F0000F900F900F900F90898D9A8D97FD04C0DC
:1014000082E060EF78E10CC08E5F9F4F21F482E0B4
:1014100068EE78E105C084E00E94D566BC0182E0F8
:101420000E94972081E0888F8E8B8B81813058F0CD
:10143000833020F08450823030F402C083E001C059
:1014400088E08F8B01C01E8ADF91CF911F91089594
:101450009C01FB018130910569F0823091051CF4FB
:101460000097D9F027C083309105F1F085309105C0
:1014700009F517C08EEF9FEF928F818F4091A906DB
:101480005091AA06CA0101978050944018F45583E0
:10149000448310C0358324830DC0CB010E94AC89E6
:1014A00009C081E0838306C083E090E040E050E023
:1014B0000E944A8980E090E008951F93182F81E0F0
:1014C00060E00E94C31E113049F0113028F0123044
:1014D00039F0133071F406C083E105C084E103C024
:1014E00085E101C086E10E94D566BC0182E00E94D0
:1014F00097201F9108951F93CF93DF93EB018230C4
:10150000910509F493C0833091051CF4892B31F0C7
:10151000BBC0863091050CF0B7C075C081E060E0BB
:101520000E94C31E8A818823A1F000D000D00F92B0
:10153000EDB7FEB7319682E0ADB7BEB711968C938A
:101540008AE898E1928381838C819D81948383834F
:1015500046C020919A0630919B0640919C0650917E
:101560009D06211531054105510509F440C08DB78F
:101570009EB707970FB6F8949EBF0FBE8DBFEDB70D
:10158000FEB7319612E0ADB7BEB711961C9382E854
:1015900098E19283818323833483458356830E9419
:1015A0003D206C817D818DB79EB707960FB6F8946C
:1015B0009EBF0FBE8DBF6115710509F465C000D0D7
:1015C00000D00F92EDB7FEB73196ADB7BEB711960A
:1015D0001C938DE798E192838183748363830E94D7
:1015E0003D200F900F900F900F900F904DC08C8169
:1015F0009D8197FF49C084E00E94D566BC0182E0CE
:101600000E94972041C08330910551F410929A06B0
:1016100010929B0610929C0610929D061D821C82C1
:10162000BE0142E050E00E944A892EC08A81882390
:1016300071F41D821C8283E08B838FEF9FE39F8375
:101640008E8391E0988F85E08F8B9E8B17C01E8ACA
:101650008C819D810E946F9E60939A0670939B0679
:1016600080939C0690939D061B82611571058105F0
:10167000910521F48FEF9FEF9D838C8390E08A8109
:10168000882309F491E09A8380E090E0DF91CF9184
:101690001F910895FF920F931F93CF93DF93EC0157
:1016A0008B01F42E0E940567FC01C230D10509F4BC
:1016B0008BC0C330D10534F42097D1F0219709F0C5
:1016C0009BC00DC0C430D10509F463C0C430D1053E
:1016D0000CF463C0C530D10509F08EC05EC0FF2098
:1016E00019F08485D8016DC08385F801818384C099
:1016F00081E060E00E94C31EFF2059F1D8011196DD
:101700002C91EDB7FEB737970FB6F894FEBF0FBE1A
:10171000EDBF319682E0ADB7BEB711968C9385E9E7
:1017200098E192838183822F6AE00E94009F8383E5
:101730001482822F0E94009F958316820E943D2072
:10174000EDB7FEB737960FB6F894FEBF0FBEEDBFEC
:1017500053C000D000D00F92EDB7FEB7319682E0B3
:10176000ADB7BEB711968C938FE898E192838183D1
:10177000D80111968C9122E3829FC0011124948399
:1017800083830E943D200F900F900F900F900F9039
:1017900033C0F80181818F3F79F1FF2019F44BEEBE
:1017A0005FEF02C040E05FEFCE01B8010E944A89BE
:1017B000FF2011F1D80111968C9111978823E1F443
:1017C00081E011968C9318C0D80112968C911297D3
:1017D000882349F011968C91FF2011F0848701C075
:1017E00083870E94716990E0F8018281882309F45F
:1017F00091E0D80112969C9380E090E0DF91CF9128
:101800001F910F91FF90089541E00E944A8B089527
:1018100040E00E944A8B08951F93CF93DF93EB0122
:1018200082309105C1F18330910534F40097C1F005
:10183000019709F04CC005C0863091050CF047C0F7
:1018400025C00E940567FC01808185FF02C082E0FF
:1018500003C084FF03C081E0898339C0198237C087
:1018600081E060E00E94C31E8981825F0E94D5668C
:1018700000D00F9222E0EDB7FEB7218393838283DD
:101880000E943D200F900F900F9021C043E050E048
:101890000E944A891CC08A81882399F00E940567AA
:1018A000FC0110811F7C8981813011F4106103C01B
:1018B000823009F410620E940567FC0110830E94C7
:1018C000716990E08A81882309F491E09A8380E02D
:1018D00090E0DF91CF911F910895CF93DF93EB01BB
:1018E0008230910581F1833091052CF4009781F0CD
:1018F0000197C9F504C086309105ACF51FC00E9460
:101900000567FC0187818983843068F119822BC0C7
:1019100081E060E00E94C31E8981865F0E94D566D7
:1019200000D00F9222E0EDB7FEB72183938382832C
:101930000E943D200F900F900F9015C044E050E0A2
:101940000E944A8910C08A81882339F00E94056765
:101950002981FC0127830E94716990E08A81882394
:1019600009F491E09A8380E090E0DF91CF910895AF
:101970001F93CF93DF939C01EB018230910509F413
:1019800084C0833091053CF4009749F18130910582
:1019900009F0AEC005C0863091050CF0A9C070C03A
:1019A0008C819D8101978C5F934010F03D832C8347
:1019B0008CEF93E09F838E8311E01B831E8B83E06B
:1019C0008F8B188F8C819D810197880F991F0E94A2
:1019D0009C9E1982039709F08BC0198389C081E00E
:1019E00060E00E94C31E8B81813079F52C813D819E
:1019F0008DB79EB707970FB6F8949EBF0FBE8DBFE9
:101A0000EDB7FEB7319682E0ADB7BEB711968C93B5
:101A100080EA91E092838183348323832D5F3F4F5B
:101A2000368325830E946A208DB79EB707960FB62E
:101A3000F8949EBF0FBE8DBF89818C5F0E947C662B
:101A4000BC0182E00E94972053C000D000D00F92CA
:101A5000EDB7FEB7319682E0ADB7BEB711968C9365
:101A60008AEA91E0928381838C819D819483838330
:101A70000E946A200F900F900F900F900F9038C027
:101A800042E050E00E944A8933C08A81882399F05D
:101A90002C813D818981882319F461E070E002C0C6
:101AA00063E070E021503040C901880F991F0E9407
:101AB000999E1A821DC08B81813019F48A831E8AF7
:101AC00017C08C819D8101978C7F01969D838C83AB
:101AD0000197880F991F0E949C9E1982039711F409
:101AE00081E0898391E09B839E8B83E08F8B988F2D
:101AF00080E090E0DF91CF911F910895CF93DF9325
:101B0000EB018230910541F1833091052CF400976F
:101B100089F00197E9F504C086309105CCF517C02E
:101B200080E090E00E949C9E1982039789F581E0F5
:101B300089832EC081E060E00E94C31E89818E5F90
:101B40000E947C66BC0182E00E94972021C042E096
:101B500050E00E944A891CC08A81882399F081E064
:101B600060E00E94C31E82E06DE978E10E94972048
:101B70008981882319F481E090E002C083E090E03D
:101B80000E94969E90E08A81882309F491E09A83CE
:101B900080E090E0DF91CF910895CF93DF93EB0148
:101BA0008230910509F450C08330910534F40097D8
:101BB00069F0019709F054C005C0863091050CF01A
:101BC0004FC03DC00E94B09E89834AC081E060E062
:101BD0000E94C31E69816623A9F48CE10E94D56628
:101BE00000D00F9222E0ADB7BEB711962C9311979B
:101BF00013969C938E9312970E943D200F900F9006
:101C00000F902EC000D000D00F92EDB7FEB73196E6
